:100000000C94190D0C943E0D0C943E0D0C943E0D69
:100010000C943E0D0C943E0D0C943E0D0C943E0D34
:100020000C943E0D0C943E0D0C94F00F0C943E0D70
:100030000C943E0D0C943E0D0C943E0D0C943E0D14
:100040000C943E0D0C943E0D0C943E0D0C943E0D04
:100050000C943E0D0C943E0D0C943E0D0C943E0DF4
:100060000C943E0D0C943E0D0C943E0D0C943E0DE4
:100070000C943E0D0C943E0D0C943E0D0C943E0DD4
:100080000C943E0D0C943E0D0C945F2B0C947C3420
:100090000C943E0D0C943E0D0C943E0D0C943E0DB4
:1000A0000C943E0D0C943E0D0C943E0D0C943E0DA4
:1000B0000C943E0D0C943E0D0C943E0D0C942C2C87
:1000C0000C943E0D0C94BF2F0C94E4350C943E0D13
:1000D0000C943E0D0C943E0D0C943E0D0C943E0D74
:1000E0000C943E0D0C943E0D0C94D51C0C943E0DBE
:1000F0000C943E0D0C943E0D0C943E0D0C943E0D54
:100100000C943E0D0C943E0D0C943E0D0C943E0D43
:100110000C94BD350C949A2F0C943E0D0C943E0D0E
:100120000C943E0D0C943E0D0C943E0D0C943E0D23
:100130000C943E0D0C943E0D0C943E0D0C94952B9E
:100140000C94770D0C94CC2E0C94A5340C943E0D8D
:100150000C943E0D0C94112F0C941A360C943E0DF9
:100160000C943E0D0C943E0D0C943E0D0C943E0DE3
:100170000C943E0D0C943E0D0C943E0D0C943E0DD3
:100180000C943E0D0C943E0D0C943E0D0C943E0DC3
:100190000C943E0D0C943E0D0C943E0D0C943E0DB3
:1001A0000C943E0D0C943E0D0C943E0D0C943E0DA3
:1001B0000C943E0D0C943E0D0C943E0D0C943E0D93
:1001C0000C943E0D0C943E0D0C943E0D0C943E0D83
:1001D0000C943E0D0C943E0D0C943E0D0C943E0D73
:1001E0000C943E0D0C943E0D0C943E0D0C943E0D63
:1001F0000C943E0D0C9431730C943E0D6364696E47
:100200006F70737578585B001E03430068006100CF
:100210006D0065006C0065006F006E002D004D00E4
:1002200069006E00690000002A034B006100730042
:100230007000650072002000260020004F0073004F
:10024000770061006C006400200047006D006200D0
:10025000480000000403090409023E00020100C036
:10026000320904000001020201000524001001040B
:100270002402060524060001070582030800FF0981
:10028000040100020A00000007050402100005072F
:100290000583021000051201100102000008D016AB
:1002A000B20401000102DC01AF10B010B110B210B5
:1002B000B310B410A910AA10AE10AD1000000001C8
:1002C00000ED2C6E2D8D2D663982398C39A9108D5B
:1002D000399E3DB13D4000070001ED2C6E2D8D2D66
:1002E000F03886398C39A9108D399E3DB13DC0005A
:1002F000070001ED2C6E2D8D2D7A3982398C39A9AC
:10030000108D399E3DB13D5000070001ED2C6E2D42
:100310008D2D7E3982398C39A9108D399E3DB13DA4
:10032000A400070001ED2C6E2D8D2D8E3EA83FAC54
:100330003FA910AD3FA347BF474001040001ED2C8A
:100340006E2D8D2DDE3EA83FAC3FA910AD3FA347DB
:10035000BF470004040001ED2C6E2D8D2D063FA833
:100360003FAC3FA910AD3FA347BF470004070001C2
:10037000ED2C6E2D8D2D173FA83FAC3FA910AD3F42
:10038000A347BF470010040001ED2C6E2D8D2D3FBB
:100390003FA83FAC3FA910AD3FA347BF47001007A0
:1003A0000001ED2C6E2D8D2D503FA83FAC3FA910C4
:1003B000AD3FA347BF470004040001ED2C6E2D8D17
:1003C0002D7D3FA83FAC3FA910AD3FA347BF4700DD
:1003D00010040001D4369137B237595E675E6C5E07
:1003E0006D5E6F5EAE10AD100000000100322EBADF
:1003F0002E5B3097569A56A756A8564D59AE10AD5B
:100400001000000000003962BC62EF626E6371632D
:100410007463756376635A6461640020080005396B
:1004200062BC62EF62B210B310B410A910AA10AE91
:1004300010AD1000000001003962BC62EF62686418
:100440006B646E646F6470646A6671660020080095
:10045000053962BC62EF6278669666A466A566C5D9
:1004600066B76616682C000800053962BC62EF6248
:100470004269596969696A691E6DB06C3B6ED0004A
:10048000080005004E4F4E4500000000000000002F
:10049000000000000000000000000000000000005C
:1004A00000000000014D465F554C5452414C4947F5
:1004B00048540000000000000000000000000000A0
:1004C0000000000000034D465F554C5452414C491A
:1004D0004748545F4556315F383042000000000005
:1004E000000000000000044D465F554C5452414C42
:1004F000494748545F4556315F3136344200000069
:1005000000000000000000024D465F554C5452416F
:100510004C494748545F43000000000000000000C1
:100520000000000000000000054D465F434C4153B1
:100530005349435F4D494E495F344200000000007B
:10054000000000000000000000064D465F434C41E3
:10055000535349435F314B0000000000000000008E
:1005600000000000000000000000074D465F434C03
:1005700041535349435F314B5F3742000000000055
:100580000000000000000000000000084D465F432E
:100590004C41535349435F344B00000000000000BE
:1005A000000000000000000000000000094D465F50
:1005B000434C41535349435F344B5F374200000083
:1005C000000000000000000000000000000A4D468E
:1005D0005F444554454354494F4E5F314B00000042
:1005E00000000000000000000000000000000B4DB3
:1005F000465F444554454354494F4E5F344B0000D9
:100600000000000000000000000000000000000CDE
:1006100049534F3134343433415F534E49464600D9
:1006200000000000000000000000000000000000CA
:100630000D49534F3134343433415F5245414445C1
:100640005200000000000000000000000000000058
:10065000000E564943494E4954590000000000001D
:10066000000000000000000000000000000000008A
:1006700000000F49534F31353639335F534E4946E9
:100680004600000000000000000000000000000024
:1006900000000010534C3253323030320000000062
:1006A000000000000000000000000000000000004A
:1006B0000000000011544954414749545354414EDD
:1006C000444152440000000000000000000000000F
:1006D000000000000012454D3432333300000000AA
:1006E000000000000000000000000000000000000A
:1006F00000000000000001000001000101000001F5
:1007000001000100000100010100010000010100E1
:1007100000010001010000010100010000010100D1
:1007200000010001010001000001000101000001C1
:1007300001000100000100010100010000010100B1
:1007400000010001010001000001000101000001A1
:100750000100010000010100000100010100000191
:100760000100010000010001010001000001010081
:100770000001000101000001010001000001010071
:100780000001000101000100000100010100000161
:100790000100010000010100000100010100000151
:1007A0000100010000010001010001000001010041
:1007B0000001000101000100000100010100000131
:1007C0000100010000010001010001000001010021
:1007D0000001000101000001010001000001010011
:1007E0000001000101000100000100010100000101
:1007F000010001000001008040C020A060E01090D6
:1008000050D030B070F0088848C828A868E8189818
:1008100058D838B878F8048444C424A464E4149400
:1008200054D434B474F40C8C4CCC2CAC6CEC1C9CB8
:100830005CDC3CBC7CFC028242C222A262E21292DC
:1008400052D232B272F20A8A4ACA2AAA6AEA1A9AB8
:100850005ADA3ABA7AFA068646C626A666E61696A0
:1008600056D636B676F60E8E4ECE2EAE6EEE1E9E58
:100870005EDE3EBE7EFE018141C121A161E111919A
:1008800051D131B171F1098949C929A969E9199988
:1008900059D939B979F9058545C525A565E5159570
:1008A00055D535B575F50D8D4DCD2DAD6DED1D9D28
:1008B0005DDD3DBD7DFD038343C323A363E313934C
:1008C00053D333B373F30B8B4BCB2BAB6BEB1B9B28
:1008D0005BDB3BBB7BFB078747C727A767E7179710
:1008E00057D737B777F70F8F4FCF2FAF6FEF1F9FC8
:1008F0005FDF3FBF7FFF004E4F4E4500000000000E
:1009000000000000000000000000000000000000E7
:1009100000000000000000015549445F52414E4470
:100920004F4D00000000000000000000000000002B
:100930000000000000000000025549445F4C45469D
:10094000545F494E4352454D454E5400000000004F
:10095000000000000000000000035549445F5249B8
:100960004748545F494E4352454D454E54000000A0
:1009700000000000000000000000045549445F4CE6
:100980004546545F44454352454D454E5400000092
:100990000000000000000000000000055549445F11
:1009A00052494748545F44454352454D454E5400D3
:1009B0000000000000000000000000000643594352
:1009C0004C455F53455454494E47530000000000C6
:1009D0000000000000000000000000000007435974
:1009E000434C455F53455454494E47535F44454338
:1009F000000000000000000000000000000008539C
:100A0000544F52455F4D454D00000000000000006E
:100A100000000000000000000000000000000009CD
:100A2000524543414C4C5F4D454D000000000000D5
:100A300000000000000000000000000000000000B6
:100A40000A544F47474C455F4649454C4400000017
:100A50000000000000000000000000000000000096
:100A6000000B53544F52455F4C4F470000000000AD
:100A70000000000000000000000000000000000076
:100A800000000C434C4541525F4C4F4700000000B2
:100A90000000000000000000000000000000000056
:100AA0000000000D434C4F4E4500000000000000C8
:100AB0000000000000000000000000000000000036
:100AC00000000000004F464600000000000000004B
:100AD0000000000000000000000000000000000016
:100AE0000000000000014D454D4F5259000000002C
:100AF00000000000000000000000000000000000F6
:100B0000000000000000024C4956450000000000B3
:100B100000000000000000000000000000000000D5
:100B200000000000000000004E4F4E450000000095
:100B300000000000000000000000000000000000B5
:100B4000000000000000000001504F57455245448E
:100B50000000000000000000000000000000000095
:100B6000000000000000000000025445524D494EB4
:100B7000414C5F434F4E4E0000000000000000005B
:100B800000000000000000000000035445524D49E1
:100B90004E414C5F525854580000000000000000C5
:100BA0000000000000000000000000045345545401
:100BB000494E475F4348414E474500000000000052
:100BC000000000000000000000000000054D454D41
:100BD0004F52595F53544F524544000000000000EB
:100BE00000000000000000000000000000064D456D
:100BF0004D4F52595F4348414E4745440000000065
:100C00000000000000000000000000000000084399
:100C10004F4445435F5258000000000000000000B0
:100C200000000000000000000000000000000009BB
:100C3000434F4445435F545800000000000000004B
:100C400000000000000000000000000000000000A4
:100C5000074649454C445F44455445435445440088
:100C60000000000000000000000000000000000084
:100C7000000A4C4F474D454D5F46554C4C00000017
:100C80000000000000000000000000000000000064
:100C9000000025632C25630025632C256300256354
:100CA0002C256300496E76616C696420426175642D
:100CB000726174652E0D0A55736520446566617511
:100CC0006C742062617564726174652034363038EA
:100CD00030302E0D0A0053657420256C6420457257
:100CE000726F722E0D0A00256C640025632C25633B
:100CF0000025356400416E7920696E746567657200
:100D00002066726F6D203020746F2025752E205262
:100D100065666572656E636520766F6C7461676584
:100D20002077696C6C2062652028564343202A2076
:100D30005448524553484F4C44202F2034303935C5
:100D400029206D562E002575002535640030203D84
:100D5000206E6F2074696D656F75740D0A312D36C4
:100D60003030203D20313030206D73202D20363042
:100D7000303030206D732074696D656F7574002597
:100D800075206D730025342E345800253575206D7F
:100D900056002575202866726F6D20776869636834
:100DA000202575206E6F6E2D766F6C6174696C6591
:100DB000290025750025750025632C256300524107
:100DC0004E444F4D004E4F205549442E004368611C
:100DD0006D656C656F6E4D696E6920526576472052
:100DE000636F6D70696C65642061742025532025E4
:100DF0005328255329207573696E67204C55464149
:100E00002025532077697468204156522D4743436B
:100E10002025532E00323032302D30362D32320024
:100E200031313A30383A3434003461633731353453
:100E30000031353131313500352E342E30000D0A78
:100E4000000D0A000D0A000D0A000D0A000D0A002F
:100E5000643130303A4F4B000000000000000000C9
:100E60000000000000000000000000000000000082
:100E700000653130313A4F4B205749544820544592
:100E800058540000000000000000000000000000B6
:100E900000006E3131303A57414954494E4720469F
:100EA0004F5220584D4F44454D00000000000000B7
:100EB000000000C83230303A554E4B4E4F574E204E
:100EC000434F4D4D414E4400000000000000000023
:100ED00000000000C93230313A494E56414C494475
:100EE00020434F4D4D414E4420555341474500004E
:100EF0000000000000CA3230323A494E56414C4997
:100F00004420504152414D455445520000000000DC
:100F1000000000000000783132303A46414C534521
:100F200000000000000000000000000000000000C1
:100F300000000000000000793132313A545255452A
:100F400000000000000000000000000000000000A1
:100F50000000000000000000CB3230333A54494D0D
:100F6000454F555400000000000000000000000044
:100F700000000000000000000056455253494F4E4B
:100F8000000000000000000000000000000000E47D
:100F90001F434F4E4649470000000000000000007C
:100FA000000000000010200A205549440000000005
:100FB000000000000000000000000000007120326E
:100FC00020524541444F4E4C5900000000000000A3
:100FD0000000000000D920CD2055504C4F41440066
:100FE00000000000000000000006210000000000DA
:100FF00000444F574E4C4F41440000000000000099
:10100000000B210000000000005245534554000031
:10101000000000000000000000102100000000009F
:1010200000555047524144450000000000000000B8
:10103000001B210000000000004D454D53495A455A
:10104000000000000000000000000000000000267A
:101050002155494453495A45000000000000000052
:10106000000000000000003E2152425554544F4EF3
:10107000000000000000000000000000005C21549F
:101080002152425554544F4E5F4C4F4E4700000082
:1010900000000000007B2173214C425554544F4EF8
:1010A000000000000000000000000000009A2192F3
:1010B000214C425554544F4E5F4C4F4E4700000058
:1010C0000000000000B921B1214C4544475245457C
:1010D0004E000000000000000000000000D721D0FA
:1010E000214C45445245440000000000000000002F
:1010F0000000000000F321EC214C4F474D4F4445C8
:10110000000000000000000000000000000E2208A7
:10111000224C4F474D454D000000000000000000EC
:101120000000000000000025224C4F47444F574E5E
:101130004C4F414400000000004B22000000000022
:10114000004C4F4753544F52450000000000000030
:101150000050220000000000004C4F47434C454126
:1011600052000000000000000054220000000000B7
:101170000053455454494E47000000000000000051
:1011800000000000005D225822434C4541520000FF
:1011900000000000000000000065220000000000C8
:1011A0000053544F524500000000000000000000B2
:1011B000006922000000000000524543414C4C00F1
:1011C0000000000000000000006D22000000000090
:1011D000004348415247494E4700000000000000CC
:1011E00000000000000000712248454C5000000043
:1011F0000000000000000000007922000000000054
:10120000005253534900000000000000000000009D
:1012100000000000000000B5225359535449434BCD
:10122000000000000000000000000000000000E8D6
:101230002253454E445F5241570000000000000019
:101240000000008E230000000053454E44000000C3
:101250000000000000000000000000042300000067
:1012600000474554554944000000000000000000BC
:10127000004A2400000000000044554D505F4D46D8
:101280005500000000000000002D240000000000B8
:10129000004944454E5449465900000000000000F2
:1012A00000672400000000000054494D454F55548C
:1012B00000000000000000000000000000A42484E2
:1012C000245448524553484F4C440000000000004D
:1012D00000000000001125F7244155544F43414CB4
:1012E000494252415445000000A42500000000007E
:1012F000004649454C44000000000000000000008A
:10130000000000000066259025434C4F4E4500002C
:10131000000000000000000000D0250000000000D8
:10132000005549444D4F44450000000000000000B6
:1013300000000000006B269C2653414B4D4F444556
:1013400000000000000000000000000000A426EAE9
:101350002600000000000000000000000000000067
:101360000000000000000000004C45444D4F444583
:101370000000000000000000000000000024265FC4
:1013800026444554454354494F4E00000000000098
:101390000000000000DB3ED53E424155445241541E
:1013A000450000000000000000000000000000E711
:1013B0002553414B3A09005549443A0900415451DB
:1013C000413A090054686572652069732061742090
:1013D0006C65617374206F6E65206D6F726520633C
:1013E00061726420747970652063616E6469646100
:1013F00074652C206275742074686572652077614D
:1014000073206E6F7420656E6F75676820746572E7
:101410006D696E616C2062756666657220737061BD
:1014200063652E0D0A000D0A000400010901000089
:1014300000000000000000000000000000000000AC
:101440004E585000000000000000000000000000A6
:101450004D4946415245204D696E6900000000002B
:10146000000000000000000000000000000000007C
:10147000000000000000000000000000000000006C
:10148000000000000000000000000000000000005C
:10149000040001080100000000000000000000003E
:1014A000000000000000004E585000000000000046
:1014B000000000000000004D494641524520436CA9
:1014C000617373696320316B00000000000000004D
:1014D000000000000000000000000000000000000C
:1014E00000000000000000000000000000000000FC
:1014F00000000000000000020001180100000000D0
:1015000000000000000000000000000000004E5835
:1015100050000000000000000000000000004D49E5
:101520004641524520436C617373696320346B00FC
:1015300000000000000000000000000000000000AB
:10154000000000000000000000000000000000009B
:101550000000000000000000000000000000440047
:101560000100010000000000000000000000000079
:1015700000000000004E5850000000000000000075
:1015800000000000004D494641524520556C7472E0
:10159000616C6967687400000000000000000000D2
:1015A000000000000000000000000000000000003B
:1015B000000000000000000000000000000000002B
:1015C00000000000004403012001757781028000C3
:1015D0000000000000000000000005004E58500010
:1015E0000000000000000000000000004D494641DE
:1015F00052452044455346697265000000000000D2
:1016000000000000000000000000000000000000DA
:1016100000000000000000000000000000000000CA
:101620000000000000000000000000004403012052
:1016300001757781028000000000000000000000BA
:101640000005004E5850000000000000000000009F
:101650000000004D494641524520444553466972B9
:101660006520455631000000000000000000000029
:10167000000000000000000000000000000000006A
:10168000000000000000000000000000000000005A
:1016900000000004030128013877B14A434F50335A
:1016A0003100000000000000090149424D00000027
:1016B000000000000000000000004A434F5033319A
:1016C000000000000000000000000000000000001A
:1016D000000000000000000000000000000000000A
:1016E00000000000000000000000000000000000FA
:1016F0000000000000000000000048000120017808
:1017000077B1024A434F5076323431000000000C6A
:101710000149424D000000000000000000000000F0
:10172000004A434F5033312076322E342E310000A0
:1017300000000000000000000000000000000000A9
:101740000000000000000000000000000000000099
:101750000000000000000000000000000000000089
:101760000048000120013833B14A434F503431560C
:101770003232000000000C0149424D000000000020
:1017800000000000000000004A434F503431207632
:10179000322E3200000000000000000000000000B7
:1017A0000000000000000000000000000000000039
:1017B0000000000000000000000000000000000029
:1017C000000000000000000004000128013833B1CF
:1017D0004A434F503431563233310000000D014935
:1017E000424D000000000000000000000000004A20
:1017F000434F5034312076322E332E31000000001A
:1018000000000000000000000000000000000000D8
:1018100000000000000000000000000000000000C8
:1018200000000000000000000000000000000004B4
:10183000000188010000000000000000000000001E
:10184000000000000000496E66696E656F6E000062
:101850000000000000004D494641524520436C61A4
:101860007373696320316B0000000000000000000A
:101870000000000000000000000000000000000068
:101880000000000000000000000000000000000058
:1018900000000000000002000198010000000000AC
:1018A0000000000000000000000000000047656D1F
:1018B000706C75730000000000000000004D504384
:1018C0004F53000000000000000000000000000076
:1018D0000000000000000000000000000000000008
:1018E00000000000000000000000000000000000F8
:1018F00000000000000000000000000000000C01DB
:1019000000000000000000000000000000000000D7
:1019100000000000496E6E6F766973696F6E205229
:10192000265400004A6577656C0000000000000046
:1019300000000000000000000000000000000000A7
:101940000000000000000000000000000000000097
:101950000000000000000000000000000000000087
:10196000000000000200013801000000000000003B
:1019700000000000000000000000004E6F6B696175
:1019800000000000000000000000004D49464152E8
:101990004520436C617373696320346B202D20658F
:1019A0006D756C6174656420283632313220436C69
:1019B00061737369632900000000000000000000EB
:1019C00000000000000000000000000800013801D5
:1019D0000000000000000000000000000000000007
:1019E00000004E6F6B696100000000000000000005
:1019F00000004D494641524520436C617373696351
:101A000020346B202D20656D756C61746564202811
:101A100036313331204E46432900000000000000DB
:101A200000000000000000000000000000000000B6
:101A3000000011241FBECFEFCDBFDFE3DEBF00E00B
:101A40000CBF18BE19BE1ABE1BBE14E2A0E0B0E265
:101A5000EEE5FAEF00E00BBF02C007900D92A03C4C
:101A6000B107D9F71BBE2DE3A0ECB4E201C01D9273
:101A7000A531B207E1F7BFD10C942D7DA8C23BB7C9
:101A80008BBFFB01879196913BBF08953BB78BBFFE
:101A9000CB0142E20D94F00F3BB70B0143E20D94F2
:101AA000F00F3BB78BBFCB0145E20D94F00F3BB776
:101AB00046E208C02091CF0127FDFCCF22272093CA
:101AC000CA0108954093CA0128ED31E02093340003
:101AD0003093CB016091C4017091C5018091C60122
:101AE00099270895FC014093CA01849108950F92AB
:101AF00000240F932F933F934F935F930FB70F9350
:101B0000EF93FF93EAB1FBB15191442735B124B172
:101B1000569578F400928C080092000806E10A9528
:101B2000F1F700C001E00093000803E000938C0887
:101B300004C00AE10A95F1F700002150304019F481
:101B40000E94022F0CC04F5F477011F4519102C0E8
:101B500000C000C00AE00A95F1F700C0D9CFFF919C
:101B6000EF910F910FBF5F914F913F912F910F9187
:101B70000F901895F190E190D190C190B190A19003
:101B8000919081900B941B942B943B944B945B9479
:101B90006B947B948B949B94AB94BB94CB94DB948D
:101BA000EB94FB940895F801D894E4DF5894E2DFB5
:101BB000D894E0CFF801D894DDDF5894DBDFF8014A
:101BC000D894D8CFF801D894D5CFF8015894D2CF73
:101BD000F80170965894CEDFF8013896D894CADF91
:101BE000F8015894C7CFF8015894C4DFD894C2DFE5
:101BF000F8015894BFCFFF90EF90DF90CF90BF9047
:101C0000AF909F908F907F906F905F904F903F909C
:101C10002F90112408952F923F924F925F926F92CE
:101C20007F928F929F92AF92BF92CF92DF92EF926C
:101C3000FF920F931F93FB0171906190519041901F
:101C400031902190119001908A01CDDFFC017192B9
:101C500061925192419231922192119201921F917F
:101C60000F91C9CF2F923F924F925F926F927F92C6
:101C70008F929F92AF92BF92CF92DF92EF92FF929C
:101C80000F931F93FC01719061905190419031909E
:101C90002190119001908A018DDFFB017192619278
:101CA0005192419231922192119201921F910F9182
:101CB000A2CF2F923F924F925F926F927F928F921C
:101CC0009F92AF92BF92CF92DF92EF92FF92CF930B
:101CD000DF93EB01DA01BF01F9017190619051903E
:101CE00041903190219011900190F990E990D99014
:101CF000C990B990A990999089907F246E245D2411
:101D00004C243B242A2419240824FB0109957D92A4
:101D10006D925D924D923D922D921D920D92019782
:101D200021F7D9017D926D925D924D923D922D9257
:101D30001D920D92DF91CF915ECF2F923F924F92E5
:101D40005F926F927F928F929F92AF92BF92CF924B
:101D5000DF92EF92FF92CF93DF93EB01DA01BF01A5
:101D6000788069805A804B803C802D801E800F8057
:101D7000FB010995F901F190E190D190C190B190EA
:101D8000A190919081907F246E245D244C243B246B
:101D90002A2419240824F990E990D990C990B9907F
:101DA000A99099908990F901F192E192D192C19212
:101DB000B192A192919281927D926D925D924D929B
:101DC0003D922D921D920D92019751F6DF91CF9188
:101DD00012CFFDE0EAED6DCFFDE0EAEDAECFFDE024
:101DE000E3EF67CFFDE0E3EFA8CFFDE0E3ED61CFE8
:101DF000FDE0E8EEA2CF0DD10E94311A0E94131B24
:101E000099D40E94AB3E1092520684E08093420621
:101E100082E680938601C1E0C0932606C093210626
:101E200086E080932206C093310612E010933206BA
:101E300010922A0610922B068FE08093290689E5DE
:101E4000809380019AE5909381018093820180E4E0
:101E500080934106809346069091B200907F9093C4
:101E6000B2009091B20092609093B20090E3909390
:101E700041069093460680935006C0934606109301
:101E8000450603E00093410683E18093010821E0C9
:101E900030E02093260830932708209328083093B9
:101EA000290810928C0880938008109223031092C6
:101EB0002103D8E0D093220381E180932003E091B5
:101EC000F033F091F13382859385809338039093BA
:101ED00039038CE380938203D09380038093830340
:101EE000D09381036FD10E94811FD4D1C4D7C093F6
:101EF0000002109201021093020200930402C093A8
:101F00002002D09321020E94E3181ED10E94231EBA
:101F10000E946B1ECCD08823B9F00E94AF1BD0D199
:101F20000E94911FB0D70E94251AE091E233F091F0
:101F3000E33319950E94B7290E94831C0E94931EC7
:101F400061E181E00E94041B0E94781D0E94DF1E57
:101F50000E94851F0E94F017E091E033F091E13379
:101F60001995E091DA33F091DB331995D3CF292F0E
:101F700033272230310559F02330310569F0213003
:101F80003105E9F482E190E026E932E01CC08EE3FD
:101F900090E028E532E017C099278130910549F09B
:101FA00028F0029761F4E8E0F2E005C0E4E5F2E031
:101FB00002C0E8E2F2E0849190E09F0104C080E07A
:101FC00090E020E030E0FA012083318308951F92F1
:101FD0000F920FB60F92112408B60F9218BEFFCFC2
:101FE0001F920F920FB60F92112408B60F9218BECF
:101FF0008F939F938EB19FB186599F4F8EB99FB992
:102000009F918F910F9008BE0F900FBE0F901F9061
:1020100018958091780083FF0AC088E0809378004B
:1020200088ED84BF81E0809380000D94FE008BECEE
:10203000809352008091500088608093500080917E
:10204000510083FFFCCF82EC8093550080915000BB
:102050008061809350008091510084FFFCCF88ED17
:1020600084BF84E0809340001EB81FB881E0809355
:10207000430029E630E020930A0430930B042093B8
:102080000C0430930D04809300048093020480E8D4
:1020900080930001089588ED84BF81E080937900EA
:1020A000089588ED84BF8BE180938000089580912E
:1020B000030481FF09C08091010480FDFCCF82E010
:1020C0008093030481E0089580E00895809150009A
:1020D0008260809350008091510081FFFCCF82E0AC
:1020E0008093CA01EDE1F0E0E491E0936200ECE15D
:1020F000F0E0E491E09363001092CA0180E88093DD
:1021000065008BEB8093660080915600897F8093F9
:102110005600809156008460809356008091600044
:102120008160809360000895E0E4F0E084818E7F18
:102130008483E0E6F0E080818E7F8083E0E5F0E05C
:1021400080818D7F8083089587E08093A2007894BA
:102150000895089580E090E0089508950895089501
:1021600008950895089508950895CF93C82FE09194
:10217000D833F091D93319950E94EF29E091F033CB
:10218000F091F133C58389E1C89FB00111246855EE
:102190007D4F49E150E086ED93E30E94F07580E8C1
:1021A000CD3019F48093460602C080934506E09135
:1021B000D633F091D7331995E091DC33F091DD33CC
:1021C000CF91199449E150E068EA72E086ED93E31B
:1021D0000E94F075E0E4F6E080E881838683E09178
:1021E000F033F091F1338581C0CF0F931F93E091CD
:1021F000F033F091F1338B019C01458163E183E879
:1022000094E00E941F1C1F910F910895FF920F935D
:102210001F93CF93DF931F92CDB7DEB7F82E092F10
:102220009E012F5F3F4F482F592F63E183E894E0D1
:102230000E94371C182F8823F1F08091EF338830EB
:1022400018F089818D30B1F489818FDFEF2DF02F67
:1022500040E08191882319F04F5F4F31D1F7E09131
:10226000C524F091C624309731F06F2D702F81E195
:10227000199501C010E0812F0F90DF91CF911F9130
:102280000F91FF9008959B01AC0163E183E894E016
:102290000C945E1C08950C94E27508950F931F939F
:1022A000CF938C01C62FCC2339F00E94E275F80140
:1022B00081938F01C150F7CFCF911F910F91089556
:1022C0000E94E2750E94E2750E94E2750C94E2752C
:1022D000CF93DF93EC0161507109DA01420F531F74
:1022E000FC01CF018C1B9D0BA417B50721F41082B4
:1022F000DF91CF91089562307105C8F39D91392F18
:1023000032953F703A3010F4305D01C0395C308353
:102310009F709A3010F4905D01C0995C9183329661
:1023200062507109DECFCF93DF93EC01DA0120E038
:1023300030E05C91552351F111969C9111979923AE
:1023400039F12617370711F180ED850F8A3020F01B
:102350008FEB850F8630E0F480ED890F8A3020F016
:102360004FEB490F4630A0F4E52FF0E0513408F070
:10237000F797E295E07F913410F4982F01C09753BE
:102380009E2B99932F5F3F4F1296D3CFC90102C066
:1023900080E090E0DF91CF9108954115510509F457
:1023A00049C020E12093660623E02093A0092091F4
:1023B000A10927FFFCCF2091A0097093A0092091CB
:1023C000A10927FFFCCF2091A0096093A0092091CB
:1023D000A10927FFFCCF2091A00921E02093120141
:1023E00080931C0190931D0140931401509315019B
:1023F0001092220182EC94E28093280190932901AB
:1024000040932401509325018091100180688093AE
:10241000100180912001806880932001809110013B
:1024200087FDFCCF80E3809311018093210180E13F
:10243000809365060895CF92DF92EF92FF92CF933B
:10244000DF939091EF33983008F061C0C091EA3388
:10245000D091EB33209709F45AC080E1809366064F
:1024600086E08093A0098091A10987FFFCCF80912D
:10247000A00980E180936506000000008093660655
:1024800082E08093A0098091A10987FFFCCF809111
:10249000A0091092A0098091A10987FFFCCF80912B
:1024A000A0091092A0098091A10987FFFCCFC92E35
:1024B000D12CE12CF12C8DE0CC0CDD1CEE1CFF1C92
:1024C0008A95D1F78FEFE81AF80A8091A009C230F7
:1024D000D105D0F0C701B601D2DA8093A00980916E
:1024E000A10987FFFCCF8091A0099093A00980915A
:1024F000A10987FFFCCF8091A00982E0C80ED11C02
:10250000E11CF11C2297E3CF80E180936506E09106
:10251000F033F091F13385818D3029F0E091DC3397
:10252000F091DD3319958091010480FDFCCF82E0AC
:1025300080930304DF91CF91FF90EF90DF90CF90D5
:102540000895CF92DF92EF92FF92CF93DF93809125
:10255000EF33883038F0DF91CF91FF90EF90DF902C
:10256000CF9069CFC82ED12CE12CF12C8DE0CC0C72
:10257000DD1CEE1CFF1C8A95D1F78FEFE81AF80AD4
:10258000C1E2D0E0219739F395DAC701B6017EDACE
:1025900091DA8FEFD81AE80AF80AF4CFCF92DF92D7
:1025A000EF92FF920F931F934115E0E25E076105E2
:1025B000710508F06EC0C090EA33D090EB33E12C87
:1025C000F12C4C155D056E057F0508F062C06901B0
:1025D000E12CF12C00E010E220E030E0041B150BB0
:1025E000260B370BC016D106E206F30610F497014E
:1025F00086010115110509F44EC020E120936606FD
:1026000023E02093A0092091A10927FFFCCF20916E
:10261000A009252F33272093A0092091A10927FF86
:10262000FCCF2091A0094093A0092091A10927FF88
:10263000FCCF2091A00921E02093120180931C017E
:1026400090931D0100931401109315011092220123
:1026500082EC94E280932801909329010093240155
:102660001093250180911001806880931001809162
:1026700020018068809320018091100187FDFCCFAC
:1026800080E3809311018093210180E180936506AE
:1026900002C080E001C081E01F910F91FF90EF9098
:1026A000DF90CF9008958091CF0187FDFCCF0895F2
:1026B000FADF8091CF0181FF0BC086E38093CA01CE
:1026C000EBECF1E021E030E088ED90E084BF208386
:1026D0000895EF92FF920F931F93CF93DF93EC0136
:1026E0007B018A011092C201DEDFD701CE01800F8B
:1026F000911F26E048ED50E061E070E0EBECF1E086
:10270000C817D90779F0C093C0013D2F3F713093AE
:10271000C1012093CA0144BF60833091C4013D933D
:102720002196EECFC801DF91CF911F910F91FF90BD
:10273000EF90089541E050E061EC74E281E090E0B8
:10274000C8DF41E050E060EC74E280E090E0C1DF7F
:10275000E0E6F6E080E1858382E0868388E0858399
:102760008AE18183E0EAF9E01682178280EC8583B2
:1027700088E18483E0E0F1E0128A8BE6838B148A9F
:10278000158A20EA208F99E0918F128E148E158E73
:10279000168E84E0808B12A23CE633A314A215A20D
:1027A00010A611A612A624A795A716A680A3089581
:1027B0003F924F925F926F927F928F929F92AF92D1
:1027C000BF92CF92DF92EF92FF920F931F93CF931E
:1027D000DF938B01542E652E282F2F71722EEC0162
:1027E000C21BD10965DF5FDF83E38093CA011092CA
:1027F000C1011092C2017801052D162D85E3482EE6
:1028000098EDC92ED12C88248394912C3BECA32ED7
:10281000BB24B39443E3342E0115110501F17092EA
:10282000C001F70181917F018093C401015011091A
:1028300021F07394F0E27F12EFCFC093C0018D2F8F
:102840008F718093C1014092CA01C601F50184BF16
:102850008082A09628DF3092CA01712CDDCF852DB1
:10286000962DDF91CF911F910F91FF90EF90DF9008
:10287000CF90BF90AF909F908F907F906F905F9020
:102880004F903F900895EF92FF920F931F93CF9335
:10289000DF934115510509F480C08A01EB017C01E9
:1028A0008091C02481110DC06115704450F481E005
:1028B0008093C02441E050E060EC74E280E090E05E
:1028C00077DF80E18093660686E08093A00980919F
:1028D000A10987FFFCCF8091A00980E18093650664
:1028E000000000008093660682E08093A00980913A
:1028F000A10987FFFCCF8091A009D093A009809106
:10290000A10987FFFCCF8091A009C093A009809105
:10291000A10987FFFCCF8091A0091092120182ECDF
:1029200094E280931C0190931D0100931401109375
:10293000150180E180932201E0922801F0922901A3
:1029400000932401109325018091100180688093E9
:1029500010018091200180688093200180911001F6
:1029600087FDFCCF80E3809311018093210180E1FA
:1029700080936506CD2B41F4E091F033F091F13373
:1029800085818D3009F0F1DB61E186E0DF91CF9147
:102990001F910F91FF90EF9037C6DF91CF911F915C
:1029A0000F91FF90EF900895CF92DF92EF92FF92F8
:1029B0000F931F93CF93DF931091EF33183008F0EC
:1029C00071C0C091EA33D091EB33209709F46AC00B
:1029D0008091C024882309F465C01092C02441E08E
:1029E00050E060EC74E280E090E0E2DE80E1809311
:1029F000660683E08093A0098091A10987FFFCCF40
:102A00008091A0091092A0098091A10987FFFCCFB5
:102A10008091A0091092A0098091A10987FFFCCFA5
:102A2000C150DF4FCD2FDD27C12ED12CE12CF12C51
:102A30009DE0CC0CDD1CEE1CFF1C9A95D1F78FEFAE
:102A4000E81AF80A8091A009219748F133D82FD8C5
:102A500031D800E010E01092A0098091A10987FF11
:102A6000FCCF6091A00970E01092A0098091A109AB
:102A700087FFFCCF8091A009782BC8010DD81AD808
:102A80000E5F1F4F011581E0180729F7C701B60136
:102A900008D810D88FEFD81AE80AF80AD5CF80E105
:102AA0008093650660E186E0AFD563E185E0ACD553
:102AB0008091010480FDFCCF82E080930304DF91CC
:102AC000CF911F910F91FF90EF90DF90CF900895DD
:102AD000CF92DF92EF92FF920F931F93CF93DF93EA
:102AE0004115E0E25E076105710508F098C0C090ED
:102AF000EA33D090EB33E12CF12C4C155D056E05DB
:102B00007F0508F08CC06901E12CF12C00E010E297
:102B100020E030E0041B150B260B370BC016D10646
:102B2000E206F30610F4970186010115110509F478
:102B300076C06A017B01C92FD82F8091C0248111F2
:102B40000AC081E08093C02441E050E060EC74E270
:102B500080E090E02DDE80E18093660686E0809341
:102B6000A0098091A10987FFFCCF8091A00980E195
:102B700080936506000000008093660682E08093E3
:102B8000A0098091A10987FFFCCF96018091A0093F
:102B9000D092A0098091A10987FFFCCF8091A00964
:102BA000C092A0098091A10987FFFCCF8091A00964
:102BB0001092120182EC94E280931C0190931D010B
:102BC000009314011093150180E180932201D093AA
:102BD0002801C093290100932401109325018091BD
:102BE000100180688093100180912001806880939B
:102BF00020018091100187FDFCCF80E380931101BB
:102C00008093210180E180936506232B41F4E091BC
:102C1000F033F091F13385818D3009F0A6DA81E04F
:102C2000DF91CF911F910F91FF90EF90DF90CF90A8
:102C300008951F93CF93DF93CDB7DEB7A097CDBF95
:102C4000DEBF873009F4F5C078F4833009F468C03A
:102C500028F4813011F18230B9F106C1853009F4D0
:102C6000AEC008F482C0E3C08A3009F4E7C040F483
:102C7000883009F4E1C0893009F0F6C0DCDBF4C02B
:102C80008C3009F4EEC008F4EAC08D3009F0ECC0D5
:102C900088E194E20E94ED28E7C010E08091EC33D7
:102CA000181750F4F8DAE1E0F0E0EC0FFD1FE10F47
:102CB000F11D80831F5FF2CF8091EE33853009F0E4
:102CC000A1C080EE89839EC011E08091EC338730F3
:102CD00009F010E0E091E633F091E733CE01019680
:102CE00019954091EC3331E0141708F08BC0332371
:102CF000A9F0812F90E0E1E0F0E0EC0FFD1FE80F7C
:102D0000F91F208131E02F3F09F030E0E1E0F0E0F1
:102D1000EC0FFD1FE80FF91F2F5F20831F5FE4CF2B
:102D2000E091E633F091E733CE0101961995809159
:102D3000EC3341E0815008F465C04423D9F3282FD7
:102D400030E0E1E0F0E0EC0FFD1FE20FF31F9081B7
:102D500041E09F3F09F040E0E1E0F0E0EC0FFD1FB3
:102D6000E20FF31F9F5F9083E5CF11E08091EC337A
:102D7000873009F010E0E091E633F091E733CE01BF
:102D8000019619954091EC3331E01417D8F53323AF
:102D9000A1F0812F90E0E1E0F0E0EC0FFD1FE80FE3
:102DA000F91F208131E0211130E0E1E0F0E0EC0F8B
:102DB000FD1FE80FF91F215020831F5FE6CFE09130
:102DC000E633F091E733CE01019619958091EC330B
:102DD00041E08150B8F04423E1F3282F30E0E1E0F6
:102DE000F0E0EC0FFD1FE20FF31F908141E0911125
:102DF00040E0E1E0F0E0EC0FFD1FE20FF31F915027
:102E00009083E7CFE091E833F091E933CE0101966A
:102E10001995E091C524F091C624309729F140918D
:102E2000EC33BE016F5F7F4F83E119951DC081E0D8
:102E300001C080E0BCD318C0B7DD16C08091000887
:102E4000813021F490918C08933009F080E080FD6E
:102E500003C00E94792A08C00E949F2A05C086D21A
:102E600003C073D10E949D3EA096CDBFDEBFDF910F
:102E7000CF911F910895E0E0F6E080E6828388E13B
:102E8000868B858B0895CF93C0910806C095C6FFA9
:102E900012C08091C4248A3050F08A30E1F4E0916D
:102EA000F033F091F1338181C4DE8091C4248F5FCF
:102EB0008093C42410C08C2F807669F48091C42440
:102EC00081508A3030F4E091F033F091F133808119
:102ED000B0DE1092C424C5FF12C08091C3248A3092
:102EE00050F08A30D9F4E091F033F091F1338381DE
:102EF000A0DE8091C3248F5F8093C3240FC0C0766F
:102F000069F48091C32481508A3030F4E091F03329
:102F1000F091F13382818DDE1092C324CF91089518
:102F20009B01AC016EE086EF98E0C8C4E82FF0E0AA
:102F3000E151FC4C88E0638381503D968111FBCFC9
:102F400008950F931F939B01E091F033F091F133BB
:102F5000E80FF11D8A0140816EE086EF98E06FD4A2
:102F60001F910F9108950F931F93CF93DF931F929B
:102F7000CDB7DEB7082FAB019E012F5F3F4F6EE04C
:102F800086EF98E074D4182F882319F06981802F78
:102F9000CDDF812F0F90DF91CF911F910F91089579
:102FA0000895EF92FF920F931F93CF937B01C42F4D
:102FB0000EB11FB12091080430910904022B132B8C
:102FC0004AD78C2F48D7812F46D7802F44D76C2FD4
:102FD00070E0C701CF911F910F91FF90EF9062C7F2
:102FE00008953F924F925F926F927F928F929F923D
:102FF000AF92BF92CF92DF92EF92FF920F931F9307
:10300000CF93DF937C01E901C0900020D090012094
:10301000960122503843C901A0E0B0E04817590793
:103020006A077B0708F05FC0E2E0CE1AE0E4DE0A40
:103030002A013B014C0E5D1E611C711C481659068D
:103040006A067B0648F0241B350B8E01021B130B0E
:10305000E9013324339403C000E010E0312C460131
:10306000A12CB12C481559056A057B0510F5CA013C
:103070008E5F9F4B2A013B014C0E5D1E611C711C33
:10308000481459046A047B0428F4AE01BC01C7014A
:1030900084D918C0C41AD50AA601BC01C7017DD9BC
:1030A000AE014C195D096CEC74E2C7018C0D9D1DDD
:1030B00007C04C195D09BA0164537B4DAE01C701CD
:1030C0000E941E76332041F00C0F1D1FF701E00F08
:1030D000F11FCE0DDF1D02C081E006C0EC17FD0719
:1030E000D9F31292FBCF80E0DF91CF911F910F9126
:1030F000FF90EF90DF90CF90BF90AF909F908F9018
:103100007F906F905F904F903F9008952091C824DA
:103110003091C92480E098E0821B930BECECF4E240
:103120009F012C5C34422817390710F41192F8CF14
:103130008CEC94E28093CA249093CB2480E098E0B6
:103140008093C8249093C9240895E0DF82E090E43E
:10315000809300209093012042E050E060E070E412
:1031600080E090E290DB60E18AE04EC28091C8246A
:103170009091C92490592091002030910120821B08
:10318000930B0895EFEEF3E387833D9694E3E735E1
:10319000F907D1F7813049F018F0823059F00895DD
:1031A0001092C72480ED97E109C08093C72489E37A
:1031B00099E104C01092C72481ED97E18093C52462
:1031C0009093C6240895CF93DF931F92CDB7DEB7B7
:1031D000E091F033F091F1338481D4DFECECF4E250
:1031E000E093CA24F093CB2480E098E08093C82435
:1031F0009093C924DF019C011D9221503040E1F7DA
:1032000041E050E0BE016F5F7F4F82E090E061DA05
:1032100089818A3541F442E050E060E070E480E06A
:1032200090E2BBD817C082E090E480930020909396
:10323000012042E050E060E070E480E090E223DBB7
:103240008AE5898341E050E0BE016F5F7F4F82E0F5
:1032500090E0AEDAE091C524F091C624309729F0D1
:1032600040E060E070E08FEF19950F90DF91CF9113
:1032700008950F931F93CF93DF93CEB1DFB1A09149
:103280000804B09109042091C8243091C924E42F86
:10329000F0E08F010C5F1F4F2017310778F1CA2B28
:1032A000DB2B245031092E1B3F0B2093C824309375
:1032B000C924A091CA24B091CB248C9311964C932D
:1032C00011971296DC931297CD0104968093CA242D
:1032D0009093CB241396CC93DB01EC01415018F072
:1032E0002D912993FBCFE80FF91FE093CA24F093A7
:1032F000CB24DF91CF911F910F91089580E042DFA1
:1033000061E18AE0DF91CF911F910F917DC11F9301
:10331000CF93DF931F92CDB7DEB79E012F5F3F4F54
:10332000AC0163E084EC9AE0A2D2182F882311F05C
:10333000898128DF812F0F90DF91CF911F91089510
:103340000F931F93E091F033F091F1338B019C01C7
:10335000448163E084EC9AE072D21F910F9108954A
:103360009B01AC0163E084EC9AE0A8C20F931F9329
:10337000CF93DF938091C8249091C924811528E0D0
:10338000920708F05DC06091002070910120C0E0BC
:10339000D0E7C61BD70B00E018E0A801481B590B6B
:1033A000C417D507A0F08CEC94E26DDA8091002070
:1033B00090910120985F2091C8243091C924821BEC
:1033C000930B8093002090930120A0DE2EC02097C5
:1033D000B9F1AE018CEC94E256DAA8014C1B5D0BFE
:1033E000BE0164537B4D8CEC94E20E942776809161
:1033F000CA249091CB248C1B9D0B8093CA2490935C
:10340000CB248091C8249091C9248C0F9D1F809358
:10341000C8249093C9248091002090910120C80F66
:10342000D91FC0930020D093012042E050E060E01B
:1034300070E480E090E2DF91CF911F910F9123CA59
:10344000DF91CF911F910F9108958091C724811131
:103450008DCF089548E750E06FEE73E383E090E08E
:10346000A7C948E750E06FEE73E383E090E031D9FD
:103470008091EF33893068F42DE0829FC0011124E0
:103480008E509C4C2091F0333091F133281739073E
:1034900041F188E08093EF338AE594E38093F03341
:1034A0009093F133EFEEF3E397E086E071E064E0B0
:1034B00042E350E020E931E01086958383839683D0
:1034C000848317827187628743875487258736876D
:1034D0003D96A4E3E436FA0779F78DE080935F34F4
:1034E000B9CF0895EF92FF920F931F93CF93DF937D
:1034F0001F92CDB7DEB7082F80E3800F8983E0915C
:10350000C524F091C624309731F041E0BE016F5FD1
:103510007F4F82E119951FEF100F193008F03EC060
:103520000E94EF298091EF33181791F13DDA109343
:10353000EF332DE0129FC00111249C012E503C4C12
:103540002093F0333093F133FC01E151FC4C808542
:103550000E94B510E091F033F091F133848112DED6
:103560000E941B1283E090E09C012F5E334379019F
:103570006091EF33C90181519C4C0E94BF7C6091E6
:10358000F0337091F133C70180519C4C0E94C87C8C
:103590006FE1600F84E038D081E001C080E00F90DF
:1035A000DF91CF911F910F91FF90EF90089590912F
:1035B000EF3328E03DE0983018F02F5F90E006C030
:1035C000882311F09F5F01C0995F9770399FF001C8
:1035D0001124E151FC4C4085442319F081E0890F0E
:1035E00081CF215041F70895FC019091EF339F5C0A
:1035F000908311820895FC012181211103C08081F3
:10360000805370CF80E00895E091F033F091F13372
:103610009781981302C06093CD2C9681891302C0C4
:103620006093CC2C0895E0E0F6E088E1818381E0AE
:103630008283E0E8F6E092E0928382830895893005
:1036400008F04EC095E0899FF0011124ED5FFF4D19
:103650008081882321F080E18093050603C080E10A
:10366000809306068181882321F088E080930506F7
:1036700003C088E0809306068281811104C081E046
:103680008093060604C0813029F480930506809358
:10369000010603C081E0809302068381811104C08A
:1036A00082E08093860605C0813031F482E0809309
:1036B00085068093810603C082E080938206848120
:1036C000811104C081E08093860604C0813029F412
:1036D0008093850680938106089581E08093820619
:1036E0000895FB016D5C7C4219F0AEECBCE202C0B7
:1036F000AFECBCE29081923181F030F49031A1F0D6
:1037000048F4992359F129C0933151F090529930DE
:1037100070F023C08093050620C0809307061DC06B
:1037200090910406982371F08093060616C09C9130
:103730009F5F913011F09C9308951C929091040624
:10374000982319F4809305060895809306068081D6
:10375000803219F0815080830895108208958091FD
:103760003020811108C06CEC7CE280E1BADF6DECA6
:103770007CE288E0B6CF8091EF33909102208917E8
:1037800019F0809302205BCF08959B01AC016BE0A0
:1037900087E29BE093C0EFEEF3E398E0282F2870D8
:1037A0008071211162878111618791503D9691113D
:1037B000F8CF222329F098E0909306061092CD2CA2
:1037C000882329F080E1809306061092CC2C08957E
:1037D0000F931F939B018A01883031F4E091F033FD
:1037E000F091F133478107C0803149F4E091F03323
:1037F000F091F13346816BE087E29BE020D01F918E
:103800000F9108950F931F93CF93DF931F92CDB71E
:10381000DEB7082FAB019E012F5F3F4F6BE087E2C1
:103820009BE025D0182F882319F06981802FB3DF02
:10383000812F0F90DF91CF911F910F9108950F93DA
:103840001F93FC01662379F094916150941309C091
:10385000BF016F5F7F4FA801C9010E94027681E01E
:1038600003C0B196EFCF80E01F910F910895CF92E2
:10387000DF92EF92FF921F93CF93DF93EC017A01D7
:103880006901162F112389F0BE016F5F7F4FC701B9
:103890000E94F9751150892B31F4FE01C491F60193
:1038A000C08381E003C0A196EDCF80E0DF91CF918E
:1038B0001F91FF90EF90DF90CF900895CF930196E6
:1038C000CCE26623D1F0FC01DA01AD0174917723DB
:1038D00041F021153105A9F07D9331962150310930
:1038E000F4CF623038F02115310559F0FD01C08365
:1038F0004F5F5F4F61508196E4CF232B11F0FA01A7
:103900001082CF91089580912002806880932002D8
:103910008091230280FFFCCF81E080932302A0915D
:103920001002B0911102AE5BB109B7FF02C0A0E076
:10393000B0E020E038EB4BE050E00E947C75843F23
:10394000914060F460E187E05FDE8091EC33882392
:1039500041F0E091DE33F091DF33199461E187E0CB
:1039600053CE08958091D62E9091D72E2091D42EAB
:103970003091D52E2817390771F09C012F5F3F4FEA
:103980002093D62E3093D72E9170FC01EC52F14D3E
:10399000848190E008958FEF9FEF08959091A10AA0
:1039A00095FFFCCF8093A00A08951F920F920FB647
:1039B0000F92112408B60F9218BE09B60F9219BEC5
:1039C0000BB60F921BBE2F933F934F935F936F9352
:1039D0007F938F939F93AF93BF93EF93FF938091C8
:1039E000A10A8C7109F58091D42E9091D52E209149
:1039F000D62E3091D72EAC01421B530B9A012227B1
:103A00003E7F232B69F42091A00AFC01F170EC5257
:103A1000F14D248301968093D42E9093D52E0EC021
:103A200085E4BCDF80E306C085E4B8DF81E3B6DF70
:103A30008091A10AB3DF8091A00AB0DFFF91EF91DE
:103A4000BF91AF919F918F917F916F915F914F91B6
:103A50003F912F910F900BBE0F9009BE0F9008BEA3
:103A60000F900FBE0F901F9018950F931F93CF9339
:103A7000DF93EC018C01060F171FC017D10711F15E
:103A80008091D02C9091D12C2091D22C3091D32C9C
:103A9000AC01421B530B9A0122273E7F232B61F47A
:103AA0002881FC01F170E053F34D2483019680934B
:103AB000D02C9093D12C04C085E470DF82E36EDFBC
:103AC0002196DBCFDF91CF911F910F9108950F9336
:103AD0001F93CF938C01C62FCC2331F0F801819135
:103AE0008F015CDFC150F8CFCF911F910F910895E6
:103AF000BF92CF92DF92EF92FF920F931F93CF93DB
:103B0000DF93CDB7DEB7C454D109CDBFDEBF00917E
:103B1000D02C1091D12C8091D22C9091D32C081BB9
:103B2000190B95EAC92E25E7B22E01151105D1F121
:103B300078010134110518F080E4E82EF12CC982D7
:103B4000BA82DE2CEB821C826091D22C862F90915F
:103B5000D32C282F261B30E0AC014F5F5F4F2E1572
:103B60003F0570F4A5E0B0E0AC0FBD1FA20FB31F7E
:103B70009170FC01E053F34D84818C93CA01E9CF2D
:103B80008093D22C9093D32C60E070E0CE0101960C
:103B90008BD08C8364E06D0DCE01019698DF0E19F9
:103BA0001F09C3CFCC5BDF4FCDBFDEBFDF91CF910D
:103BB0001F910F91FF90EF90DF90CF90BF900895ED
:103BC000611524E8720723E08207910599F06115D9
:103BD00028E0720727E08207910589F0611522EC41
:103BE000720721E082079105D1F42EE62093A60A00
:103BF00023EA09C027E92093A60A21EA04C027E5A1
:103C00002093A60A21E92093A70A6093312070939C
:103C10003220809333209093342081E0089580E017
:103C200098E0A7E0B0E08093312090933220A093F9
:103C30003320B093342087E58093A60A81E98093EE
:103C4000A70A80E00895CF93DF93E4EDFEE21082AF
:103C50001182128213821482E0EDFCE21082118242
:103C6000128213821482E0E8F6E088E08183858383
:103C700084E0828388E1828BC0EADAE08D818F73F1
:103C80008D8383E08D8360E078E087E090E098DFCB
:103C90008C8188608C838C8180618C838B81806334
:103CA0008B83DF91CF910895FC016115710519F4A3
:103CB000BC016C5F7F4F928120818181820F890FCF
:103CC0008195362FFB012E2F231B291718F42191E4
:103CD000821BF9CF08951092D8301092D9301092EB
:103CE000673408950F931F93CF93DF938C01EB01FB
:103CF0008091DB30811112C0F8018281882371F03C
:103D000088810E942B27811103C088810E940D2980
:103D10002196F801828181508283EECFDF91CF918D
:103D20001F910F910895CF93DF93CDB7DEB7A6977C
:103D3000CDBFDEBF809135208F5F843118F4809332
:103D4000352022C01092352080914F208823E1F049
:103D500085EA898381E68A8382E28B8381E08D8391
:103D60001E8289E1E6E3F0E2DE01179601900D92F2
:103D70008A95E1F760E070E0CE01019695DF8C83D3
:103D800066E2CE010196A3DEA696CDBFDEBFDF912F
:103D9000CF91089580E00E94B51057DB80E18093B9
:103DA000050688E080930606D0E1C8E00E9457101F
:103DB0008823E1F3D0930706C0930706F7CFCF938C
:103DC000D1DD97FD46C02091D8303091D930F9012E
:103DD000E959FB4C80832115310521F4809167342A
:103DE000853A71F7C90101968093D8309093D93004
:103DF0008430910528F3209169342C3F28F530E078
:103E00002C5F3F4F82179307D8F2C0916A3460E06D
:103E100070E087E694E348DFC81316C080916834E9
:103E2000803769F0853729F0813671F410924F2080
:103E30000BC06BE674E387E694E354DF05C06BE6E2
:103E400074E387E694E3A6DF1092D8301092D9305D
:103E5000B7CFCF910895CF93DF931F92CDB7DEB741
:103E600089838091DB30882331F0698181E590E29C
:103E70000E94F27305C061E070E0CE010196F5DDAD
:103E80000F90DF91CF910895CF93DF93FC01849140
:103E9000EF012196882319F0DEDFFE01F8CFDF91D4
:103EA000CF9108952091DB30222331F0AB01BC018A
:103EB00081E590E20C94CE73D8CDFC0101900020F6
:103EC000E9F73197BF01681B790BECCFCF93DF93F4
:103ED00081E590E20E947774EC0197FD0FC081E0CC
:103EE0008093DB3063E183E08FDB8C2FB4D78111CB
:103EF00005C08C2FDF91CF910C940D29DF91CF91CC
:103F0000089580E28093620608958091DA308230CD
:103F100039F481E590E20E945B740E94636FD6CF12
:103F200008958091DA30813079F028F08230D9F02C
:103F3000833031F132C08091680685FF36C089E058
:103F40008093502081E00CC080915020815080935C
:103F5000502081112AC00E9466100E94FB7282E0EC
:103F60008093DA301AC08091680685FD1AC089E016
:103F70008093502083E08093DA301092DB300DC0C4
:103F80008091502081508093502081110EC00E945A
:103F9000C0720E9494101092DA308091DA30823030
:103FA00021F40E9462280C94B729089561E182E00F
:103FB0002BCB60E182E028CB81E590E20C94A973E1
:103FC00081E590E20C94CA7428E33EE03F932F937E
:103FD00021E33EE03F932F9329E23EE03F932F936E
:103FE00020E23EE03F932F9325E13EE03F932F9365
:103FF0002DEC3DE03F932F9322E02F931F929F9350
:104000008F930E9487768DB79EB740968DBF9EBFD7
:1040100085E6089560E072E00E94F51085E6089557
:10402000FB0120812F3349F42181211106C060E07A
:1040300072E00E94431185E60895CB010E940611AB
:10404000882371F0E091F033F091F133CF018A5E73
:10405000934365818D5F9F4F0E94BF7C84E60895E6
:104060008AEC0895EF92FF920F931F93CF93DF9303
:10407000CDB7DEB7A097CDBFDEBF7C010091EC339A
:1040800010E00115110591F485EC9DE09F938F934D
:1040900082E08F931F92FF92EF920E9487760F909B
:1040A0000F900F900F900F900F9010C0E091E6339B
:1040B000F091E733CE01019619959801AE014F5F5B
:1040C0005F4F60E072E0C7010E94681185E6A0962C
:1040D000CDBFDEBFDF91CF911F910F91FF90EF9089
:1040E0000895DF92EF92FF920F931F93CF93DF9388
:1040F000CDB7DEB7A097CDBFDEBF7B010091EC331B
:1041000010E06EEB7DE0C7010E94F975892BC1F4C8
:10411000D12CED2CF12CE016F10658F40E944B1135
:10412000E1E0F0E0EC0FFD1FEE0DFF1D8083D39466
:10413000F0CF8091EE33853069F480EE89830AC038
:10414000A70160E270E0CE0101960E94931108176A
:104150001907A9F4E091E833F091E933CE01019613
:104160001995E091C524F091C624309751F0409103
:10417000EC33BE016F5F7F4F83E1199502C08AEC7B
:1041800001C084E6A096CDBFDEBFDF91CF911F9125
:104190000F91FF90EF90DF900895FC018091ED3337
:1041A000882311F081E301C080E38083118285E6DA
:1041B0000895FB012181211127C02081213321F4A1
:1041C00081E08093ED3304C0203321F41092ED336D
:1041D00084E608952F33C1F41F9220E32F931F929A
:1041E00021E32F9328EB3DE03F932F9322E02F9381
:1041F0001F929F938F930E9487768DB79EB70A96E2
:104200008DBF9EBF85E608958AEC089588E695E106
:10421000F1D58EE608958EEC92E107D68EE60895EC
:10422000E0ECF4E081818E7F81830E94C0720E9465
:104230004B1084E60895E0ECF4E081818E7F818369
:104240000E94C0720E94511084E60895E6EDF3E3E7
:1042500025892F9324892F9325EB3DE03F932F93BE
:1042600022E02F931F929F938F930E9487768DB7A2
:104270009EB708968DBF9EBF85E608952091EC33CA
:104280001F922F9322EB3DE03F932F9322E02F9339
:104290001F929F938F930E9487768DB79EB7089643
:1042A0008DBF9EBF85E6089540E052E0BC0180E0EE
:1042B0000E94A11785E60895FB0120812F3349F460
:1042C0002181211106C060E072E00E94901785E60E
:1042D000089580E00E94B317882319F0BBD884E6C4
:1042E00008958AEC089540E052E0BC0181E00E940C
:1042F000A11785E60895FB0120812F3349F4218120
:10430000211106C060E072E00E94901785E60895D2
:1043100081E00E94B317882319F09CD884E60895A1
:104320008AEC089540E052E0BC0182E00E94A117AF
:1043300085E60895FB0120812F3349F42181211165
:1043400006C060E072E00E94901785E6089582E062
:104350000E94B317882319F07DD884E608958AEC6B
:10436000089540E052E0BC0183E00E94A11785E679
:104370000895FB0120812F3349F42181211106C0CA
:1043800060E072E00E94901785E6089583E00E9445
:10439000B317882319F05ED884E608958AEC08954F
:1043A00040E052E0BC0188E013DA85E60895FB01A5
:1043B00020812F3341F42181211105C060E072E09A
:1043C000E4D985E6089588E01DDA882319F042D8FB
:1043D00084E608958AEC089540E052E0BC0180E153
:1043E000F7D985E60895FB0120812F3341F421811F
:1043F000211105C060E072E0C8D985E6089580E12A
:1044000001DA882319F026D884E608958AEC089505
:1044100060E072E00E94A01985E60895FB0120810A
:104420002F3349F42181211106C060E072E00E941F
:10443000B01985E60895CB010E948719882319F0E9
:1044400009D884E608958AEC0895CF93DF93EC01B0
:104450000E94B618813028E0920718F09C0138506D
:1044600002C020E030E03F932F939F938F9382E927
:104470009DE09F938F9382E08F931F92DF93CF9362
:104480000E9487768DB79EB70A968DBF9EBF85E640
:10449000DF91CF91089581EF97E1C7D48EE608951B
:1044A0000E94B61984E608950E94A51884E608952E
:1044B00060E072E099D885E60895CB019CD881111F
:1044C00002C08AEC089584E608950E94A11284E651
:1044D00008950E94D41484E608950E941B1284E675
:1044E00008958091680680FD02C089E7089588E7F5
:1044F0000895DF92EF92FF920F931F93CF93DF9374
:10450000EC010FEF11E089E7E82E8FE0F82E9CE236
:10451000D92EB70183E394E20E94F975892BD1F07B
:1045200001151105B9F0DE01F7012491ED01219685
:10453000C8010197222341F00130110529F02C9385
:10454000DE0131968C01F1CFDC928C0188E1E80E1E
:10455000F11CDFCF2197188285E6DF91CF911F9163
:104560000F91FF90EF90DF900895FC018091200261
:104570008068809320028091230280FFFCCF81E03D
:1045800080932302A0911002B0911102AE5BB10999
:10459000B7FF02C0A0E0B0E020E038EB4BE050E015
:1045A0000E947C75AA27BB279F938F938BE89DE081
:1045B0009F938F9382E08F931F92FF93EF930E94BC
:1045C00087768DB79EB708968DBF9EBF85E6089506
:1045D0004EB15FB12091080430910904242B352B92
:1045E0003F932F9325E83DE03F932F9322E02F93B5
:1045F0001F929F938F930E9487768DB79EB70896E0
:104600008DBF9EBF85E608950F931F93CF93DF93D1
:104610001F921F92CDB7DEB78B01E091F033F0917E
:10462000F13385818D3009F06FC0E091DE33F09178
:10463000DF33199581E08093603160E270E0C8015A
:104640000E943F760097F9F4F80101900020E9F705
:104650003197E01BF10BE0FD59C0F695E795E1308D
:10466000F10539F487E090E08093D4339093D5330B
:1046700037C053E0EE0FFF1F5A95E1F7E093D433B4
:10468000F093D5332DC098012C5F3F4F82179307CD
:10469000E9F5A80162E070E0CE0101960E94931155
:1046A000898190E0982F88272A81820F911D80931D
:1046B000D4339093D5330B5F1F4FF8010190002046
:1046C000E9F73197E01BF10BE0FD20C0F695E79587
:1046D00033E0EE0FFF1F3A95E1F7E817F907B0F066
:1046E0006091D4337091D533695F7F4F83E07695C5
:1046F00067958A95E1F7A80182ED92E30E949311F4
:104700000E9452338FEF03C089EC01C08AEC0F90F6
:104710000F90DF91CF911F910F910895EF92FF922B
:104720000F931F93CF93DF931F921F92CDB7DEB7E6
:104730008B01E091F033F091F13385818D3009F0F8
:1047400080C0E091DE33F091DF33199582E08093F1
:10475000603160E270E0C8010E943F767C01892BE5
:1047600031F5F80101900020E9F73197E01BF10BDA
:10477000E0FD69C0F695E795E130F10539F487E091
:1047800090E08093D4339093D53347C053E0EE0F3D
:10479000FF1F5A95E1F7CF0169E070E00E9468754C
:1047A000E81BF90BE093D433F093D53336C0C8013E
:1047B0000496E816F90609F046C0A80162E070E028
:1047C000CE0101960E949311898190E0982F88274D
:1047D0002A81820F911D8093D4339093D5338730F3
:1047E000910529F09C0127703327232B61F5870160
:1047F0000F5F1F4FF80101900020E9F73197E01B90
:10480000F10BE0FD20C0F695E79533E0EE0FFF1FBA
:104810003A95E1F7E817F907B0F06091D433709159
:10482000D533695F7F4F83E0769567958A95E1F789
:10483000A80182ED92E30E9493110E9452338FEF00
:1048400003C089EC01C08AEC0F900F90DF91CF91EB
:104850001F910F91FF90EF900895E091F033F09148
:10486000F13385818D30A1F4E091DE33F091DF33B7
:10487000199585E0809360310E9497560E945233CB
:1048800081EA96E58093EA309093EB308FEF0895BC
:1048900089EC0895E091F033F091F13385818D300A
:1048A000A1F4E091DE33F091DF33199583E080933A
:1048B00060310E9497560E94523381EA96E58093B8
:1048C000EA309093EB308FEF089589EC0895E091F2
:1048D000F033F091F13385818D30A1F4E091DE3336
:1048E000F091DF33199586E0809360310E949756EE
:1048F0000E94523381EA96E58093EA309093EB3040
:104900008FEF089589EC0895E091F033F091F13341
:104910004085518564E6649F9001659F300D1124A8
:104920003F932F932FE73DE03F932F9322E02F9368
:104930001F929F938F930E9487768DB79EB708969C
:104940008DBF9EBF85E60895CF93DF931F921F9280
:10495000CDB7DEB7FB0120812F33B1F421812111C6
:1049600013C02DE43DE03F932F9322E02F931F923D
:104970009F938F930E9487760F900F900F900F90C8
:104980000F900F9085E62EC089E592E089839A8387
:10499000CE0101969F938F9389E49DE09F938F931F
:1049A0007F936F930E94BD760F900F900F900F90A2
:1049B0000F900F90892BA9F069817A816935F2E017
:1049C0007F0778F4E091F033F091F13360877187DD
:1049D000CF01875E93438D5F9F4F0E94C87C84E622
:1049E00001C08AEC0F900F90DF91CF910895E09174
:1049F000F033F091F13323852F9322852F9326E412
:104A00003DE03F932F9322E02F931F929F938F932C
:104A10000E9487768DB79EB708968DBF9EBF85E6AC
:104A20000895CF93DF931F921F92CDB7DEB7FB019E
:104A300020812F33B1F42181211113C02FE02F9356
:104A40002FEF2F9325EF3CE03F932F9322E02F93FE
:104A50001F929F938F930E948776CDBFDEBF85E61E
:104A600030C019821A82CE0101969F938F9381EFF5
:104A70009CE09F938F937F936F930E94BD760F90DE
:104A80000F900F900F900F900F90892BC9F06981B4
:104A90007A81611590E1790798F4609338037093F7
:104AA0003903E091F033F091F13362877387CF01DE
:104AB000855E93438D5F9F4F0E94C87C84E601C052
:104AC0008AEC0F900F90DF91CF910895FB01208128
:104AD0002F33D9F42181211121C01F9220E32F937C
:104AE0001F9221E32F932BEE3CE03F932F9322E084
:104AF0002F931F929F938F930E9487768DB79EB7B7
:104B00000A968DBF9EBF85E60895213311F4F1D436
:104B100003C0203319F413D584E608958AEC089570
:104B2000FC0180910008813029F480918C0891E08B
:104B3000833009F090E090FF02C081E301C080E380
:104B40008083118285E60895E091F033F091F1338E
:104B500085818D3079F4E091DE33F091DF33199562
:104B600084E0809360310E9497560E94523381EA1C
:104B700096E50EC08C3091F4E091DE33F091DF3396
:104B8000199581E080933C320E94595E8EE69EE545
:104B90008093EA309093EB308FEF089589EC08957D
:104BA0008DE00E94B510E091DE33F091DF3319956E
:104BB00087E0809360310E9497560E94523381EAC9
:104BC00096E58093EA309093EB308FEF0895209133
:104BD00034202F93209133202F93209132202F9334
:104BE000209131202F932EE134E23F932F9322E046
:104BF0002F931F929F938F930E9451768DB79EB7EC
:104C00000A968DBF9EBF85E60895CF93DF9300D0AF
:104C10001F92CDB7DEB795EA998394E79A8391E026
:104C20009B838D8360E070E0CE0101963DD88C833C
:104C30006B816C5FCE0101960E94671D2496CDBFEB
:104C4000DEBFDF91CF910895FB0120812F33D9F48E
:104C50002181211132C01F9220E32F931F9221E363
:104C60002F932EE93CE03F932F9322E02F931F9246
:104C70009F938F930E9487768DB79EB70A968DBFBC
:104C80009EBF85E60895213369F028F42033A9F406
:104C90001092302010C0223549F0243571F4818102
:104CA000B4DF09C081E08093302005C081E08093AB
:104CB0004F201092DB3084E608958AEC0895FC01C1
:104CC00080913020882311F081E301C080E380834C
:104CD000118285E60895FB0120812F33D9F42181CB
:104CE000211128C01F9220E32F931F9221E32F93BD
:104CF00028E93CE03F932F9322E02F931F929F934C
:104D00008F930E9487768DB79EB70A968DBF9EBF00
:104D100085E6089580ED820F823060F48093C1248F
:104D200041E050E061EC74E281E090E00E94D81331
:104D300084E608958AEC0895FC019091C124905D69
:104D40009083118285E60895A091F033B091F133FC
:104D500015962C911597263029F0283019F02A50F5
:104D60002230A0F5FB0120812F33D9F421812111BC
:104D70002FC01F9220E32F931F9221E32F9322E94C
:104D80003CE03F932F9322E02F931F929F938F93AA
:104D90000E9487768DB79EB70A968DBF9EBF85E627
:104DA0000895213321F481E01C968C9304C02033B4
:104DB00079F41C961C920E942A1AE091F033F0912B
:104DC000F13385810E94B51084E6089589EC089539
:104DD0008AEC0895FC01A091F033B091F1331C9658
:104DE0008C91882311F081E301C080E380831182DC
:104DF00085E6089521E02093E9302093E8302CE304
:104E00002093E63025E030E02093E4303093E53025
:104E10001092DE301092DF301092E0301092E130CC
:104E20008093DC309093DD30089527E02093E930C3
:104E30002CE231E02093E4303093E5301092DE3004
:104E40001092DF301092E0301092E1308093DC302D
:104E50009093DD300895CF939091E930953009F427
:104E60003FC030F4933019F130F5913068F426C129
:104E7000973009F4A2C008F448C0983009F4A4C0DF
:104E8000993009F48DC01AC1813031F41092E230AA
:104E90001092E33083E021C0843011F486E07EC0BC
:104EA000883109F47DC08B3109F07CC079C08093D2
:104EB000E73084E012C090E04091E7302FEF30E01F
:104EC000241B31098217930721F485E006C0891756
:104ED00069F185E10E942B1F82E08093E93062C076
:104EE0002091E2303091E330A9014F5F5F4F409352
:104EF000E2305093E330F901E959FA4C80834038AD
:104F0000510509F04FC086E0E8CF2091E73090913D
:104F1000E830291349C0E7E6F5E327EE35E390E0F2
:104F20002E173F07A1F24191940FFACF4091DE3046
:104F30005091DF306091E0307091E130E091DC30F1
:104F4000F091DD3020E830E087E695E31995C82F31
:104F5000882301F18091E8308F5F8093E830809161
:104F6000DE309091DF30A091E030B091E130805898
:104F70009F4FAF4FBF4F8093DE309093DF30A093B1
:104F8000E030B093E13086E00E942B1F82E08093F6
:104F9000E93095C088E10E942B1F88E10E942B1FF9
:104FA0001092E930C1E08BC030E0892F90E001978A
:104FB0002817390791F786E08DCF853119F41092C3
:104FC000E83008C08B3161F3883109F467CF86304F
:104FD00009F051C08091E8308F5F8093E8304091B4
:104FE000DE305091DF306091E0307091E130E0913F
:104FF000DC30F091DD3020E830E087E695E319956C
:10500000C82F882399F181E00E942B1F8091E830FE
:105010000E942B1F8091E83080950E942B1F60E832
:1050200070E087E695E30E94521FE7E6F5E380E033
:1050300095E3E73EF90719F09191890FF9CF0E94A6
:105040002B1F8091DE309091DF30A091E030B09145
:10505000E13080589F4FAF4FBF4F8093DE30909329
:10506000DF30A093E030B093E13029C084E00E94AB
:105070002B1F89E032CF853109F094CF81E00E9467
:105080002B1F8091E8300E942B1F8091E830809583
:105090000E942B1F60E870E087E695E30E94521F94
:1050A000E7E6F5E327EE35E380E02E173F0719F03A
:1050B0009191890FFACF0E942B1F74CFC0E08C2FE3
:1050C000CF9108958091E930813019F0873019F13E
:1050D00008958091E4309091E5309C012150310990
:1050E0002093E4303093E530892B21F58091E63030
:1050F0009FEF980F9093E630882321F085E10E947E
:105100002B1F02C01092E93085E090E08093E430DC
:105110009093E53008958091E4309091E5309C01C2
:10512000215031092093E4303093E530892B11F47C
:105130001092E9300895E0E5FEE020E030E094913F
:10514000981309C041E2429FC001439F900D112472
:105150008F5A914F08952F5F3F4FB19629303105F7
:1051600071F780E090E00895262FBA012F3311F4F3
:10517000469607C02D3311F4449611C021110CC07E
:105180004096FC01259134912115310521F187E6E6
:1051900095E3F90119950DC02032E9F44296FC011E
:1051A0002591349121153105B1F087E695E3F90198
:1051B00019958F3F89F491E09093EE304EB15FB135
:1051C0002091080430910904242B352B2093EC30D6
:1051D0003093ED30089589EC08950F931F93CF938A
:1051E000DF938C01C9E7DFE0BE01C8010E94F975B9
:1051F000892B49F440E050E060E0CE01DF91CF918F
:105200001F910F91B1CF689683E1C13BD80761F739
:10521000DF91CF911F910F910895EF92FF921F930D
:10522000CF93DF93982F9F7D91549A3160F090ED4A
:10523000980F9A3040F08F3531F0982F9D7F9D3335
:1052400011F08032D1F49FE9980F9A3108F480521E
:105250002091EF303091F0302F3F91E0390708F086
:105260007FC0A9014F5F5F4F4093EF305093F03004
:10527000F901E959FA4C808373C08D3009F040C0C0
:10528000E091EF30F091F030E959FA4C1082109231
:10529000EF301092F0308091EE30811161C080913A
:1052A0006735982F9F7D09F440C08D7F8D33E9F1DC
:1052B000E7E6F5E37F011191112331F01F3321F06F
:1052C0001D3311F01032B1F7F7011082C9E7DFE0AA
:1052D000BE0187E695E30E94F975892B59F4109277
:1052E0006735A7014F5F5F4F612FCE013DDF8F3FD5
:1052F000B9F124C06896F3E1C13BDF0749F715C057
:10530000883061F48091EF309091F030009741F156
:1053100001978093EF309093F03022C08B3101F5EC
:105320001092EF301092F0301BC088EC04DF0E9426
:10533000441F8DE49EE00E94441F12C0FCDE0E94C8
:10534000441F8DE49EE00E94441F809167358823AE
:1053500039F087E695E30E945D1F8AE49EE0EBCF7B
:1053600081E0DF91CF911F91FF90EF9008958091A0
:10537000EE30882399F1E091F033F091F1332085FC
:1053800031852115310551F14EB15FB1809108048D
:1053900090910904842B952B4091EC305091ED3085
:1053A000841B950B64E670E00E94687562177307B2
:1053B000A8F01092EE308BECBEDE0E94441F87E412
:1053C0009EE00E94441FE091EA30F091EB3030976C
:1053D00029F019951092EA301092EB3008958091DF
:1053E000EE308823A9F01092EE308BECA4DE0E9400
:1053F000441F87E49EE00E94441FE091EA30F09150
:10540000EB30309729F019951092EA301092EB307A
:105410000895CF93DF939091EE309923A9F0EB019B
:105420001092EE3088DE0E94441F84E49EE00E94C9
:10543000441F209749F0CE010E945D1F81E49EE049
:10544000DF91CF910C94441FDF91CF910895EF929B
:10545000FF920F931F93CF937C019B01613081E0FA
:10546000780710F020E031E08B01021B130BA7013D
:1054700060E072E087E695E30E94681187E695E3B5
:105480000E945D1FC1E0013081E01807A8F01A9565
:105490004C2F50E0542F44274E0D5F1D20E032E08A
:1054A00060E072E087E695E30E94681187E695E385
:1054B0000E945D1FCF5FE7CF0115110589F04C2FCA
:1054C00050E0542F44274E0D5F1D980160E072E0BC
:1054D00087E695E30E94681187E695E30E945D1FC9
:1054E0008EE39EE0CF911F910F91FF90EF900C946F
:1054F000441F80910008813021F490918C089330F2
:1055000009F080E080FD1AC08091F330811116C04F
:1055100081E08093000893E090938C088093F130B1
:105520001092F2302EB13FB180910804909109049D
:10553000822B932B8093F8309093F930089510923A
:105540008C0810920008E1EFF0E3108211820895B8
:105550009091F1309923F1F08091F230811115C0D2
:105560002091F1302223B9F04EB15FB120910804AF
:1055700030910904242B352B4091F8305091F930AB
:10558000241B350B2634310530F081E08093F23056
:10559000892F089581E00895CF93C091F330CC23F3
:1055A000C1F02EB13FB18091080490910904822B83
:1055B000932B2091F6303091F730821B930B209182
:1055C000F4303091F5308217930718F01092F330D1
:1055D00090DF8C2FCF910895E091F033F091F1336B
:1055E0008287938780933803909339030895E091DD
:1055F000F033F091F13382859385409682879387CB
:105600008093380390933903828593850895E091C0
:10561000F033F091F13380E991E0828793878093B2
:105620003803909339030895A0E2B6E081E015961F
:105630008C93159727E637E328B939B927EE37E376
:105640002AB93BB910B813B812B816B817B811B8C0
:10565000E0E0F9E010A211A22FEF30E026A337A37B
:105660002FEF3FEF20A731A7808398E8938390E145
:10567000948793E097831C968C931C9782E01A96EC
:105680008C930895E0E0F9E013828FE790E086AB19
:1056900097AB81E190E080AF91AFE0E0FAE010A23B
:1056A00011A28FEF9FEF86A397A389E883831682C9
:1056B00081E084878EE0808310922A0608951F92ED
:1056C0000F920FB60F92112408B60F9218BE09B6AA
:1056D0000F9219BE0BB60F921BBE2F933F934F93A1
:1056E0005F936F937F938F939F93AF93BF93EF934A
:1056F000FF93E091D233F091D3331995FF91EF915D
:10570000BF91AF919F918F917F916F915F914F91D9
:105710003F912F910F900BBE0F9009BE0F9008BEC6
:105720000F900FBE0F901F9018951F920F920FB6FB
:105730000F92112408B60F9218BE0BB60F921BBE23
:105740002F933F938F939F93EF93FF93209128067E
:1057500093B1267081E009F080E0990F892B83B91D
:1057600082B1882309F463C012B883B1877087308F
:1057700059F51092000980E180930C091092030AF8
:105780001B9B03C08CEA94E002C08CE694E08093FB
:10579000260A9093270A82E081B981E080930C0A5F
:1057A00083E08093060A86B197B1877049F090B183
:1057B0008F5F893011F09695FBCFE8B1F9B19083F6
:1057C00081E08093FA3036C083B1982F9C7091F1BC
:1057D000847091B191111CC020B12695882311F0DD
:1057E00080E001C080E8282B20B986B197B10196EE
:1057F00086B997B987709927892BE1F4E8B1F9B197
:10580000CF01019688B999B9208381E081B912C08E
:1058100091B1913079F4EAB1FBB19F012F5F3F4F15
:105820002AB93BB9811190E0908311B803C082B1CD
:10583000809582B988E880930309FF91EF919F9149
:105840008F913F912F910F900BBE0F9008BE0F903C
:105850000FBE0F901F9018951F920F920FB60F92C8
:10586000112408B60F9218BE0BB60F921BBE2F93D1
:105870003F938F939F93EF93FF9381B1823008F40E
:105880009DC081B18D3008F099C0E1B1F0E0EE0F1C
:10589000FF1FEA58FF4D0190F081E02D19948FE72A
:1058A00090E08093260A9093270A88C08E9A8EE013
:1058B000809340088FE390E08093260A9093270A14
:1058C00085E06FC08E9886E081B98FEF82B914B8F9
:1058D00015B8E8B1F9B1808180B970C0009B05C0EE
:1058E0008E9A82B1809582B901C08E9887E059C0A6
:1058F000009B02C08E9801C08E9A80B1869580B9B7
:1059000084B195B1019684B995B984B195B1877088
:105910009927892B11F488E044C024B135B186B1B0
:1059200097B128173907B1F52BC0EAB1FBB1309711
:1059300011F0808101C082B1882311F08E9A01C0DC
:105940008E9889E02EC0EAB1FBB1309751F080818A
:10595000882311F08E9801C08E9A3196EAB9FBB96E
:1059600008C082B1882311F08E9801C08E9A8FEF03
:1059700082B924B135B186B197B12817390711F42E
:105980008AE00FC0E8B1F9B1CF01019688B999B9A1
:10599000818180B986E005C08E988BE002C08E9828
:1059A0008CE081B90BC01092000A1092060A109286
:1059B00040081092410881E08093FB30FF91EF9105
:1059C0009F918F913F912F910F900BBE0F9008BE2A
:1059D0000F900FBE0F901F901895CF93DF93EAEFB3
:1059E000F0E3108211828AE09EE28093D03290939D
:1059F000D13282E49BE28093D2339093D333E0E4BC
:105A0000F6E0128A84E08283C0E8D1E082E68E83E9
:105A1000A0E2B6E081E016968C93169711968C93CF
:105A2000119796E012969C93129751968C935197EA
:105A300032E052963C9352971A961C921A971B96F4
:105A40001C921B979FE019969C9399E598832AE5F1
:105A500029839A8390E491839683A0EBB0E0129619
:105A60002C911297207F12962C93129712962C91BC
:105A70001297226012962C9320E321832683908B29
:105A80008683358383E08183E0E0F8E083E18183EE
:105A900021E030E026A337A320A731A7E0E8F8E013
:105AA00014868083E0E2F3E01382118288E082832F
:105AB00091E19083A091F033B091F1331A962D913A
:105AC0003C911B97208F318FE0E8F3E09CE39283B9
:105AD000808393838183DF91CF91A6CDA0E2B6E04E
:105AE0001A961C921A97EAEFF0E310821182E0E016
:105AF000F9E010821382178280E18487E0E0FAE007
:105B000010821382168281E08487E0E4F8E010823C
:105B1000118216968C938E980895CF93DF9380917F
:105B2000FA30882309F46AC01092FA30C6B1D7B1AE
:105B3000C730D10508F45DC0E091C524F091C624BA
:105B4000309761F0AE01495F5F4F93E056954795FE
:105B50009A95E1F767E677E380E4199563E188E0D9
:105B60000E94041BE091E433F091E533BE0187E627
:105B700097E31995EC0194FF06C0DF7E87EE97E36B
:105B80008AB99BB902C01AB81BB8209791F1E0916D
:105B9000C524F091C624309761F0AE01495F5F4F94
:105BA00083E0569547958A95E1F767E677E381E4C8
:105BB000199563E189E00E94041BC6B9D7B987E64D
:105BC00097E388B999B910926008109261088FE044
:105BD00090E0809366089093670888E090E0809357
:105BE0006A0890936B0883E28093410883E081B94F
:105BF00005C01092000A1092060A16DD8091FB3053
:105C0000882329F01092FB30DF91CF910DCDDF91E9
:105C1000CF910895E0E0F9E080E484871782E0E81E
:105C2000F3E082E0878389EB818387E697E38AB993
:105C30009BB981E090E084B995B916B82EB13FB117
:105C40008091080490910904822B932B8093FD305E
:105C50009093FE3081E08093013118B817B810920C
:105C6000FC300895CF93DF93E0E4F6E0128A84E0FD
:105C70008283C0E8D1E082E68E83A0E2B6E081E0D4
:105C800016968C93169711968C93119796E0129610
:105C90009C93129751968C93519732E052963C9375
:105CA00052971A961C921A971B961C921B979FE06C
:105CB00019969C93199799E598832AE529839A83E5
:105CC00090E491839683C0EBD0E02A81207F2A83E1
:105CD0002A8122602A8320E321832683908B868376
:105CE000358393E09183E0E0F8E093E1918321E054
:105CF00030E026A337A320A731A7E0E8F8E0148618
:105D00009083E0E2F3E01382118298E0928321E134
:105D10002083C091F033D091F1332A853B85208FC9
:105D2000318FE0E8F3E02CE3228390832383918397
:105D30002AE03EE22093D0323093D13215968C93F4
:105D4000E0E0F9E02FEF30E026A337A312A613A678
:105D500014A615A610821682178280831092000A5C
:105D60001092FC30EFEFF0E3108212821182DF918B
:105D7000CF91089581E080932606E1DBE0E0F9E031
:105D800010821782E0E0FAE010821782EFEFF0E372
:105D900011821282108208951F920F920FB60F92F5
:105DA000112408B60F9218BE09B60F9219BE0BB691
:105DB0000F921BBE2F933F934F935F936F937F93ED
:105DC0008F939F93AF93BF93EF93FF93E091D03264
:105DD000F091D1321995FF91EF91BF91AF919F91C1
:105DE0008F917F916F915F914F913F912F910F9084
:105DF0000BBE0F9009BE0F9008BE0F900FBE0F9004
:105E00001F901895E0E0F9E08FEF94E086A397A348
:105E100080E6848780E387838FEF90E086AB97AB43
:105E200008951F920F920FB60F92112408B60F9289
:105E300018BE0BB60F921BBE2F933F934F935F93E9
:105E40008F939F93EF93FF931092070A1092000A8B
:105E50001092470910924009809181038E7F8093B0
:105E6000810384B195B180FF1AC0379B03C086B10E
:105E7000869503C086B18695806886B984B195B150
:105E8000019684B995B987709927892B41F4EAB1B5
:105E9000FBB1CF0101968AB99BB986B1808384B1E9
:105EA00095B187709927892BC9F0E4B1F5B186B116
:105EB00044B155B193E0F695E7959A95E1F7E95924
:105EC000F84C90E04770552728E030E0241B350B54
:105ED00002C0959587952A95E2F7808381E08093AB
:105EE0000031109201318FEF9FEF8093260A90933B
:105EF000270A1092200A1092210A1092060A109284
:105F0000070A1092030A84E08093000A83E08093DA
:105F1000FC30FF91EF919F918F915F914F913F9155
:105F20002F910F900BBE0F9008BE0F900FBE0F90D9
:105F30001F9018951F920F920FB60F92112408B65A
:105F40000F9218BE0BB60F921BBE8F93EF93FF9369
:105F5000E0E8F3E081818F7C8183E0E0FAE088E88B
:105F6000838381E08083FF91EF918F910F900BBE2F
:105F70000F9008BE0F900FBE0F901F9018951F92A4
:105F80000F920FB60F92112408B60F9218BE0BB6DF
:105F90000F921BBE8F939F93EF93FF9380916009A5
:105FA000109260091092610993E090934009813545
:105FB00020F4813308F472C01BC08137E8F484B147
:105FC00095B180FF2EC086B18695806886B984B170
:105FD00095B1019684B995B987709927892B41F4B9
:105FE000EAB1FBB1CF0101968AB99BB986B1808332
:105FF00086B1869580682CC086B18695806886B902
:1060000084B195B1019684B995B987709927892B88
:1060100041F4EAB1FBB1CF0101968AB99BB986B1CF
:10602000808386B18695806886B984B195B10196E2
:1060300084B995B987709927892B41F4EAB1FBB1EE
:10604000CF0101968AB99BB986B1808386B18695C6
:1060500086B984B195B1019684B995B987709927AD
:10606000892B41F4EAB1FBB1CF0101968AB99BB902
:1060700086B1808386B1869586B984B195B1019643
:1060800084B995B987709927892B41F4EAB1FBB19E
:10609000CF0101968AB99BB986B18083FF91EF91B8
:1060A0009F918F910F900BBE0F9008BE0F900FBE67
:1060B0000F901F9018950F931F93CF93DF93CDB739
:1060C000DEB7DA95CDBFDEBF80910131882309F4B8
:1060D00083C04EB15FB18091080490910904209172
:1060E000FD303091FE30842B952B821B930B209139
:1060F0006C2030916D202F5F3F4F2817390708F033
:106100006BC01092070A1092000A10924709109271
:106110004009809181038E7F8093810384B195B182
:1061200080FF1AC0379B03C086B1869503C086B135
:106130008695806886B984B195B1019684B995B980
:1061400087709927892B41F4EAB1FBB1CF01019601
:106150008AB99BB986B1808384B195B1877099273C
:10616000892BC9F0E4B1F5B186B144B155B113E062
:10617000F695E7951A95E1F7E959F84C90E04770E4
:10618000552728E030E0241B350B02C095958795F4
:106190002A95E2F7808381E08093003110920131EB
:1061A0002FEF3FEF2093260A3093270A1092200A00
:1061B0001092210A1092060A1092070A1092030AFE
:1061C00094E09093000A93E09093FC3014B815B8D3
:1061D0008093003110920131DFD981115BC2B8D9AF
:1061E000882309F457C280910131811153C28091F3
:1061F000FF30811105C080910031882309F44AC223
:106200008091FC30833041F48091200A9091210AE2
:106210008532914008F43EC280910031882309F410
:1062200098C084B195B1892B09F493C084B195B11C
:10623000089718F414B815B88CC044B155B1495F2B
:106240005F4FB3E056954795BA95E1F767E677E378
:10625000CE0101960E941E7687E697E38AB99BB924
:1062600044B155B114B815B889818695869589834E
:1062700022E030E024173507B0F5F901A3E0F695E8
:10628000E795AA95E1F781E090E08C0F9D1FE80F5C
:10629000F91F8081982F9695969590838370813011
:1062A00049F030F08230D1F486B18695806804C020
:1062B00081E015C086B1869586B984B195B1019605
:1062C00084B995B987709927892B41F4EAB1FBB15C
:1062D000CF0101968AB99BB986B1808380E02E5F99
:1062E0003F4F882339F284B195B187709927892B64
:1062F000C9F0E4B1F5B186B144B155B173E0F6959A
:10630000E7957A95E1F7E959F84C90E04770552701
:1063100028E030E0241B350B02C0959587952A951F
:10632000E2F7808363E188E00E94041B44B155B129
:10633000E091C524F091C624309759F0495F5F4F32
:1063400063E0569547956A95E1F767E677E382E45F
:1063500019951092FF301092003164B175B1E0913F
:10636000E433F091E53387E697E3199584B995B95D
:1063700084B195B1892B09F48DC189E8809381039B
:106380001092000A1092200A1092210A2FEF3FEF7C
:106390002093260A3093270A8FE590E08093280AFD
:1063A0009093290A1092060A80E180930C0A93E0E8
:1063B0009093070A10926009109261092093660970
:1063C0003093670920EA30E0209368093093690927
:1063D0001092460980934C0981E08093470981E13E
:1063E00080938001109288011092800310922906F8
:1063F00063E189E00E94041B44B155B1E091C524DA
:10640000F091C624309759F0495F5F4F33E05695BD
:1064100047953A95E1F767E677E383E4199504B188
:1064200015B1013094E0190708F024C114B815B86B
:10643000A801495F5F4F23E0569547952A95E1F7FC
:1064400067E677E387EE97E30E941E7687E697E399
:106450008AB99BB986B18695806886B984B195B1B1
:10646000019684B995B987709927892B39F488E604
:1064700097E38AB99BB986B18093673786B18695D1
:1064800086B984B195B1019684B995B98770992779
:10649000892B41F4EAB1FBB1CF0101968AB99BB9CE
:1064A00086B1808380E041E050E0E7EEF7E3041737
:1064B000150708F495C0908190FF2BC086B1869592
:1064C00086B984B195B1019684B995B98770992739
:1064D000892B41F4AAB1BBB1CD0101968AB99BB910
:1064E00086B18C9386B18695806886B984B195B162
:1064F000019684B995B987709927892B09F063C0F3
:10650000AAB1BBB1CD0101968AB99BB986B18C9372
:106510005AC0882351F186B1869586B984B195B168
:10652000019684B995B987709927892B41F4AAB14E
:10653000BBB1CD0101968AB99BB986B18C9386B166
:10654000869586B984B195B1019684B995B987705D
:106550009927892B41F4AAB1BBB1CD0101968AB923
:106560009BB986B18C9380E02FC096B196959068C8
:1065700096B924B135B12F5F3F4F24B935B9277093
:106580003327232B49F4AAB1BBB19D012F5F3F4FA5
:106590002AB93BB996B19C9396B1969596B924B118
:1065A00035B12F5F3F4F24B935B927703327232BDF
:1065B000D1F6AAB1BBB19D012F5F3F4F2AB93BB9BC
:1065C00096B19C9301C081E09081969590839A0149
:1065D00027703327232B09F431964F5F5F4F67CF26
:1065E000811129C086B18695806886B984B195B13C
:1065F000019684B995B987709927892B41F4EAB13E
:10660000FBB1CF0101968AB99BB986B1808386B16F
:10661000869586B984B195B1019684B995B987708C
:106620009927892B41F4EAB1FBB1CF0101968AB9D0
:106630009BB986B1808384B195B187709927892BE6
:10664000C9F0E4B1F5B186B144B155B193E0F69526
:10665000E7959A95E1F7E959F84C90E0477055278E
:1066600028E030E0241B350B02C0959587952A95CC
:10667000E2F7808381E08093FC3087E697E38AB974
:106680009BB980E280930C098CE08093070985E533
:106690008A95F1F7D395CDBFDEBFDF91CF911F91E2
:1066A0000F91089514B815B881E08093FF300C94D1
:1066B000792A1092070A1092000A10924709109244
:1066C0004009809181038E7F8093810384B195B1CD
:1066D00080FF1AC0379B03C086B1869503C086B180
:1066E0008695806886B984B195B1019684B995B9CB
:1066F00087709927892B41F4EAB1FBB1CF0101964C
:106700008AB99BB986B1808384B195B18770992786
:10671000892BC9F0E4B1F5B186B144B155B193E02C
:10672000F695E7959A95E1F7E959F84C90E04770AE
:10673000552728E030E0241B350B02C0959587953E
:106740002A95E2F7808381E0809300311092013135
:106750008FEF9FEF8093260A9093270A1092200ACA
:106760001092210A1092060A1092070A1092030A48
:1067700084E08093000A83E08093FC301092FC3028
:10678000109200311092FF300C949F2A8091600982
:10679000109260091092610993E09093400981354D
:1067A00020F4813308F4A7C003C0813758F165C0D5
:1067B000809102319091033180FF0AC080910231B3
:1067C000909103310297C0F085B18695806802C030
:1067D00085B1869585B986B197B1019686B997B985
:1067E00087709927892B41F4ECB1FDB1CF01019657
:1067F0008CB99DB985B1808380910231909103312C
:10680000029675C0809102319091033180FF1BC0C8
:1068100080910231909103310297A8F085B186955D
:10682000806885B986B197B1019686B997B98770A6
:106830009927892B41F4ECB1FDB1CF0101968CB9B8
:106840009DB985B1808385B1869585B986B197B1AB
:10685000019686B997B987709927892B41F4ECB1D5
:10686000FDB1CF0101968CB99DB985B1808380912E
:1068700002319091033103963AC080910231909198
:10688000033180FF2FC08091023190910331029734
:10689000A8F085B18695806885B986B197B10196D3
:1068A00086B997B987709927892B41F4ECB1FDB16E
:1068B000CF0101968CB99DB985B1808385B186954C
:1068C00085B986B197B1019686B997B9877099272E
:1068D000892B41F4ECB1FDB1CF0101968CB99DB982
:1068E00085B1808380910231909103310496809329
:1068F00002319093033108951F920F920FB60F92B9
:10690000112408B60F9218BE0BB60F921BBE8F93C0
:106910009F93EF93FF93E0E0F9E013828FE790E01D
:1069200086AB97AB81E190E086AF97AF10922B06D4
:10693000FF91EF919F918F910F900BBE0F9008BE2A
:106940000F900FBE0F901F9018951F920F920FB6C9
:106950000F92112408B60F9218BE0BB60F921BBEF1
:106960002F933F934F935F938F939F93EF93FF9357
:106970002091280694B1267081E009F080E0990FFB
:10698000892B84B983B1882309F4E0C013B884B19A
:106990008770873009F0B2C01092000980E88093B8
:1069A0000C09109207091092290686B197B18770D9
:1069B00049F090B18F5F893011F09695FBCFE8B127
:1069C000F9B1908386B197B18093063190930731E6
:1069D0008091063190910731079708F45CC081E0FF
:1069E00080930A3127E638E32CB93DB921E030E045
:1069F000209302313093033116B817B815B899E8CF
:106A0000909380031092000A1092200A1092210A9B
:106A10004FEF5FEF4093260A5093270A2FE530E0AF
:106A200020932A0A30932B0A1092060A20E2209320
:106A30000C0A9CE09093070A109260091092610979
:106A4000409366095093670940EA50E040936A0911
:106A500050936B091092460920934C099093470973
:106A600090E19093820110928A01109281038093A9
:106A7000870389EB809380032EB13FB18091080496
:106A800090910904822B932B8093083190930931C4
:106A900082E081B961C08CE08093290687E697E3A4
:106AA00088B999B987EE97E38AB99BB910B814B839
:106AB00013B816B817B811B810922009109221090E
:106AC0008FEF90E080932609909327098FEF9FEF37
:106AD00080932E0990932F0981E08093000988E824
:106AE0008093030980E880930C0980EC8093070968
:106AF00082E080932C0680932B062EC084B1982FC1
:106B00009C7039F191B191111CC020B1269582FF82
:106B100002C080E001C080E8282B20B986B197B17F
:106B2000019686B997B987709927892B91F4E8B1B6
:106B3000F9B1CF01019688B999B9208381E081B973
:106B400008C081B1813029F411B803C083B18095A8
:106B500083B988E880930309FF91EF919F918F910A
:106B60005F914F913F912F910F900BBE0F9008BEF8
:106B70000F900FBE0F901F9018951F920F920FB697
:106B80000F92112408B60F9218BE0BB60F921BBEBF
:106B90008F93EF93FF93E0E8F3E080818F7C808315
:106BA000E0E0FAE08AE8838381E0808383E081B9D2
:106BB000FF91EF918F910F900BBE0F9008BE0F9039
:106BC0000FBE0F901F9018951F920F920FB60F9245
:106BD000112408B60F9218BE09B60F9219BE0BB653
:106BE0000F921BBE2F933F934F935F936F937F93AF
:106BF0008F939F93AF93BF93EF93FF93E091CE3228
:106C0000F091CF321995FF91EF91BF91AF919F9184
:106C10008F917F916F915F914F913F912F910F9045
:106C20000BBE0F9009BE0F9008BE0F900FBE0F90C5
:106C30001F9018951F920F920FB60F92112408B64D
:106C40000F9218BE0BB60F921BBE2F933F934F931C
:106C50005F938F939F93EF93FF931092070A109285
:106C6000000A1092030A109247091092400980917D
:106C700080038E7F80938003809102319091033155
:106C800080FF15C085B18695806885B986B197B1BA
:106C9000019686B997B987709927892B41F4ECB191
:106CA000FDB1CF0101968CB99DB985B1808386B1C4
:106CB00097B187709927892BC9F0E6B1F7B185B1F3
:106CC00046B157B193E0F695E7959A95E1F7E95902
:106CD000F74C90E04770552728E030E0241B350B37
:106CE00002C0959587952A95E2F7808386B197B182
:106CF000809304319093053186B197B1049718F0D1
:106D000081E080930B311092000A1092070A1092D2
:106D1000820110928A018CE38093820388E0809341
:106D200080038CE08093290687E697E388B999B9B8
:106D300087EE97E38AB99BB910B814B813B816B8A0
:106D400017B811B810922009109221098FEF90E026
:106D500080932609909327098FEF9FEF80932E0948
:106D600090932F0981E08093000988E880930309BC
:106D700080E880930C0980EC8093070982E080937F
:106D80002C0680932B06FF91EF919F918F915F913D
:106D90004F913F912F910F900BBE0F9008BE0F9017
:106DA0000FBE0F901F901895CF93DF93A0E4B6E02D
:106DB00052961C92529784E012968C931297C0E8D8
:106DC000D1E082E68E83E0E2F6E081E08683818393
:106DD00096E09283818B92E0928B128613862FE04D
:106DE000218729E528833AE539832A8320E411960F
:106DF0002C93119716962C931697C0EBD0E03A81FE
:106E0000307F3A833A8132603A8330E311963C9383
:106E1000119716963C93169750962C93509716966A
:106E20008C93169715969C93159723E011962C93A7
:106E3000A0E0B8E023E111962C93119741E050E0D7
:106E400096964D935C93979798964D935C939997EC
:106E5000A0E8B8E01C961C921C972C93A0E2B3E02B
:106E600013961C92139711961C92119728E0129674
:106E70002C93129731E13C93C091F033D091F133D0
:106E80004A855B8558964D935C935997A0E8B3E08B
:106E90003CE312963C9312972C9313963C931397D2
:106EA00011962C9326EC33E32093CE323093CF32DD
:106EB0008583AAE0B1E31C9211961C922CE02187F5
:106EC00027E637E328B939B927EE37E32AB93BB9C2
:106ED00010B814B813B816B817B811B8A0E0B9E0D4
:106EE00090961D921C9291972FEF30E096962D93DD
:106EF0003C9397972FEF3FEF9E962D933C939F9750
:106F00008C9388E813968C93139780E81C968C9347
:106F10001C9780EC17968C9394879387DF91CF9181
:106F20000895E0E0FAE010821782E0E8F1E01282D2
:106F30001286E0E8F3E08CE3828388E08083A0E2BD
:106F4000B6E01B961C921B9719961C921997E0E0CD
:106F5000F9E010821382178280E8848781E0169618
:106F60008C93089580910A31882341F110920A315F
:106F70004091063150910731E091C524F091C6242B
:106F8000309759F0495F5F4F93E0569547959A9532
:106F9000E1F767E677E384E4199563E188E00E940E
:106FA000041B1092CD326091063170910731E0914F
:106FB000E433F091E53387E697E3199580910B313F
:106FC000882349F110920B314091043150910531E1
:106FD000E091C524F091C624309759F0495F5F4F86
:106FE00083E0569547958A95E1F767E678E387E46D
:106FF000199563E188E00E94041B81E08093CD3203
:107000006091043170910531E091E433F091E53302
:1070100087E698E3199521B1223009F055C06EB189
:107020007FB18091080490910904409108315091FA
:107030000931862B972B841B950B40916C20509126
:107040006D204817590708F03FC01092000A1092AF
:10705000070A1092820110928A018CE380938203C6
:1070600088E0809380038CE08093290687E697E38D
:1070700088B999B987EE97E38AB99BB910B814B863
:1070800013B816B817B811B8109220091092210938
:107090008FEF90E080932609909327098FEF9FEF61
:1070A00080932E0990932F0981E08093000988E84E
:1070B0008093030980E880930C0980EC8093070992
:1070C00020932C0620932B060895982F809134311D
:1070D000882359F080912E31811108C081E02091E0
:1070E0002D31921718F080E0089581E008950F93F4
:1070F0001F93CF93DF931F92CDB7DEB7009131314D
:10710000000F000F005182E08093343110E0B8018D
:107110006D5F7F4F41E050E08DE291E30E94CD1121
:10712000B8016C5F7F4F41E050E0CE0101960E94B4
:10713000CD118981881F8827881F80932C3181E099
:10714000809333311092323110922E3110923031BF
:107150000F90DF91CF911F910F9108950F931F937F
:10716000CF93DF931F921F92CDB7DEB78C0142E021
:1071700050E069E270E0CE0101960E94CD112981B4
:107180003A81F80190812115310549F4218130E0DF
:10719000322F2227A901490F511DCA010DC09F702E
:1071A000F8019083892F90E0A901409550954817E8
:1071B000590770F0820F931F89839A8342E050E051
:1071C00069E270E0CE0101960E94431481E001C0A3
:1071D00080E00F900F90DF91CF911F910F91089554
:1071E000CF93DF931F92CDB7DEB781E08093343128
:1071F00040E150E060EB70E08CE091E30E94CD1143
:1072000060911231509111314091103130910F3114
:1072100020910E3190910D3180910C31709113318C
:1072200070930C3160930D3150930E3140930F31B8
:107230003093103120931131909312318093133198
:1072400060911A31509119314091183130911731B4
:1072500020911631909115318091143170911B312C
:107260007093143160931531509316314093173158
:10727000309318312093193190931A3180931B3138
:1072800080E38093313141E050E068EA70E08DE2C4
:1072900091E30E94CD1141E050E06CEA70E0CE0134
:1072A00001960E94CD1181E09981911180E0809337
:1072B0002C3181E0809333311092323110922E3193
:1072C000109230310F90DF91CF91089510923431A8
:1072D00080E1809331318FEF80932D3110922C31EA
:1072E00081E0809333311092323110922E3110921E
:1072F0003031089584E180933131F9CE89E2809371
:107300003131F5CE81E080933331089510922E31E2
:1073100081E080933331089508958F929F92AF92C8
:10732000BF92CF92DF92EF92FF920F931F93CF9372
:10733000DF93CDB7DEB76097CDBFDEBF7C01DC0148
:107340008C91909133319230F1F038F0943079F1A2
:1073500020F1963009F455C0E7C0292F20952170FF
:1073600020933231992311F0863219F0823509F0D9
:10737000DBC084E4F7018083118282E080933331A3
:1073800080E190E0CBC390913231911102C08632FE
:10739000B9F0823509F0CBC013C090913231911110
:1073A00002C0863269F0823509F0F3C009C09091BD
:1073B0003231911102C0863219F0823509F09BC139
:1073C00084E4D7018C9311961C9281E0892716C022
:1073D000809130318111A3C1D7018C91803509F49E
:1073E0009CC008F0ADC1803309F4C8C1909134311C
:1073F000913009F430C208F055C281E080933331F6
:1074000093C08F3A09F080C0695F7F4F93E0769513
:1074100067959A95E1F762507109C7010E94134878
:10742000882309F471C0FE0131966F0188E0DF0105
:107430001D928A95E9F75701BFEFAB1ABB0A0CE022
:1074400011E32CE131E3AF01B50181E090E00E944E
:10745000F20E2CE131E3AE01475F5F4FB701675F8A
:107460007F4F81E090E00E94F20E90912431888954
:10747000981323C090912531898598131EC090914F
:1074800026318A85981319C0909127318B859813DE
:1074900014C0909128318C8598130FC09091293198
:1074A0008D8598130AC090912A318E85981305C056
:1074B00081E020912B319F85291380E080FF24C03B
:1074C000198147E050E0BE016E5F7F4FC6010E9408
:1074D000277618870CE011E32CE131E3A501B60112
:1074E00081E090E00E94E90EF701108269E070E00F
:1074F000C7010E94E84781E080932E3184E08093A9
:10750000333188E590E00AC381E08093333186E02F
:10751000D7018C9384E090E001C3D70111968C9140
:1075200081111DC11092333180E090E0F7C28339A0
:1075300009F063CF19821A821B821C8288E8898332
:1075400043E050E060E070E0CE0102960E94CD1171
:10755000F7018181803261F1803709F05CC0F70169
:10756000928189819813C2C093818A819813BEC089
:1075700094818B819813BAC095818C819813B6C081
:1075800084E0808361E070E0C7010E94E84783E007
:107590003EC0853909F031CF44E050E064E070E04E
:1075A000CE0101960E94CD11F70181818032A9F4AC
:1075B0003981D7013C932A8111962C9311979B8195
:1075C00012969C9312978C8113968C931397232772
:1075D0009227892714968C9387C08037E1F4F701AE
:1075E00092818981981382C093818A8198137EC089
:1075F00094818B8198137AC095818C81981376C081
:10760000108261E070E0C7010E94E84784E0809347
:10761000333138E16CC0082F02950F700250182FDB
:107620001F7088E090E0811B91092FEF30E0690125
:1076300002C0D594C7948A95E2F7053021F0043052
:1076400051F51123E1F044E050E0B7016E5F7F4F48
:10765000CE0101960E941176892B69F499818A8165
:1076600089279B8189279C818927D70116969C9120
:1076700089278C2161F1043071F4111137C044E085
:1076800050E0B7016E5F7F4FCE0101960E941176E8
:10769000892BE9F02BC0043048F510E0A801B701B0
:1076A0006E5F7F4FCE0101960E941176892BF1F417
:1076B000D701A00FB11FE1E0F0E0EC0FFD1FE00FDC
:1076C000F11F12969C9180818927C82279F4398113
:1076D000F70130832A8121839B8192838C8183836C
:1076E000232792278927848338E201C030E020E0F5
:1076F000832F922F13C2695F7F4F83E07695679542
:107700008A95E1F76330710508F477CE625071090C
:10771000C7010E94134881115BCE81E0D9C110924C
:10772000303160912F316932E1F480913431813010
:10773000C1F4C701029612DD882389F08AE0E8CE01
:10774000803A09F473C0823A09F050CED7011196FD
:107750001C91193209F44BC0123008F04DC0F701EA
:1077600084C18091ED338111E9CFF4E06F9FB001C6
:10777000112444E050E0C701029655C0F701118181
:1077800080913431882369F090912C31992339F01C
:1077900090912E31911103C000912D3106C081309E
:1077A00019F00091313101C00CE21017C0F6C12C64
:1077B000D12CF4E01F9FB001112444E050E0C70138
:1077C0008C0D9D1D0E94CD111F5F011301C010E0A3
:1077D00024E0C20ED11C80E1C816D10451F760E14B
:1077E00070E0C7010E94E84780E990E097C180916E
:1077F0003431813009F49DCF80913131181708F070
:10780000AECF812F62DC811102C086E061C1C70169
:1078100002962091ED33211191CFF4E01F9FB0012A
:10782000112444E050E00E94431488CFD701119600
:107830001C91123008F493CF80913131181708F061
:107840008ECF812F42DC882301F310932F3181E00A
:10785000809330313CC18A3109F0CFCD86E08093EE
:10786000333168E084E291E30E944E1188E0ECE15C
:10787000F1E3DF011D928A95E9F7A7014F5F5F4FA2
:107880000CE011E39F0164E271E381E090E00E946B
:10789000E90E8FEAF701808369E070E0C7010E947A
:1078A000E8472FCE8C3309F416C148F4893309F424
:1078B000AEC08A33D9F18B3109F09FCD75C08B34BE
:1078C00009F418C138F48E3309F097CD8DEBD70148
:1078D0008C931DC1803621F0853A09F4B3C08DCD5B
:1078E000D7011C9284E011968C93119783E0129635
:1078F0008C93129781E013968C93139714968C9324
:10790000149715961C9280913131843111F08EE0DC
:1079100001C08BE0F701868383E0878368E070E035
:10792000C7010E94E84780E590E0F8C0D7011196B2
:10793000DC90119712960C910D1508F410CF8091E0
:107940003131D81608F00BCF081708F008CF809116
:107950002C31882351F08D2DB8DB882309F455CFC5
:10796000802FB3DB882309F450CF10E06D2D70E039
:10797000061B170B0F5F1F4F000F111F000F111F6A
:10798000660F771F660F771FA801C7010E94CD11F0
:10799000B801C7010E94E847C8010296A3E0880F1A
:1079A000991FAA95E1F7BAC000913131000F000F7D
:1079B000005110E0B801685F7F4F44E050E0CE0115
:1079C00001960E94CD119981F701818198139FCD75
:1079D0009A81828198139BCD9B818381981397CD47
:1079E0009C818481981393CD81E080932E31B801DE
:1079F000645F7F4F42E050E0C7010E94CD1162E01A
:107A000070E0C7010E94E84780E290E087C0F7017C
:107A10006181633008F0A3CE8091313170E0680F4E
:107A2000711D660F771F660F771F43E050E0C70197
:107A30000E94CD1163E070E0C7010E94E84788E230
:107A400090E06CC0D70111962C91022F10E0902F7E
:107A50008827856A092E000CAA0BBB0BF70132811F
:107A60004C015D01A32A233010F0108253CD809188
:107A70003131B801680F711D660F771F660F771FD0
:107A800044E050E0CE0101960E94CD1189819A8197
:107A9000AB81BC81880D991DAA1DBB1D89839A836A
:107AA000AB83BC830097A105B14010F084E030CDDA
:107AB00080913131B801680F711D660F771F660F15
:107AC000771F44E050E0CE0101960E9443148AE003
:107AD000F70180831FCD40E250E06AEC70E0C701FF
:107AE0000E94387660E270E0C7010E94E84780E1BA
:107AF00091E014C060913131660F660F605170E003
:107B00006B5F7F4F41E050E0C7010E94CD1161E003
:107B100070E0C7010E94E84788E190E06096CDBF21
:107B2000DEBFDF91CF911F910F91FF90EF90DF901B
:107B3000CF90BF90AF909F908F900895CF93DF9399
:107B4000EC0143E050E060E070E00E94CD1144E0C1
:107B500050E064E070E0CE010396DF91CF910C9489
:107B6000CD110F931F93CF93DF931F921F92CDB729
:107B7000DEB78C01FC0190818181892798E88927F3
:107B8000928189278A839381848189279581892796
:107B900096818927898343E050E060E070E0C80166
:107BA0000E94431441E050E063E070E0CE01029691
:107BB0000E94431444E050E064E070E0C801039682
:107BC0000E94431441E050E068E070E0CE0101966D
:107BD0000E9443140F900F90DF91CF911F910F914E
:107BE0000895CF92DF92EF92FF920F931F93CF935E
:107BF000DF9300D01F92CDB7DEB790913531992336
:107C000009F453C0CEB0DFB02091080430910904CC
:107C1000A0916E20B0916F20E8EFFFE7EA1BFB0B0D
:107C2000042F10E0780194E0E90EF11CEE16FF0637
:107C300070F081E08093010693E090938106809339
:107C4000060692E090938606809386062EC07B01FE
:107C50002C293D2989834A833B832C8344E050E0CF
:107C6000BD01CE0101960E94431460916E20709177
:107C70006F206C5F7F4F60936E2070936F20A80120
:107C8000C7010E94431480916E2090916F20080FCD
:107C9000191F00936E2010936F2042E050E060E0C7
:107CA00070E78EE690E20E9443142496CDBFDEBFBB
:107CB000DF91CF911F910F91FF90EF90DF90CF90C8
:107CC0000895CF92DF92EF92FF92CF93DF93C0900F
:107CD0006E20D0906F20E0E7DE1AE12CF12C4C15DD
:107CE0005D056E057F0580F46A017B01EC01BA0138
:107CF0007059A9010E94CD11CD28CE28CF2831F48A
:107D000089818057898302C080E001C081E0DF91D2
:107D1000CF91FF90EF90DF90CF90089581E0809316
:107D2000593184E090E0809338319093393189E083
:107D30008093373110923631089582E090E7809336
:107D40006E2090936F2042E050E060E070E78EE696
:107D500090E20C944314CF93DF931F92CDB7DEB71C
:107D600041E050E0BE016F5F7F4F8BE790E00E94E3
:107D7000691389818A3549F442E050E060E070E798
:107D80008EE690E20E94CD110CC0D7DF8AE5898390
:107D900041E050E0BE016F5F7F4F8BE790E00E94B3
:107DA000D8130F90DF91CF91089581E69EE30E9452
:107DB00015278EE60895C1DF84E6089581E080935B
:107DC000593184E090E0809338319093393188E0E4
:107DD000809337311092363110923531E091F03383
:107DE000F091F1338485882381F041E050E065E033
:107DF00070E087E391E30E94CD1142E050E066E03D
:107E000070E088E391E30C94CD11089581E08093B4
:107E1000593184E490E0809338319093393188E08F
:107E2000809337311092363110923531089581E0C8
:107E30008093593182E090E08093383190933931CA
:107E400088E1809337311092363110923531E091CC
:107E5000F033F091F1338485882381F041E050E0E4
:107E600065E070E087E391E30E94CD1142E050E0CD
:107E700066E070E088E391E30C94CD11089581E011
:107E80008093593182E490E0809338319093393176
:107E900088E1809337311092363110923531089550
:107EA00081E08093593124E030E0209338313093E1
:107EB000393198E0909337311092363180933531D3
:107EC00040E060E070E08FEF8CDEE091F033F09105
:107ED000F1338485882381F041E050E065E070E073
:107EE00087E391E30E94CD1142E050E066E070E04C
:107EF00088E391E30C94CD11089581E0809359318A
:107F000082E090E0809338319093393188E180931A
:107F100037311092363140E060E070E08FEF61DE83
:107F2000E091F033F091F1338485882381F041E0D2
:107F300050E065E070E087E391E30E94CD1142E0FC
:107F400050E066E070E088E391E30C94CD11089571
:107F500081E080935931089508958F929F92AF9256
:107F6000BF92CF92DF92EF92FF920F931F93CF9326
:107F7000DF93CDB7DEB76297CDBFDEBFFC01909136
:107F8000593167307105E1F48081992311F086320F
:107F900011F08235A9F421E0911120E020933631CF
:107FA000992311F0863211F0823551F490913831D5
:107FB00080913931908381838FEF80933A3136C03D
:107FC0005B018F01953009F4D9C050F49230A1F1D2
:107FD000C8F0933009F4ABC0943009F4C4C0DDC4D8
:107FE000983009F476C038F4963009F4D2C097304E
:107FF00009F4E3C0D2C4993009F4EBC39D3008F40E
:108000000FC4CBC4892F80958170809336318081D5
:10801000992311F0863219F0823509F0B8C4909195
:10802000383180913931F8019083818384E08093E5
:10803000593180E190E077C78081982F9D7F9134FE
:10804000C1F18033C1F462E070E0CF01ECD7882346
:1080500009F1F8016181F0E16F9FB001112440E165
:1080600050E0C8010E94CD1160E170E0C801B0D7B6
:1080700080E990E058C7803A79F0803509F055C022
:10808000F801818181114EC062E070E0C801CBD758
:10809000811111C081E03CC362E070E0CF01C3D721
:1080A0008823C1F3F80181818093503183E080936C
:1080B00059318AE02EC3E091C524F091C62430974F
:1080C00029F040E060E070E081E9199510925931A3
:1080D00064C48081803509F4F3C064E0C8010E9463
:1080E000B850F8018081803309F4F6C0803A09F471
:1080F000BAC1803C09F4D2C1813C09F4DBC1823CA5
:1081000009F4EAC1803B09F4FAC190EA980F923071
:1081100008F421C2803509F028C3F8018181882341
:1081200009F4F9C2F801108298C384E0F1C260E159
:1081300070E0CF0178D7882389F08091ED338111E9
:108140000BC060915031F0E16F9FB001112440E10C
:1081500050E0C8010E9443148AE001C081E0F801A8
:10816000808382E078C3909136318081911102C082
:108170008632C9F0823509F01DC415C090913631A0
:108180008081911102C0863271F0823509F0C0C43D
:108190000AC0909136318081911102C0863219F067
:1081A000823509F0CEC22091383180913931F80101
:1081B0002083818381E08927E7C388E0A1E7B9E3D1
:1081C00001900D928A95E1F7C8010E949C4D7801BB
:1081D000F4E0EF0EF11C64E0C7010E94B850E0919A
:1081E000C524F091C624309721F044E0B70180EA1D
:1081F0001995F80194818091513198133FC0958170
:108200008091523198133AC09681809153319813DE
:1082100035C0978180915431981330C08091553189
:108220008083809156318183809157318283809100
:108230005831838364E0C8010E94D152E091C52483
:10824000F091C624309721F044E0B80181EA1995F5
:1082500088E08093593180916739886080936739CD
:1082600084E0F801A9E7B9E301900D928A95E1F75E
:1082700046E167E679E381EAB4DC43C2E091C524D4
:10828000F091C624309729F044E061E571E380EC79
:1082900019951092793910927A3910927B3910928F
:1082A0007C3946E167E679E380EC9BDC81E08093F2
:1082B000593180913531882309F46FC386E064C356
:1082C000818181110ACF8281873509F006CF8381B0
:1082D0008D3C09F002CF26C262E070E0C801A3D64F
:1082E000882309F4AEC042E0B80180E87ADCF801E6
:1082F000618167FD04C0862F8370833029F0862F4B
:108300008F708F3009F07FC06093503180913B3186
:1083100090913C3120913D31382F32953095492F45
:108320004327407F09F03FC032273F70E1F5929527
:1083300090959227907FB9F5362F67FD02C0337074
:1083400003C03F7009F033E08095422F42954F7093
:108350003323B1F090E0032E02C0959587950A94DF
:10836000E2F7E22FF0E0032E02C0F595E7950A94BC
:10837000E2F72E2F50E002C0559547953A95E2F767
:1083800040FBCC24C0F8D12CF601EE0FFF1FEE0FFE
:10839000FF1F20FBEE24E0F8F12CEE0CFF1CEE2971
:1083A0008170E82B01C0E7E0F0E080914F31EE0FE3
:1083B000FF1FE057FF4DE80FF11D8081F801980184
:1083C000205F3F4F1192E217F307E1F790913E31A2
:1083D000F801918782FF09C090913B31968390917B
:1083E0003C31978390913D31908784FF15C0636045
:1083F000F0E16F9FB0011124665F7F4F46E050E0CF
:10840000C8010A9607C080E1689FB001112440E1CD
:1084100050E0C8010E94CD1160E170E0C801D8D5DC
:10842000E091C524F091C624309721F042E1B801D3
:1084300080E8199562E1C8010E94D15280E990E17B
:1084400072C50E94C34F91E08927F8018083E091B3
:10845000C524F091C624309709F4FFC144E0B80167
:1084600081EC1995FAC162E070E0C801DCD588237F
:1084700009F440C0F8018181811106C01092593180
:108480000E94C34F94E043C142E0B80181E8A9DBF8
:10849000F80181818093503189E029C062E070E069
:1084A000C801C1D5882331F1F80181818093503111
:1084B0008BE01DC062E070E0C801B5D58823D1F023
:1084C000F801818180935031FAE0FF2EF09259310A
:1084D0000E94C34F8F251CC162E070E0C801A3D584
:1084E000882341F0F8018181809350318CE08093A2
:1084F000593125C0E091C524F091C62424C062E022
:1085000070E0C80190D5E091C524F091C62488237D
:10851000D1F0309721F044E0B80186E819958091B8
:10852000ED3381110CC0F8016181F0E16F9FB00162
:10853000112440E150E08FE391E30E9443140E9434
:10854000C34F9AE0E4C0309709F4DEC044E0B801BC
:1085500081EC1995D9C062E070E0C80164D5882328
:1085600009F4D2C0F8018081803621F0EAE3AE2E12
:10857000B12C03C070E3A72EB12CF801D1806D2D72
:10858000D7FE0CC0607FF0E16F9F7001112480EC7A
:10859000A80EB11C66EF862E912C08C06C7F90E16E
:1085A000699F7001112456E3852E912CE091C5241A
:1085B000F091C624309721F042E0B80180E9199586
:1085C000F8018081817080934F31C70144E0969516
:1085D00087954A95E1F78093503190913A319817F9
:1085E00069F0B4016E0D7F1D44E050E08BE391E330
:1085F0000E94CD118091503180933A3168E0CE01D4
:1086000001960E944E118091EC3344E050E0873097
:1086100019F463E070E002C060E070E0CE010F96F4
:108620000E94CD11B5016E0D7F1D46E050E0CE01D8
:1086300009960E94CD118981809351318A8180935E
:1086400052318B81809353318C818093543160E41B
:1086500081E591E30E94EB54809151318093553133
:1086600080915231809356318091533180935731AC
:10867000809154318093583160E285E591E30E9406
:10868000EB548F859889A989BA8980936939909329
:108690006A39A0936B39B0936C3980914F31805A0D
:1086A000846080936739D092683984E0FE01319606
:1086B000ADE6B9E301900D928A95E1F720E0AE01B5
:1086C0004F5F5F4FBE01615F7F4FCE01099689D733
:1086D0008981F80180838A8181838B8182838C8167
:1086E0008383E058FF4F8D81808331968E81808314
:1086F00031968F81808331968885808387E080934F
:10870000593180E290E10FC40E94C34F91E0892764
:10871000F8018083A2C062E070E0C80184D488239D
:1087200009F4B8CC10925931E091C524F091C624D7
:10873000309709F432C140E060E070E081E91995BA
:108740002CC1803409F42CC1803509F499CCF0E2B5
:10875000AF16B104D1F0F8E1AF16B10409F4B6C315
:1087600090E3A916B10408F07EC3A501495F5F4FED
:1087700033E0569547953A95E1F7E091C524F0919D
:10878000C624309711F581E0FFC090EA980F92302F
:1087900008F466C2982F9F77903309F425C3803A76
:1087A00009F422C390E4980F933008F41DC3803E6F
:1087B00009F04FC38091373185FD28C3E091C5246E
:1087C000F091C6243097F9F244E0B80182E9199596
:1087D000DACF62E1CF010E94B85060E170E0C801D9
:1087E00022D4E091C524F091C624882339F1309732
:1087F00021F042E1B80181E819958091ED338111B2
:108800000BC060915031F0E16F9FB001112440E145
:1088100050E0C8010E9443140E94C34F9AE017C061
:1088200066E0CF010E94B85064E070E0C801FBD35D
:10883000811116C0E091C524F091C624309721F033
:1088400044E0B80181EC19950E94C34F91E089275B
:10885000F801808388E08093593184E090E063C31D
:1088600060915031F0E16F9FB001112440E150E080
:108870008FE391E30E94CD1190913F31809143317C
:108880008095981326C380914731981322C3909105
:10889000403180914431809598131BC380914831B9
:1088A000981317C390914131809145318095981369
:1088B00010C38091493198130CC39091423180913B
:1088C00046318095981305C380914A31981301C3AE
:1088D00090914B3180914C3180959813FAC28091E0
:1088E0004D319813F6C280914E3180959813F1C2A4
:1088F000C0903F31D0904031E0904131F090423112
:10890000F80180809180A280B380809159318B30B2
:1089100009F0E3C2E091C524F091C624309721F01C
:1089200046E0B80185E81995C818D908EA08FB0897
:10893000C0923F3133272F2D1E2D0D2D0093403136
:10894000A70166277727409341318F2D9927AA27C2
:10895000BB2780934231EC2DE095E0934331E02F2B
:10896000E095E0934431E42FE095E0934531E82F22
:10897000E095E0934631C0924731009348314093EF
:10898000493180934A3188E08093593106C0803460
:1089900021F48091C124811108C080E090E0C3C21D
:1089A0009091C124992309F4B8C282E0809359318F
:1089B0008AE0AECE833909F089CB8091EC338730E1
:1089C00009F0A1C043E050E060E070E0CE01029603
:1089D0000E94CD1188E88983F8019181903219F0C5
:1089E000903761F024C0F80180833A8131832B8174
:1089F00022839C8193832327822700C1F8018281EF
:108A0000883809F028C193818A81981324C1948100
:108A10008B81981320C195818C8198131CC184E0AF
:108A2000808361E070E0C801D3D285E09FC0E92E69
:108A3000E294BFE0EB22EA94EA949F70F92E88E07A
:108A400090E08F1991092FEF30E0690102C0D594B1
:108A5000C7948A95E2F7F5E0EF1629F084E0E81272
:108A60002AC0FF20E1F044E050E0B8016E5F7F4F84
:108A7000CE0101960E941176892B61F49A818B8137
:108A8000892798E889279C818927F8019681892779
:108A90008C2189F1F4E0EF120EC0F110DCC044E04B
:108AA00050E0B8016E5F7F4FCE0101960E941176B3
:108AB000892B09F1D0C083E08E1508F4CCC0F12CCD
:108AC000A701B8016E5F7F4FCE0101960E9411761B
:108AD000892B09F0C0C0D801AE0DBF1DE1E0F0E068
:108AE000EC0FFD1FEE0DFF1D12969C9180818927D2
:108AF000C82209F0B0C098E8F80190833A81318328
:108B00002B81228377C044E050E060E070E007C032
:108B1000853909F0DBCA44E050E063E070E0CE0143
:108B200001960E94CD11F8018181803209F45BC069
:108B3000803701F5F8019281898198138CC0938167
:108B40008A81981388C094818B81981384C0958101
:108B50008C81981380C080913731808361E070E010
:108B6000C80136D28FEF80933A3186E08093593135
:108B700038E172C0E82EE294AFE0EA22EA94EA9487
:108B80008F70F82E88E090E08F1991092FEF30E078
:108B9000690102C0D594C7948A95E2F7F5E0EF1613
:108BA00099F184E0E81671F183E08E1508F453C062
:108BB000F12CA701B8016E5F7F4FCE0101960E9494
:108BC0001176892B09F047C0D801AE0DBF1DE1E039
:108BD000F0E0EC0FFD1FEE0DFF1D12969C918081C1
:108BE0008927C822C1F53981F80130832A81218380
:108BF0009B8192838C818383232792278927848377
:108C000038E22AC0FF20E1F044E050E0B8016E5F96
:108C10007F4FCE0101960E941176892B61F49981D4
:108C20008A8189279B8189279C818927F8019681E0
:108C300089278C21C1F2F4E0EF12B6CFF1100BC0FE
:108C400044E050E0B8016E5F7F4FCE0101960E9474
:108C50001176892B41F230E020E0832F922F63C1FF
:108C600062E070E0C801DFD1882309F413CAF8017B
:108C70008081803621F0FAE3AF2EB12C03C0E0E30F
:108C8000AE2EB12CF801D1806D2DD7FE0CC0607FC7
:108C9000F0E16F9F7001112480ECA80EB11C76EFFB
:108CA000872E912C08C06C7F90E1699F7001112480
:108CB00066E3862E912CE091C524F091C62430976E
:108CC00021F042E0B80180E91995F80180818170B6
:108CD00080934F31C70154E0969587955A95E1F7F7
:108CE00080935031B4016E0D7F1D44E050E08BE362
:108CF00091E30E94CD118091503180933A3168E028
:108D0000CE0101960E944E118091EC3344E050E078
:108D1000873019F463E070E002C060E070E0CE01DB
:108D20000F960E94CD11B5016E0D7F1D46E050E0FB
:108D3000CE0109960E94CD118981809351318A819B
:108D4000809352318B81809353318C818093543145
:108D500060E481E591E30E94EB548091513180936E
:108D600055318091523180935631809153318093A7
:108D70005731809154318093583160E285E591E319
:108D80000E94EB5487E0809359318981F8018083F8
:108D90008A8181838B8182838C8183838F8598896B
:108DA000A989BA898093693990936A39A0936B39FC
:108DB000B0936C3980914F31805A80936739D0924B
:108DC000683984E0FE013196ADE6B9E301900D9279
:108DD0008A95E1F7AE014F5F5F4FBE01615F7F4F44
:108DE000CE01099651D16FC081E08093593184E062
:108DF000F8018083E091C524F091C624309709F4EE
:108E00002CCD40E060E070E082EC2BCB62E070E0C3
:108E1000C80109D1882309F4B6CC80E1F801808328
:108E200088E7818380E8828380EA8383148240E13B
:108E300050E060E070E0C80105960E94CD11F80195
:108E4000608170E0C801C4D0F801808190E0029692
:108E500034C08A3C09F0B2CC62E070E0C801E3D0D3
:108E6000811131C090CCF801258130E043E0B69407
:108E7000A7944A95E1F7F9013996AE16BF0661F459
:108E8000F801E20FF31FE680F801319690E09E159D
:108E900021F011929F5FFBCFE12CF8018083F12C30
:108EA000EE0DFF1D8AE6818382E88283B7016D5F44
:108EB0007F4FC8018DD0C701059623E0880F991F09
:108EC0002A95E1F730C080E290E02DC088E190E083
:108ED0002AC00E94C34F96E0BACC8A3079F4E09160
:108EE000C524F091C624309721F046E0B80184E80B
:108EF0001995C80CD91CEA1CFB1C1ACD8C3009F042
:108F000017CDE091C524F091C624309709F410CD17
:108F100046E0B80187E819950BCDF0E2AF16B10431
:108F200009F019CC37CC6296CDBFDEBFDF91CF916F
:108F30001F910F91FF90EF90DF90CF90BF90AF9077
:108F40009F908F900895CF93DF932091EC3327303B
:108F500071F4EC0143E050E060E070E00E94CD115C
:108F600044E050E063E070E0CE01039604C044E0CA
:108F700050E060E070E0DF91CF910C94CD11CF9381
:108F8000DF931F92CDB7DEB72091EC33273029F461
:108F900047E050E060E070E015C0FC0130812181C5
:108FA00023273281232733812327298344E050E07C
:108FB00060E070E00E94431441E050E064E070E043
:108FC000CE0101960E9443140F90DF91CF91089536
:108FD00020E42093D00026EC2093D5002093D400E9
:108FE00021E02093D000DC01680F791FA617B70796
:108FF00041F0ED91F0E0EA50F84FE491E093D300B6
:10900000F5CFE091D500F0E0EA50F84FE491EC9311
:10901000E091D400F0E0EA50F84FE4911196EC931F
:109020001092D000089520E42093D00026EC2093E5
:10903000D5002093D40021E02093D000DC01680FFC
:10904000791FA617B70741F0ED91F0E0EA50F84F0D
:10905000E491E093D300F5CFE091D500F0E0EA5041
:10906000F84FE4918C918E130AC0E091D400F0E0A7
:10907000EA50F84FE49181E011969C919E1380E0B4
:109080001092D000817008958F929F92BF92CF92DC
:10909000DF92EF92FF920F931F93CF93DF93DC0148
:1090A0008C91D12C30E08695D7948695379586950E
:1090B000D794869537958695D794869537958695D6
:1090C000D7948695379511968C9111978695D7945C
:1090D000869537958695D794869537958695D794B6
:1090E000869537958695D7948695379512968C9167
:1090F0001297F0E010E08695F7958695179586957E
:10910000F795869517958695F79586951795869583
:10911000F7958695179513968C9113978695F795E5
:10912000869517958695F795869517958695F79563
:10913000869517958695F7958695179514968C9133
:10914000149790E020E086959795869527958695CB
:1091500097958695279586959795869527958695D3
:109160009795869527951596EC91E6959795E695B2
:109170002795E6959795E6952795E6959795E69533
:109180002795E6959795E69527954B01DA014C5F73
:109190005F4F0C91E401B9904E01B026C32FD0E08F
:1091A000BE0160507F4D7B01612F70E060507E4DAD
:1091B000E701F880EB0188816F2D682BE22EF12CFE
:1091C000E701C050DD4D8881682B70E060527F4D13
:1091D000EB0188818695E7956F2F60718D2D817EDB
:1091E0006827892F80726827832F84796827812FC9
:1091F00083776827822F8A736827F62EF2946F256B
:10920000762F769576956727FB2CF6266695F626BB
:109210007D2D6F2F892FF694879567957795B69456
:10922000C72ED12CE601C050DF4D6E01E62EF12C89
:10923000E701C050DE4D7E01E601F881E70198812B
:10924000EF2EE92AC82ED12CE601C050DD4D9881C1
:10925000E92AF12CE701C052DF4D98819695E795F8
:10926000F12FF071932F917EEF2EE926922F9072BD
:10927000E926972F9479E926962F9377E926982F58
:109280009A73E926FE2CF294EF24CE2CC694C69451
:10929000EC24FB2CFE24E694FE24F69427951795E7
:1092A0003795B694C32ED12CE601C050DF4D6E0128
:1092B000E12EF12CE701C050DE4D7E01E601F88180
:1092C000E7019881EF2EE92AC22ED12CE601C05089
:1092D000DD4D9881E92AF12CE701C052DF4D9881DC
:1092E0009695E795F62FF071972F917EEF2EE92650
:1092F000982F9072E926932F9479E926912F9377EE
:10930000E926922F9A73E926FE2CF294EF24CE2CB4
:10931000C694C694EC24FB2CFE24E694FE24F82F7D
:10932000F694F79567957795B694872F90E0EC01C2
:10933000C050DF4D862F90E080509E4DF880EC01AC
:1093400088818F29EF2EF12CE701C050DD4D9881E7
:10935000892B90E080529F4DEC0188818695E7959E
:10936000912F9071832F817EE92EE826822F8072C3
:10937000E826872F8479E826862F8377E8268F2FA3
:109380008A73E826FE2CF294EF24CE2CC694C69461
:10939000EC24FB2CFE24E694FE24F69427951795E6
:1093A0003795B694832F90E0EC01C050DF4D812FAC
:1093B00090E080509E4DF880EC0188818F29E22E4C
:1093C000F12CE701C050DD4D9881892B90E080524F
:1093D0009F4DEC0188818695E795962F9071872F98
:1093E000817EF92EF8268F2F8072F826832F8479BC
:1093F000F826812F8377F826822F8A73F8269F2DEF
:109400009295F926EF2CE694E694FE249B2D9F2559
:10941000F6949F258F2F9695879567957795B694A7
:10942000C72ED12CE601C050DF4D6E01E62EF12C87
:10943000E701C050DE4D7E01E601F881E701988129
:10944000EF2EE92AC82ED12CE601C050DD4D9881BF
:10945000E92AF12CE701C052DF4D98819695E795F6
:10946000F12FF071932F917EF927922F9072F927A7
:10947000972F9479F927962F9377F927982F9A7336
:10948000F9279F2F9295F927FF2EF694F694FF2542
:109490009B2D9F27F6959F2796952795179537958E
:1094A000B694C32ED12CE601C050DF4D6E01E12EE3
:1094B000F12CE701C050DE4D7E01E601F881E701A5
:1094C0009881EF2EE92AC22ED12CE601C050DD4D45
:1094D0009881E92AF12CE701C052DF4D98819695D9
:1094E000E795F62FF071972F917E9F27F82FF07256
:1094F0009F27F32FF4799F27F12FF3779F27F22FE0
:10950000FA739F27F92FF2959F27F92FF695F69575
:109510009F27FB2DF9279695F927982F8F2F869552
:10952000979567957795D72EF62F672F70E0EB010B
:10953000C050DF4D6F2F70E060507E4DF880EB0122
:1095400088816F2D682BE92EF12CE701C050DD4D8D
:109550008881682B70E060527F4DEB018881869591
:10956000E795632F617E812F80718627622F60725D
:1095700086276D2D647986276F2F63778627692F5D
:109580006A738627682F62958627682F6695669589
:109590008627B694B8268695B826812FB694279547
:1095A00087953795182F0E270D934A175B0709F0FB
:1095B000F0CDD0925A31F0935B3190935C3130937F
:1095C0005D3180935E3120935F31DF91CF911F91A8
:1095D0000F91FF90EF90DF90CF90BF909F908F9072
:1095E00008958F929F92AF92BF92CF92DF92EF92A7
:1095F000FF920F931F93CF93DF93FC01C62FF42E9E
:10960000B52F8081A0E050E0869557958695A79567
:10961000869557958695A795869557958695A7958E
:10962000869557958695A7958181869557958695B8
:10963000A795869557958695A7958695579586956E
:10964000A795869557958695A795828130E040E04D
:10965000869547958695379586954795869537954E
:10966000869547958695379586954795869537953E
:1096700083818695479586953795869547958695F6
:10968000379586954795869537958695479586951E
:109690003795648190E080E066958795669597950B
:1096A000669587956695979566958795669597953E
:1096B0006695879566959795B5806B2D6695879588
:1096C000669597956695879566959795669587951E
:1096D000669597956695879566959795B62EEA2F28
:1096E000F0E0E050FF4D032F10E000501E4DD08100
:1096F000F8016081D62B092F10E000501D4DF801B4
:109700006081ED2FE62BF0E0E052FF4DC0800C2F82
:10971000172FCF2DDB2F7E01F4E0EF0EF11C7881A7
:10972000F801B1918F01B7276B2DC6946795F42F7F
:10973000F071E52FE17EFE27E82FE072FE27EA2F89
:10974000E479FE27E32FE377FE27E92FEA73FE276C
:10975000EF2FE295FE27DF2ED694D694FD25EB2F32
:10976000EF27F695EF2720FDEC25E69587954795A1
:109770005795B695C52ED12CF601E050FF4D6F01DF
:10978000A42EB12CF501E050FE4D5F01F601D08012
:10979000F501C080DC28E82FF0E0E050FD4DF081BD
:1097A000ED2DEF2BF0E0E052FF4DC080C6946795A1
:1097B000F32FF071EA2FE17EFE27E92FE072FE27FA
:1097C000E52FE479FE27E42FE377FE27E82FEA73FD
:1097D000FE27EF2FE295FE27DF2ED694D694FD25A7
:1097E000EB2FEF27F695EF27DA2E20FDEC25E695F7
:1097F00097953795D794CB2EC694AD2DB0E0A05059
:10980000BF4DE32FF0E0E050FE4DAC91E081EA2B3C
:10981000A92FB0E0A050BD4DFC91EF2BF0E0E0523D
:10982000FF4DB081B6956795F42FF071E52FE17E7D
:10983000FE27E82FE072FE27ED2DE479FE27E32FC7
:10984000E377FE27E92FEA73FE27EF2FE295FE2745
:10985000AF2FA695A695FA27EC2DEF27F695EF27C3
:1098600020FDEB27E695879547955795C694A52F3C
:10987000B0E0A050BF4DE42FF0E0E050FE4DAC91C1
:10988000E081EA2BA82FB0E0A050BD4DFC91EF2B5A
:10989000F0E0E052FF4DB081B6956795F32FF0717F
:1098A000ED2DE17EFE27E92FE072FE27E52FE4791A
:1098B000FE27E42FE377FE27E82FEA73FE27EF2F3A
:1098C000E295FE27AF2FA695A695FA27EC2DEF2758
:1098D000F695EF2720FDEB27E69597953795D794DA
:1098E000C694AD2DB0E0A050BF4DE32FF0E0E050A6
:1098F000FE4DAC91E081EA2BA92FB0E0A050BD4D08
:10990000FC91EF2BF0E0E052FF4DB081B6956795EA
:10991000F42FF071E52FE17EFE27E82FE072FE279D
:10992000ED2DE479FE27E32FE377FE27E92FEA7395
:10993000FE27EF2FE295FE27AF2FA695A695FA27D3
:10994000EC2DEF27F695EF2720FDEB27E695879581
:1099500047955795C694A52FB0E0A050BF4DE42F72
:10996000F0E0E050FE4DAC91E081EA2BA82FB0E092
:10997000A050BD4DFC91EF2BF0E0E052FF4DB081C7
:10998000B6956795F32FF071ED2DE17EFE27E92F57
:10999000E072FE27E52FE479FE27E42FE377FE2728
:1099A000E82FEA73FE27EF2FE295FE27AF2FA6954B
:1099B000A695FA27EC2DEF27F695EF2720FDEB274C
:1099C000E69597953795D794C694ED2DF0E0E05045
:1099D000FF4DA32FB0E0A050BE4DF081EC91EF2BD6
:1099E000A92FB0E0A050BD4DFC91EF2BF0E0E0526C
:1099F000FF4DB081B6956795F42FF071E52FE17EAC
:109A0000FE27E82FE072FE27ED2DE479FE27E32FF5
:109A1000E377FE27E92FEA73FE27EF2FE295FE2773
:109A2000AF2FA695A695FA27EC2DEF27F695EF27F1
:109A300020FDEB27E695879547955795A52FB0E034
:109A4000A050BF4DE42FF0E0E050FE4DAC91E0811E
:109A5000EA2BA82FB0E0A050BD4DFC91EF2BF0E019
:109A6000E052FF4DF081F6956795B62EED2DE17E23
:109A7000632F60716E27E92FE0726E27E52FE4797E
:109A80006E27E42FE3776E27E82FEA736E27E62F21
:109A9000E2956E27E62FE695E6956E27C694C626D4
:109AA0006695C62620FDCF26C69497953795D79400
:109AB000AD2DCD2CD12CF601E050FF4D6F01832E42
:109AC000912CF401E050FE4D4F01F601B081F401FC
:109AD0006081B62BC92ED12CF601E050FD4D60817E
:109AE000EB2FE62BF0E0E052FF4DC080E72FF0E0D7
:109AF000EA50F94FE491EC25EC837B257993EC1641
:109B0000FD0609F00CCE50935A3140935B3180939F
:109B10005C31A0935D3130935E3190935F31DF9182
:109B2000CF911F910F91FF90EF90DF90CF90BF905A
:109B3000AF909F908F900895BF92CF92DF92EF9257
:109B4000FF920F931F93CF93DF93A0915A315091BF
:109B50005B3110915C3140915D3130915E312091EB
:109B60005F31FC01BC016C5F7F4F0191952F9071BB
:109B70008A2F817E9827812F80729827842F84795D
:109B80009827832F83779827822F8A739827892F86
:109B900082959827892F869586959827C42ED12C53
:109BA000E601C050DF4D6E01E32EF12CE701C050FD
:109BB000DE4D7E01E601B881E7018881B82BE22EF7
:109BC000F12CE701C050DD4D8881CB2FC82BD0E0B0
:109BD000C052DF4DB881B027B92796959B270695CF
:109BE000812F969587955795A795B32FB071942F90
:109BF000917EB927922F9072B9279A2F9479B9271D
:109C0000952F9377B927982F9A73B9279B2F929501
:109C1000B9279B2F96959695B927CA2ED12CE60188
:109C2000C050DF4D6E01E52EF12CE701C050DE4D36
:109C30007E01E6011881E7019881192BE82EF12CAD
:109C4000E701C050DD4D9881C12FC92BD0E0C05233
:109C5000DF4D988190279B27B695B927B02EB694F3
:109C6000922FB695979537954795B52FB0712A2FB6
:109C7000217EB227282F2072B227242F2479B227E1
:109C8000232F2377B227292F2A73B2272B2F229530
:109C9000B2272B2F26952695B227C42FD0E08E0110
:109CA00000501F4D6801C32FD0E08E0100501E4DA3
:109CB0007801E6010881E7012881022BE92EF12CC9
:109CC000E701C050DD4D2881022B10E000521F4DEE
:109CD000E8012881C22FCB25CB27B695BC272B2D99
:109CE0002695B69587955795A795C32FC071B42F24
:109CF000B17EBC27C92FC072BC27CA2FC479BC272C
:109D0000C52FC377BC27C82FCA73BC27CB2FC295DA
:109D1000BC27CB2FC695C695BC27CA2FD0E0C05014
:109D2000DF4D052F10E000501E4DF880E80118812E
:109D3000F12A082F10E000501D4DE8011881CF2DA9
:109D4000C12BD0E0C052DF4DC881C227CB27B695CA
:109D5000BC272695B695979537954795C52FC07121
:109D6000BA2FB17EBC27C82FC072BC27C42FC479BC
:109D7000BC27C32FC377BC27C92FCA73BC27CB2FDF
:109D8000C295BC27CB2FC695C695BC27C42FD0E063
:109D9000C050DF4D032F10E000501E4DF880E80149
:109DA0001881F12A092F10E000501D4DE80118819B
:109DB000CF2DC12BD0E0C052DF4DC881C227CB27A9
:109DC000B695BC272695B69587955795A795D32F19
:109DD000D071B42FB17EDB27B92FB072DB27BA2F39
:109DE000B479DB27B52FB377DB27B82FBA73DB271E
:109DF000BD2FB295DB271D2F169516951D27CA2E50
:109E0000D12CE601C050DF4D6E01E52EF12CE701AB
:109E1000C050DE4D7E01E6010881E701B8810B2BC1
:109E2000E82EF12CE701C050DD4DB881C02FCB2BBF
:109E3000D0E0C052DF4DB881B227B127D12FD695DF
:109E4000DB27B22EB694D695979537954795D52FA3
:109E5000D0712A2F217ED227282F2072D227242F9B
:109E60002479D227232F2377D227292F2A73D22789
:109E70002D2F2295D2272D2F26952695BD2FB2273F
:109E8000C42FD0E08E0100501F4D6801C32FD0E0D9
:109E90008E0100501E4D7801E6010881E7012881FE
:109EA000022BE92EF12CE701C050DD4D2881022B59
:109EB00010E000521F4DE80118811B251B27DB2FE6
:109EC000D695D127D69587955795A795182F242FE6
:109ED000217E832F80712827892F807228278A2F3F
:109EE00084792827852F83772827812F8A7328272D
:109EF000B22FB2952B27B22FB695B6952B27EA2E07
:109F0000F12CE701C050DF4D7E01C52ED12CE601BA
:109F1000C050DE4D6E01E701E880E6018881E82A45
:109F2000C12ED12CE601C050DD4D8881E82AF12CEC
:109F3000E701C052DF4DB6948881CB2DC827C227D8
:109F40002695B22FBC272B2F2695979537954795A9
:109F5000292F6E177F0709F008CEA0935A3150932E
:109F60005B3110935C3140935D3130935E3190935F
:109F70005F31DF91CF911F910F91FF90EF90DF90B4
:109F8000CF90BF900895CF93DF93EAE5F1E3A081EE
:109F900071816281338124819581472F40718A2F9D
:109FA000817E8427462F40728427432F447984275B
:109FB000422F43778427492F4A738427482F42959D
:109FC0008427482F469546958427482F4695842711
:109FD000869567957795A795C32FD0E0C050DF4D44
:109FE000422F50E040505E4DB881EA018881B82B85
:109FF000492F50E040505D4DEA018881CB2FC82B9E
:10A00000D0E0C056DF4D88818695522F5071432F86
:10A01000417E4527592F507245275A2F547945279D
:10A02000572F53774527562F5A734527542F52954C
:10A030004527542F569556954527542F5695452715
:10A040004695979527953795CA2FD0E0C050DF4D9C
:10A05000472F50E040505E4DB881EA014881B42B53
:10A06000462F50E040505D4DEA014881CB2FC42B74
:10A07000D0E0C056DF4D4881842B8695572F507114
:10A080004A2F417E4527562F50724527532F54792A
:10A090004527522F53774527592F5A734527542F59
:10A0A00052954527542F569556954527542F56952A
:10A0B0004527469567957795A795C32FD0E0C05063
:10A0C000DF4D422F50E040505E4DB881EA0148819B
:10A0D000B42B492F50E040505D4DEA014881CB2F11
:10A0E000C42BD0E0C056DF4D4881842B8695CA2F03
:10A0F000D0E0C050DF4D472F50E040505E4DB8815A
:10A10000EA014881B42B462F50E040505D4DEA01F2
:10A110004881CB2FC42BD0E0C056DF4D4881842B23
:10A12000532F517E422F40714527592F507245279A
:10A130005A2F54794527572F53774527562F5A734F
:10A140004527542F52954527542F56955695452708
:10A15000542F569545274695979527953795A08373
:10A1600071836283338324839583DF91CF91089534
:10A17000BF92CF92DF92EF92FF920F931F93CF93F4
:10A18000DF9350915A31C0915B31B0905C31409176
:10A190005D3130915E3120915F31FC01615008F4F6
:10A1A000EAC19C2F9071852F817E98278B2D80721C
:10A1B0009827842F84799827832F83779827822F55
:10A1C0008A739827892F82959827792F7695769587
:10A1D0009727892F86959827AC2F8B2D9695879555
:10A1E000A7955795C42FD0E0C050DF4D032F10E046
:10A1F00000501E4D7881E8019881792B022F10E0E4
:10A2000000501D4DE8019881C72FC92BD0E0C054E4
:10A21000DF4D18811695732F7071942F917E9727BB
:10A22000722F70729727752F747997277A2F73770B
:10A230009727782F7A739727792F72959727792FF9
:10A24000769576959727792F76957927922F272FD0
:10A250002695979537954795C52ED12CE601C05088
:10A26000DF4D6E01EA2EF12CE701C050DE4D7E017C
:10A27000E6017881E7012881722BE82EF12CE701B5
:10A28000C050DD4D2881C72FC22BD0E0C054DF4D18
:10A290002881122B16957A2F7071252F217E272762
:10A2A000782F70722727742F74792727732F73776D
:10A2B0002727792F7A732727722F72952727722FD6
:10A2C000769576952727722F76952727BA2F26958C
:10A2D0008795B7955795C42ED12CE601C050DF4D18
:10A2E0006E01E32EF12CE701C050DE4D7E01E60148
:10A2F0007881E7012881722BE92EF12CE701C0500B
:10A30000DD4D2881C72FC22BD0E0C054DF4DA8817E
:10A31000A12BA695732F7071242F217E2727792FCB
:10A3200070722727752F747927277B2F737727273C
:10A33000782F7A732727722F72952727722F769599
:10A3400076952727722F76957227232F372F3695EC
:10A35000979527954795C52FD0E0C050DF4D0B2F1F
:10A3600010E000501E4D7881E8013881732B082FD2
:10A3700010E000501D4DE8013881C72FC32BD0E0FD
:10A38000C054DF4DD881AD2BA6957B2F7071352F32
:10A39000317E3727782F70723727742F74793727DB
:10A3A000722F73773727792F7A733727732F729528
:10A3B0003727732F769576953727732F769537271E
:10A3C00036958795B7955795C42FD0E0C050DF4D8F
:10A3D000022F10E000501E4D7881E8013881732B68
:10A3E000092F10E000501D4DE8013881C72FC32B05
:10A3F000D0E0C054DF4DD881AD2BA695722F70717F
:10A40000342F317E7327392F30727327352F3479EB
:10A4100073273B2F33777327382F3A737327372FE0
:10A4200032957327372F369536957327372F369504
:10A430007327342F7695979527953795C52FD0E0BC
:10A44000C050DF4D0B2F10E000501E4D7881E80109
:10A450004881742B082F10E000501D4DE801488101
:10A46000C72FC42BD0E0C054DF4DD881DA2BD6954E
:10A470007B2F7071452F417E7427482F40727427BF
:10A48000432F44797427422F43777427492F4A7307
:10A490007427472F42957427A72FA695A6957A274C
:10A4A000472F469574274B2F769587954795579557
:10A4B000C42FB82EA32FB0E08D0100501F4D6801AE
:10A4C000A22FB0E08D0100501E4D7801D6010C91F5
:10A4D000D7018C91082BE92EF12CD701A050BD4D4E
:10A4E0008C91082B10E000541F4DD8018C91D82B73
:10A4F000D695732F717E822F80717827892F807275
:10A500007827852F84797827842F837778278B2D58
:10A510008A737827872F82957827A72FA695A695E7
:10A520007A27872F86957827432F322F272F269536
:10A53000979537954795292F852F90E080509F4D0F
:10A540000C2F10E000501E4DDC019C91D8018C9125
:10A55000892B0B2D10E000501D4DD8019C91892BAB
:10A5600090E080549F4DDC019C918D2F892B908130
:10A570008927819313CE50935A31C0935B31B092A7
:10A580005C3140935D3130935E3120935F31DF91D8
:10A59000CF911F910F91FF90EF90DF90CF90BF90E0
:10A5A0000895EF92FF920F931F93CF93DF937091D3
:10A5B0005A3150915B3120915C3140915D31309145
:10A5C0005E31C0915F31E42FF0E0E050FF4DA32FEA
:10A5D000B0E0A050BE4DF081EC91EF2BAC2FB0E07D
:10A5E000A050BD4DFC91EF2BF0E0E052FF4D1081EB
:10A5F000DC01D0E0615008F4DBC11695D795952FAA
:10A600009071872F817E8927922F90728927942FAE
:10A6100094798927932F937789279C2F9A73892779
:10A62000982F92958927E82FE695E6958E27982F03
:10A63000969589278695279557957795D695932F43
:10A640009071842F817E89279C2F90728927972F64
:10A6500094798927952F93778927922F9A73892741
:10A66000982F92958927E82FE695E6958E27982FC3
:10A67000969589279C2F8695979537954795E72F2F
:10A68000F0E0E050FF4D052F10E000501E4DC0815E
:10A69000F8018081C82B022F10E000501D4DF801F9
:10A6A0008081EC2FE82BF0E0E054FF4D8081D82B27
:10A6B000D695E52FE071872F817E8E27E22FE072FD
:10A6C0008E27E42FE4798E27E32FE3778E27E92F77
:10A6D000EA738E27E82FE2958E27E82FE695E69518
:10A6E0008E27E82FE6958E2786952795579577959F
:10A6F000E42FF0E0E050FF4D032F10E000501E4D1E
:10A70000C081F8018081C82B092F10E000501D4D39
:10A71000F8018081EC2FE82BF0E0E054FF4D8081C0
:10A72000D82BD695E32FE071842F817E8E27E92FD9
:10A73000E0728E27E72FE4798E27E52FE3778E27C7
:10A74000E22FEA738E27E82FE2958E27E82FE69511
:10A75000E6958E27E82FE6958E278695979537956F
:10A760004795E72FF0E0E050FF4D052F10E0005037
:10A770001E4DC081F8018081C82B022F10E00050CF
:10A780001D4DF8018081EC2FE82BF0E0E054FF4DE7
:10A790008081D82BD695E52FE071872F817E8E277B
:10A7A000E22FE0728E27E42FE4798E27E32FE37700
:10A7B0008E27E92FEA738E27E82FE2958E27E82F60
:10A7C000E695E6958E27E82FE6958E2786952795C0
:10A7D00057957795E42FF0E0E050FF4D032F10E000
:10A7E00000501E4DC081F8018081C82B092F10E058
:10A7F00000501D4DF8018081EC2FE82BF0E0E05473
:10A80000FF4D8081D82BD695E32FE071842F817E78
:10A810008E27E92FE0728E27E72FE4798E27E52F28
:10A82000E3778E27E22FEA738E27E82FE2958E27B3
:10A83000E82FE695E6958E27E82FE6958E278695F4
:10A84000979537954795E72FF0E0E050FF4D052F9E
:10A8500010E000501E4DC081F8018081C82B022FEE
:10A8600010E000501D4DF8018081EC2FE82BF0E046
:10A87000E054FF4D8081D82BD695E52FE071872FCE
:10A88000817E8E27E22FE0728E27E42FE4798E27D7
:10A89000E32FE3778E27E92FEA738E27E82FE295DF
:10A8A0008E27E82FE695E6958E27E82FE6958E27EA
:10A8B0008695279557957795E42FF0E0E050FF4D6A
:10A8C000032F10E000501E4DC081F8018081C82B7D
:10A8D000092F10E000501D4DF8018081EC2FE82B6E
:10A8E000F0E0E054FF4D8081D82BD695E72FF0E0C3
:10A8F000E050FF4D052F10E000501E4DC081F801C3
:10A900008081C82B022F10E000501D4DF80180817E
:10A91000EC2FE82BF0E0E054FF4D8081D82BE42FA2
:10A92000E17E832F8071E827892F8072E827872FA7
:10A930008479E827852F8377E827822F8A73E82791
:10A940008E2F8295E8278E2F86958695E8278E2F65
:10A950008695E827E695979537954795C92FE42F73
:10A96000F0E0E050FF4D832F90E080509E4D10812D
:10A97000FC018081182B8C2F90E080509D4DFC01B4
:10A980008081E12FE82BF0E0E052FF4D10818C91A7
:10A99000E82FF0E0EA50F94FE4917D01F0E8EF0E86
:10A9A000F11C9E2F9127F70190838D278D9322CE46
:10A9B00070935A3150935B3120935C3140935D31F9
:10A9C00030935E31C0935F31DF91CF911F910F9132
:10A9D000FF90EF9008950F931F93FC01862F408105
:10A9E0005181628173818B0122273327803208F4E1
:10A9F00071C0D80123E0B695A7952A95E1F70A27FB
:10AA00001B2798013695279536952795BBE07695B7
:10AA1000679557954795BA95D1F70227132720E0F8
:10AA200030E095E1000F111F221F331F9A95D1F7D7
:10AA3000402B512B622B732B8B0122273327D801FC
:10AA400033E0B695A7953A95E1F70A271B279801B9
:10AA50003695279536952795BBE07695679557955A
:10AA60004795BA95D1F70227132720E030E095E10A
:10AA7000000F111F221F331F9A95D1F7402B512B26
:10AA8000622B732B8B0122273327D80133E0B69535
:10AA9000A7953A95E1F70A271B2798013695279540
:10AAA00036952795BAE07695679557954795BA9567
:10AAB000D1F70227132720E030E096E1000F111FA5
:10AAC000221F331F9A95D1F7402B512B622B732BEA
:10AAD000805289CF40835183028373831F910F91EA
:10AAE0000895AF92BF92CF92DF92EF92FF920F93B1
:10AAF0001F93CF93DF936730710509F451C09B0119
:10AB000027703327232B09F04EC05B016C01EB014A
:10AB100083E0D695C7958A95E1F77B0196E0F69498
:10AB2000E7949A95E1F7EC0EFD1EEC0CFD1C8E01EE
:10AB3000015011090C0D1D1DA701401B510B60E0B8
:10AB400070E0C80101960E9438760C151D0520F1B1
:10AB5000D801EC91F0E0EA50F94F2491D701CD01F2
:10AB60000A171B0768F4FC018081982F990F8E91BA
:10AB7000881F8827881F892B11968C931197EFCFF8
:10AB800011968C9111978E7FE22FE170E82B119630
:10AB9000EC9301501109D9CFC5018C0F9D1F04C042
:10ABA00087E090E001C0CB01DF91CF911F910F9121
:10ABB000FF90EF90DF90CF90BF90AF900895CF932C
:10ABC000DF93EC0182EC888361E070E0CE010E94AB
:10ABD000E8478AE080933A3210923B3268E170E0B5
:10ABE000CE01DF91CF917DCFEF92FF920F931F9314
:10ABF000CF93DF93EC01CB0168307105D8F169E0A8
:10AC000070E00E946875DE0180E090E008E010E0EE
:10AC10008617970751F1FC0133E0F695E7953A95D1
:10AC2000E1F7E80FF91FAC0147705527EC0FFD1F46
:10AC3000208130E0042E02C0359527950A94E2F772
:10AC40002C934115510571F0E181F0E07801E41A8F
:10AC5000F50AA7017F0102C0EE0CFF1C4A95E2F73E
:10AC60002E292C9301961196D3CF23E0880F991F9C
:10AC70002A95E1F7DF91CF911F910F91FF90EF900F
:10AC80000895EF92FF920F931F93CF93DF939C0150
:10AC9000CB016730710509F440C069E070E00E94A3
:10ACA000687580E090E048E050E086179707A9F1CA
:10ACB000DC01E3E0B695A795EA95E1F7A80FB91F87
:10ACC000EC01C770DD27A20FB31FEC91F0E00C2E52
:10ACD00002C0F595E7950A94E2F7209759F011968E
:10ACE0000C9111977A01EC1AFD0A01C0000FEA9449
:10ACF000EAF7E02BF0E0EA50F94FE4911196AC91BD
:10AD0000B0E002C0B595A795CA95E2F7ED01CE2750
:10AD1000FE01E0FD04C00196C8CF81E001C080E0E3
:10AD2000DF91CF911F910F91FF90EF9008951092B6
:10AD30003A32089510923A321092603110923B32BA
:10AD40000895F8DF0E94593310923A320895089519
:10AD50000895DC0123E633E66150E8F04D91942F2D
:10AD6000922780E1989FA00111244927E42FF0E069
:10AD7000232F332742954F70C9018427AC013E2F02
:10AD800022272427352743E0EE0FFF1F4A95E1F7DE
:10AD90002E273F27E1CFC9010895EF92FF921F931D
:10ADA000CF93DF93EC017B0180913B32882339F014
:10ADB00080913A32823008F0DBC010923B32E114CD
:10ADC000F10461F0B701CE015CDF882309F4D3C040
:10ADD000B701CE0109DF7C0181E001C082E0109162
:10ADE0003A32163090F4133070F51230A8F484E043
:10ADF00090E080936C2090936D2082E5888382E0C0
:10AE000080933A3287E090E0C9C0193008F467C0F7
:10AE10001A3009F496C0ACC090E1E916F10411F4BF
:10AE200080FD03C010923A3292C08881998180934C
:10AE30002C3290932D3283E9888380E2898383E0EA
:10AE400080933A326AC080FFEDCF88E2E816F104C1
:10AE500048F32881898182279A8189279B818927C4
:10AE60009C818913DFCFA12FB0E01397CD01880F0C
:10AE7000991FA80FB91FA15DBD4C283821F483E0AC
:10AE8000FE01319602C084E0FE0101900D928A9588
:10AE9000E1F745E050E0BE01CE0102960E94277620
:10AEA000133021F0143021F485E903C083E901C097
:10AEB00087E9888380E7898367E070E0CE010E949C
:10AEC000E84780913A328D5F80933A3268E470E0CF
:10AED000CE01DF91CF911F91FF90EF9002CE80FFC6
:10AEE000A1CF98E1E916F10409F09CCF63E0CE010F
:10AEF00030DF009709F096CF288122FF11C018306B
:10AF000079F0163011F485E901C087E9888380E281
:10AF100089832EEF210F20933A3260E170E0D8CF81
:10AF200021E020933B32212F30E026503109322F8F
:10AF3000330F230F2C5F20933932288120932E3238
:10AF40002DC0982F927031F081E080933A320E94A8
:10AF500052330EC080FF05C063E0CE01FADE892BBC
:10AF600099F3CE01DF91CF911F91FF90EF9027CE03
:10AF700080E090E013C0E091C524F091C6243097A2
:10AF800059F0A701495F5F4F63E0569547956A9571
:10AF9000E1F7BE0181EC199580E021CFDF91CF91DF
:10AFA0001F91FF90EF9008959F92AF92BF92CF9222
:10AFB000DF92EF92FF920F931F93CF93DF93CDB762
:10AFC000DEB7C756D109CDBFDEBF8C017B01FB01C7
:10AFD00060817181E2DED0903B32DD2009F449C10D
:10AFE00080913A329AEF980F933008F057C0F801E9
:10AFF00080818072C82E10921C3259E2A52E54E135
:10B00000B52E912C47E650E0B501CE0101960E9485
:10B01000F0758B81882349F029813A8180912C3207
:10B0200090912D3228173907B9F48D81882329F0A2
:10B030009C8180912E3298130FC08F89882311F044
:10B04000CC2051F0E0911C3281E08E0F80931C32B5
:10B05000F0E0E35EFD4C90829394F7E6AF0EB11CF6
:10B060008FE09812CFCFC1100DC080913A329AEF85
:10B07000980F943008F0B0C020911C32EDE1F2E35B
:10B0800080E091C080EEF801808380E8818362E0F7
:10B0900070E0C8010E94E84789E097C0893029F72D
:10B0A000F70160817181C801ECDDF7016081718178
:10B0B000811117C0CB01089667E070E00E946875A7
:10B0C000462FE091C524F091C624309719F0B801BD
:10B0D00081EC1995C80173DDF70180839183D12C30
:10B0E000CBC0C80181DDF70180839183F8016081C5
:10B0F000262F30E043E0969587954A95E1F7029731
:10B100002817390739F76E5FC80123DE892B11F73D
:10B11000C12C97E6992E5801FFEFAF1ABF0A809114
:10B120001C32C81608F0A1CFEC2DF0E0E35EFD4C18
:10B130006081969EB0011124675D7B4E47E650E02A
:10B14000CE0101960E94F0758F89882349F14E89BE
:10B1500050E0F801808190E001974817590741F0CD
:10B1600020911C32422F50E0415051093C2D08C023
:10B17000B501CE0106960E941176892B89F710C081
:10B18000832F90E0841795073CF4FC01E35EFD4CAF
:10B19000818180833F5FF4CF215020931C32CA9479
:10B1A000C394BDCF8F5F821709F466C0919194500C
:10B1B0009230C0F782E0F801808380E6818362E00C
:10B1C00070E0C8010E94E8478BE080933A3260E269
:10B1D00070E0C80186DC80CF8B3009F04DC0F701EC
:10B1E000608171816115710509F440C0C80149DDB4
:10B1F000D82EF70160817181811115C0CB010896AD
:10B2000067E070E00E946875462FE091C524F091D8
:10B21000C624309719F0B80181EC199510921C32B0
:10B22000C801CDDC26C0C801DFDCF7018083918333
:10B23000BC0183E0769567958A95E1F7C80189DDC1
:10B24000892B19F010921C3245CFF8018581882393
:10B2500031F0813059F480931C3285E004C081E0E4
:10B2600080931C3284E080931D3206C010921C3201
:10B2700003C0F701808391838D2DC959DF4FCDBF66
:10B28000DEBFDF91CF911F910F91FF90EF90DF9084
:10B29000CF90BF90AF909F9008955F926F927F92F2
:10B2A0008F929F92AF92BF92CF92DF92EF92FF92D6
:10B2B0000F931F93CF93DF93CDB7DEB7C254D24025
:10B2C000CDBFDEBF7C01CF5BDD4F68837983C15486
:10B2D000D24080916031843009F48BC140F48230D7
:10B2E00009F4D6C008F060C1813051F08CC48630BA
:10B2F00009F41EC308F446C2873009F4C8C383C4E6
:10B300000091D4331091D53301151105C1F0A80176
:10B31000495F5F4F63E0569547956A95E1F762EDA7
:10B3200072E3C7010E941E766091D4337091D533C9
:10B33000C701D7DB1092D4331092D53321C2CF5B33
:10B34000DD4F68817981C154D2406115710509F4DE
:10B35000C7C0C70196DCD82ECF5BDD4F68817981ED
:10B36000C154D240C70140DCCF5BDD4F8883998355
:10B37000C154D2409C01295F3F4FC901880F991FDA
:10B3800053E0969587955A95E1F706968138910591
:10B3900078F062E274E2CE0101960E944A76109241
:10B3A0006031BE016F5F7F4F85E60E94092A6CC441
:10B3B000B3E036952795BA95E1F7A70160E870E00C
:10B3C000CE0101960E9468117C01CF5BDD4F888120
:10B3D000C154D240CE5BDD4F9881C254D240CF5F82
:10B3E000DD4F9883C150D240CE5FDD4F8883C2507D
:10B3F000D24081E394E29F938F9380E8A82EB12CF2
:10B40000C5018E199F099F938F9381E090E08C0F67
:10B410009D1F8E0D9F1D9F938F930E945176E80E66
:10B42000F91EB5016E197F0922E030E0AE014F5FD1
:10B430005D4F81E090E08C0F9D1F8E0D9F1D0E943F
:10B4400068118E0D9F1D0F900F900F900F900F9011
:10B450000F909501281B390B41E050E04C0F5D1F08
:10B46000840F951FD11003C044E354E202C043E4AB
:10B4700054E25F934F933F932F939F938F930E9438
:10B4800051760F900F900F900F900F900F9087CFE5
:10B490000091D4331091D53301151105C1F0A801E5
:10B4A000495F5F4FA3E056954795AA95E1F762ED96
:10B4B00072E3C7010E941E769091D4338091D533F8
:10B4C0001092D4331092D533092F182FDDC3CF5BE0
:10B4D000DD4F28813981C154D2402115310551F405
:10B4E00088E0E7EBF4E2DE01119601900D928A9577
:10B4F000E1F755CF295F3F4FE3E036952795EA9571
:10B50000E1F7A70160E870E0CE0101960E946811A2
:10B510007C01CF5BDD4F8881C154D240CE5BDD4FD3
:10B520009881C254D240CF5FDD4F9883C150D24042
:10B53000CE5FDD4F8883C250D24081E394E29F9377
:10B540008F93F0E8CF2ED12CC6018E199F099F93BF
:10B550008F9381E090E08C0F9D1F8E0D9F1D9F9318
:10B560008F930E9451768E0D9F1DB601681B790B3B
:10B5700022E030E0AE014F5F5D4FA1E0B0E0AC0FE4
:10B58000BD1F8A0F9B1F0E94681110926031BE017F
:10B590006F5F7F4F85E60E94092A0F900F900F90F2
:10B5A0000F900F900F9070C3CF5BDD4F6881798152
:10B5B000C154D240C701F1DB20913B32222309F470
:10B5C00025C32091393230E04FE252E364E170E06C
:10B5D000CE0101960E946811BE016F5F7F4F85E624
:10B5E0000E94092A10923B32109260310E949F2AD9
:10B5F0000AC380911B32811108C080E890E00E944C
:10B60000EC2A81E080931B327BC0813009F07AC044
:10B6100080913A32823008F075C080911A328F5F83
:10B6200080931A32803109F06DC00E94F72A8C0194
:10B630009350409768F00115B8E01B0708F460C00C
:10B64000E0E1F0E020E030E0A12CB12C60E040C06F
:10B65000A2EAB1E340E050E020E030E080E090E09A
:10B66000E0E0F0E060E07D91703149F4473251054F
:10B6700009F406C361110EC0FA0161E00BC0662334
:10B6800049F0BA016E1B7F0B6817790710F09F0114
:10B69000CB0160E04F5F5F4F4832510521F78430A6
:10B6A000910508F03BC22CC0D601ED906D01F12C44
:10B6B000EE16FF06B0F4611119C04F5F5F4F4837B7
:10B6C000510591F7009709F029C2319709F426C274
:10B6D00072EAC72E71E3D72E40E050E080E090E0A0
:10B6E000E3CF6111EACF5A0161E0E7CFBA016A19ED
:10B6F0007B096817790710F09501CB0160E0DDCF79
:10B7000010921A32CF5BDD4F68817981C154D240EB
:10B71000C70143DB20913B32222309F477C2E09139
:10B72000F033F091F1330284F385E02DE058F10914
:10B7300054E0F695E7955A95E1F7EE55FE4C808179
:10B740008F5F808380911A32803121F40E94F72A22
:10B7500010921A3210923A320E94523380E5F70169
:10B760008083118262E070E0C7010E94E84781E0B7
:10B7700080933A3210923B3260E270E0C701B1D957
:10B780008C0182C2CF5BDD4F68817981C154D24088
:10B79000C70103DB20913B32222309F437C2D0904A
:10B7A000A131DD2009F445C0CF5BDD4F088119814F
:10B7B000C154D2400115110549F41092A1311092E3
:10B7C0003B3210923A320E9452335EC2023A110565
:10B7D00038F0B801C70155DA01E08027082F02C010
:10B7E00001E010E0CF5BDD4F68817981C154D24028
:10B7F000C701FAD9CF5BDD4F88839983C154D2400A
:10B8000000FD05C062E1C701A4DA892B29F0ACEF85
:10B81000AD0DA093A1312AC0F4E0DF9ED001112428
:10B82000AF5ABE4C80E1F70101900D928A95E1F785
:10B830001DC042E050E06EE575E1CE0101960E9428
:10B84000F075E1E6F5E1E49120912C3230912D3252
:10B8500089819A812817390721F480912E32E817BF
:10B8600029F010923A320E945233CDC18091A13119
:10B87000803109F04DC010923B321092A1311092EC
:10B88000603120E130E041E651E367E870E0CE014D
:10B8900001960E94681161E374E2CE0181960E94D4
:10B8A0004A7620E130E041E751E365E670E0CE0101
:10B8B00083960E94681161E374E2CE018D5B9F4F15
:10B8C0000E944A7620E130E041E851E363E470E011
:10B8D000CE018B5B9F4F0E94681161E374E2CE0141
:10B8E0008B599F4F0E944A7620E130E041E951E3B5
:10B8F00061E270E0CE0189599F4F0E9468110E9459
:10B900009F2ABE016F5F7F4F85E60E94092A7BC197
:10B9100090E3D7019C9311968C9362E070E0C7018D
:10B920000E94E8478091A1318C5F8093A13124CFA0
:10B93000BE016F5B7D4FC70137DB882309F4E7C089
:10B9400080911C32811103C069E574E227C0813007
:10B95000A1F0912C80E090E000E010E027E6822E3C
:10B960007E01BFEFEB1ABDEFFB0A3CE6C32E34E2CB
:10B97000D32EA12C42E0B42E40C060911D32E7E6E8
:10B980006E9FB0011124605B7B4E40E450E0CE011D
:10B9900001960E94F075BE016F5F7F4F85E60E94A1
:10B9A000092A55C00130F2E01F0760F5E92DF0E0EB
:10B9B000E35EFD4C6081869EB0011124605B7B4E8E
:10B9C00040E450E0C7010E94F075FF92EF92DF92D1
:10B9D000CF92C501801B910B9F938F9381E090E0E4
:10B9E0008C0F9D1F800F911F9F938F930E94517604
:10B9F000080F191F9394CDBFDEBF20911C32921601
:10BA000088F204C0081B190BF12C06C0013032E08B
:10BA10001307C0F7FF24F394EDEFFFEFEC0FFD1FCA
:10BA2000E00FF11F8EE28083EEEFFFEFEC0FFD1FC2
:10BA3000E00FF11F1082BE016F5F7F4F85E60E940D
:10BA4000092AF11004C084EC93E10E94441F8DEB9D
:10BA500093E10E94441F62E070E08CE292E30E9456
:10BA6000272A87EB93E10E94441F6091393270E0EE
:10BA70008FE292E30E94272A81EB93E10E94441F08
:10BA800061E070E08EE292E30E94272A37C0BE0197
:10BA90006F5B7D4FC70188DA8823C9F180911C3222
:10BAA000813039F580911D32833009F4BCC028F40F
:10BAB000813059F0823099F0E0C08A3031F008F4DA
:10BAC000DCC08D50823058F0D8C08091393284303B
:10BAD00009F4ABC0873009F0D0C017E0A9C080914D
:10BAE0003932843009F4A3C0873009F0C6C019E0A8
:10BAF0009FC063E774E285E60E94092A10926031D4
:10BB000010921C320E949F2A10923B327CC0CF5B65
:10BB1000DD4F08811981C154D240B6C010921B324A
:10BB2000009709F475C096958795285F3F4F820F5F
:10BB3000931F54E0880F991F5A95E1F70E94EC2A51
:10BB4000E091F033F091F13362857385CF01855E2A
:10BB500093438D5F9F4F0E94C87C60E070E085E654
:10BB60000E94092A0115184008F455C0B8E7AB2E09
:10BB7000B12C02EA11E360E8E62EF12C7FE4672E97
:10BB800074E2772EEAE05E2EFE0131966F01F5E554
:10BB90008F2EF4E29F2EFF92EF927F926F921F9270
:10BBA0005F92DF92CF920E945176C6010E945D1F84
:10BBB000D8018C91CDBFDEBF882389F11F928F936E
:10BBC0009F928F921F925F92DF92CF920E94517646
:10BBD000C6010E945D1FCDBFDEBF86E294E10E94D8
:10BBE000441FD8011D928D01B0E1EB0EF11CC8017C
:10BBF000825A91438A159B0570F210923B32109243
:10BC000060310E94593300E010E03EC08C013CC01E
:10BC10000E94072B95CFA8E2AA2EB12CAACF8DE2C5
:10BC20000E942B1FDACF11E003C016E001C018E01C
:10BC300069E974E285E60E94092A812F0E94B51005
:10BC4000E091DE33F091DF331995E091E833F09124
:10BC5000E9338FE292E31995E091C524F091C6246F
:10BC6000309731F04091EC336FE272E383E1199544
:10BC70000E94D4140E942A1A41CF64EA74E23BCF96
:10BC8000662309F40CCDFDCCC801CE5BDD4FCDBFE2
:10BC9000DEBFDF91CF911F910F91FF90EF90DF906A
:10BCA000CF90BF90AF909F908F907F906F905F905C
:10BCB000089581E08093B532E091F033F091F13353
:10BCC00082859385809370209093712008951092BF
:10BCD000B53210923C32089508950895F8CF0F932D
:10BCE0001F93CF93DF93CDB7DEB72A97CDBFDEBFCB
:10BCF00020913C32213009F023C18C018091B53272
:10BD0000833009F446C028F4813061F08230D1F0EC
:10BD100017C1853009F451C008F474C0863009F4A5
:10BD200097C00EC180E1809306068091CD328111CB
:10BD300007C1F8018081863219F0823509F000C10F
:10BD400082E074C08091CD328130B1F462317105EE
:10BD500099F4F801808185FD0FC08181807E61F4B6
:10BD6000828180FD09C062E170E0C8010E944156F5
:10BD7000882311F083E05AC08091CD32811159C0DF
:10BD8000F8018081863209F4DBC0823509F051C0A8
:10BD9000D7C08091CD3281114CC06031710509F05E
:10BDA00048C0F8018081982F907F903909F041C0F8
:10BDB00089708130F1F585E039C08091CD328130D4
:10BDC00061F46D32710549F46DE270E0C8010E94C2
:10BDD0004156882311F084E029C081E08093B53278
:10BDE00080E18093060680917020909171208115EA
:10BDF00028E0920708F493C060E070E088E70E94B2
:10BE0000092A9EC08091CD32811113C0683471051A
:10BE100081F4F8018081982F907F903951F48970D6
:10BE2000813039F48181803721F486E08093B53206
:10BE300087C081E08093B53280E1809306068091CF
:10BE40007020909171208115F8E09F07A8F667C0D7
:10BE50008091CD32813009F053C06B31710509F00A
:10BE60004FC06BE170E0C8010E944156882309F47D
:10BE700047C0F801808182FD7DCF81E08093B5329B
:10BE800080E180930506E0917020F0917120E058E8
:10BE9000F10994E0F695E7959A95E1F7E35CFD4C9E
:10BEA00080818F5F808360E070E085E60E94092AD0
:10BEB000809171208F93809170208F938FE494E212
:10BEC0009F938F931F928AE08F938E010F5F1F4F76
:10BED0001F930F930E945176C8010E945D1FE0914D
:10BEE000F033F091F13362857385CF01855E934322
:10BEF0008D5F9F4F0E94C87CEADECDBFDEBF20C0B1
:10BF000081E08093B53280E18093060680917020B5
:10BF1000909171208115E8E09E0708F06DCFFC013B
:10BF2000E058F10984E0F695E7958A95E1F7E35C3E
:10BF3000FD4C10820E94F72A80937020909371200C
:10BF400080E090E02A96CDBFDEBFDF91CF911F91B8
:10BF50000F910895E0E0F9E080E4848780E387832F
:10BF600010922A06089593B120912806267081E048
:10BF700009F080E0990F892B83B986B197B10196BA
:10BF800086B997B9089709F0C9C016B817B8809153
:10BF9000C0328130E9F020F0823009F44EC0BEC0DA
:10BFA00083B18B3749F481E08093C0321092B8326C
:10BFB0001092B93212B8B2C083B18E3709F079C08D
:10BFC00082E08093C0321092B8321092B932A6C08B
:10BFD00083B18F3DB1F183B18095803439F482B162
:10BFE0008F5F82B980B18695869521C0803149F4F2
:10BFF00082B18F5F82B980B18695869580B9069AA5
:10C0000017C0843049F482B18F5F82B980B18695C0
:10C01000869580B9079A0CC0813051F482B18F5F48
:10C0200082B980B18695869580B980B1806C80B9DF
:10C0300082B1843009F072C062C083B18F3D09F0D3
:10C0400040C080E094E08093BC329093BD328091F8
:10C050006737982F927081FF06C020E031E020936F
:10C06000BC323093BD3280FF0BC020EF33E0209311
:10C07000BA323093BB32992359F08CEF90E004C070
:10C080008091BC329091BD328093BA329093BB3292
:10C090001092030A80E280930C0A8CE08093070AD6
:10C0A0008091BC329091BD3201978093360A909373
:10C0B000370A81E08093C23210920009109207097A
:10C0C0002DC08091B8329091B9329695879523B161
:10C0D0002095203411F484500BC0203111F483508A
:10C0E00007C0243011F4825003C0213029F481505C
:10C0F00080B982B18F5F82B982B1813079F412B890
:10C10000E8B1F9B180B1808388B199B1019688B95D
:10C1100099B98091BE328F5F8093BE328091B832E0
:10C120009091B93201968093B8329093B9320895C4
:10C1300081B1882309F459C181B18C3008F055C10F
:10C14000E1B1F0E0EE0FFF1FE050FC4D0190F081F7
:10C15000E02D19948DE18093BF3214B815B8809109
:10C16000BF3287FF02C08E9A01C08E988EE0809306
:10C1700040088091BF32880F8093BF3284B195B15F
:10C18000019684B995B984B195B187709927892BA7
:10C1900011F483E082C082E01BC18091BF3280FF36
:10C1A00002C08E9801C08E9A84E012C18091BF3285
:10C1B00080FF02C08E9A01C08E988091BF32869512
:10C1C0008093BF3284B195B1019684B995B983E06B
:10C1D00081B984B195B187709927892B09F005C180
:10C1E0008091BE3281508093BE328111B6C088EBFF
:10C1F0008093BF3218C08091BF3287FF02C08E9AF1
:10C2000001C08E988091BF32880F8093BF3284B175
:10C2100095B1019684B995B984B195B18770992784
:10C22000892B09F4D2C085E0D3C08DE18093BF3261
:10C2300014B815B88E9A8EE0809340088091BF3272
:10C2400087FF0BC08FE190E08093660890936708AA
:10C250008091BC329091BD320AC08BE190E0809316
:10C260006608909367088091BA329091BB3201972B
:10C270008093260A9093270A8091BF32880F80937B
:10C28000BF3284B195B1019684B995B984B195B1A5
:10C2900087709927892B19F488E081B95EC087E0FF
:10C2A00097C08091BF3280FF0BC08BE190E08093FC
:10C2B0006608909367088091BA329091BB320AC0A9
:10C2C0008FE190E080936608909367088091BC327C
:10C2D0009091BD3201978093260A9093270A89E0B6
:10C2E00077C08091BF3280FF0BC08FE190E08093D8
:10C2F0006608909367088091BC329091BD320AC065
:10C300008BE190E080936608909367088091BA3241
:10C310009091BB3201978093260A9093270A8091CF
:10C32000BF3286958093BF3284B195B1019684B9AE
:10C3300095B988E081B984B195B187709927892B27
:10C3400009F053C08091BE3281508093BE3281117A
:10C3500004C088EB8093BF323AC0E8B1F9B1CF0195
:10C36000019688B999B980818093BF3208958091F0
:10C37000BF3287FF0BC08FE190E0809366089093F7
:10C3800067088091BC329091BD320AC08BE190E089
:10C3900080936608909367088091BA329091BB327F
:10C3A00001978093260A9093270A8091BF32880FC5
:10C3B0008093BF3284B195B1019684B995B984B1A7
:10C3C00095B187709927892B11F48BE001C08AE021
:10C3D00081B908951092000A1092070A109240083D
:10C3E0001092410881E08093C332089587E697E375
:10C3F00088B999B9E2ECF2E3108211821092C0324E
:10C4000011B810B813B816B817B81092B832109205
:10C41000B93212B81092BE321092BF32A0E2B6E02A
:10C4200081E015968C931597E0E0F9E010A211A237
:10C430008FE790E086A397A381E390E084A795A778
:10C4400082E0808398E8938320E424871782E0E0E9
:10C45000FAE093832FE531E126AB37AB16821782E2
:10C460009EE0908393E01C969C931C971A968C9365
:10C470000895CF93DF93E0E4F6E0128A84E08283AC
:10C48000C0E8D1E082E68E83A0E2B6E081E01696B5
:10C490008C93169711968C93119796E012969C9315
:10C4A000129751968C93519732E052963C93529743
:10C4B0001A961C921A971B961C921B979FE019962E
:10C4C0009C9399E598832AE529839A8390E4918344
:10C4D0009683A0EBB0E012962C911297207F1296D3
:10C4E0002C93129712962C911297226012962C93ED
:10C4F00020E321832683908B8683358383E08183A9
:10C50000E0E0F8E083E1818321E030E026A337A377
:10C5100020A731A7E0E8F8E014868083E0E2F3E0AA
:10C520001382118288E0828391E19083A091F0339D
:10C53000B091F1331A962D913C911B97208F318F3A
:10C54000E0E8F3E09CE3928380839383818383EB31
:10C550009FE58093D0329093D1328AEA9FE5809311
:10C56000D2339093D33388E990E68093CE32909380
:10C57000CF32DF91CF913ACFA0E2B6E01A961C926B
:10C580001A9787E697E388B999B9E2ECF2E310824B
:10C5900011821092C03211B810B813B816B817B87B
:10C5A0001092B8321092B93212B81092BE32109274
:10C5B000BF32E0E0F9E010821382178280E48487C2
:10C5C000E0E0FAE01382178280E28487E0E4F8E09A
:10C5D0001082118281E016968C938E9808950F93A5
:10C5E0001F93CF938091C232882309F469C01092BF
:10C5F000C2324091BE32042F10E00115110509F43A
:10C600005AC0E091C524F091C624309721F067E626
:10C6100077E380E4199563E188E00E94041BC091F0
:10C620006737C170E091E433F091E533B80187E6F4
:10C6300097E319958C010097F1F1E091C524F091F1
:10C64000C624309729F0482F67E677E381E41995EF
:10C6500063E189E00E94041B0093BE3287E697E302
:10C6600088B999B91092600810926108CC2389F0BA
:10C670008BE190E080936608909367088EE090E0ED
:10C6800080936A0890936B0883E28093410886E068
:10C6900010C08FE190E0809366089093670880E176
:10C6A00090E080936A0890936B0883E2809341083E
:10C6B00081E081B905C01092000A1092070A96DE47
:10C6C0008091C332882331F01092C332CF911F91F1
:10C6D0000F918CCECF911F910F9108951092C5327A
:10C6E00008951092C532089508950895EF92FF922B
:10C6F0000F931F93CF93DF93CDB7DEB72897CDBFAE
:10C70000DEBF6430710518F480E090E0C9C08C0190
:10C7100062507109C8D48823B9F3F801F1804091BF
:10C72000EC3350E060E070E0CE0101960E94CD1144
:10C730008091C532882321F0823009F46EC0A5C0F3
:10C74000F1E0FF1217C0F801108211828885828300
:10C750008F8183838E8184838D8185838C81868381
:10C760008B8187838A818087898181879AE0E92EFE
:10C77000F12C8FC0F2E0FF1228C0F801808185FF04
:10C7800020C092818885981380C093818F819813EF
:10C790007CC094818E81981378C095818D81981387
:10C7A00074C096818C81981370C097818B81981387
:10C7B0006CC090858A81981368C09185898198138F
:10C7C00064C082E08093C53260C0FBE2FF125DC0AE
:10C7D000F801808185FFB7CF92818885981355C075
:10C7E00093818F81981351C094818E8198134DC08D
:10C7F00095818D81981349C096818C81981345C08D
:10C8000097818B81981341C090858A8198133DC090
:10C8100091858981981339C096CFF6E2FF1235C011
:10C820004091EC3350E060E070E0CE0101960E9450
:10C83000CD11F801808185FF20C0928188859813F1
:10C8400024C093818F81981320C094818E81981386
:10C850001CC095818D81981318C096818C81981386
:10C8600014C097818B81981310C090858A8198138A
:10C870000CC091858981981308C0F801108210922C
:10C88000C532EE24E394F12C04C0E12CF12CC70155
:10C8900007C0B701C801F7D3F2E0EF0EF11CF7CFE4
:10C8A0002896CDBFDEBFDF91CF911F910F91FF90F2
:10C8B000EF9008954091EC3350E060E070E00C940C
:10C8C000CD114091EC3350E060E070E00C944314E3
:10C8D0001092C63208951092C632089508950895B0
:10C8E0006F927F929F92AF92BF92CF92DF92EF9220
:10C8F000FF920F931F93CF93DF93CDB7DEB72897A7
:10C90000CDBFDEBF6430710518F480E090E0D1C186
:10C910008C0162507109C7D38823B9F3F801F18003
:10C920004091EC3350E060E070E0CE0101960E944F
:10C93000CD118091C632882321F0823009F480C164
:10C94000B5C1F1E0FF1217C0F8011082118288858D
:10C9500082838F8183838E8184838D8185838C8183
:10C9600086838B8187838A818087898181879AE00A
:10C97000E92EF12C93C1F2E0FF1228C0F80180816A
:10C9800085FF20C092818885981390C193818F8103
:10C9900098138CC194818E81981388C195818D8163
:10C9A000981384C196818C81981380C197818B8163
:10C9B00098137CC190858A81981378C1918589816B
:10C9C000981374C182E08093C63270C1FBE2FF12FB
:10C9D00043C0F8019081888595FF1FC0928198130C
:10C9E00065C123819F81291361C124819E812913FF
:10C9F0005DC125819D81291359C126819C812913FF
:10CA000055C127819B81291351C120859A81291302
:10CA10004DC121859981291349C1F80110829FE0F8
:10CA2000918382838F8183838E8184838D818583AB
:10CA30008C8186838B8187838A81808789818187A6
:10CA4000128682EC838783E08487858781E08687EE
:10CA50008FE0E82EF12C22C1F0E2FF1247C0F8016E
:10CA6000808185FF20C02281988529131FC12381E1
:10CA70009F8129131BC124819E81291317C1258100
:10CA80009D81291313C126819C8129130FC1278100
:10CA90009B8129130BC120859A81291307C1218508
:10CAA0009981291303C1F801628570E086FF10C0E7
:10CAB00010821182660F771F660F771F44E050E0E7
:10CAC000C80102960E94CD11B6E0EB2EF12CE6C013
:10CAD0001192CF01660F771F660F771F44E050E079
:10CAE0000E94CD11F5E0EF2EF12CD8C0F3E2FF1239
:10CAF0006FC0F801908195FF20C02281888528139E
:10CB0000D5C023818F812813D1C024818E81281321
:10CB1000CDC025818D812813C9C026818C81281321
:10CB2000C5C027818B812813C1C020858A81281325
:10CB3000BDC0218589812813B9C0F8016285C384ED
:10CB4000D12CFFEFCF1ADF0A98012F5F3F4F70E023
:10CB500096FF2BC058017B01EE0CFF1CEE0CFF1C56
:10CB6000612C712C912C892D90E08C159D0598F4E9
:10CB7000F5011182B701660D771D44E050E0C50153
:10CB800002960E94CD119394F5E0AF0EB11C84E0A3
:10CB9000680E711CE8CF85E08C9D70018D9DF00CB6
:10CBA0001124EFEFEE1AFE0A10C07601EE0CFF1C06
:10CBB000EE0CFF1C660F771F660F771FA701C901D8
:10CBC0000E94CD11FFEFEF1AFF0AF801108266C034
:10CBD000FCE2FF126BC0F801808185FF20C09281CA
:10CBE0008885981363C093818F8198135FC0948167
:10CBF0008E8198135BC095818D81981357C0968163
:10CC00008C81981353C097818B8198134FC0908566
:10CC10008A8198134BC091858981981347C0F80188
:10CC2000E384E3941082902FF8018E2F891B8E15D8
:10CC300010F41192FACFF12CFFEFEF1AFF0A2EC079
:10CC400086E2F81233C0F801808185FF20C092810E
:10CC5000888598132BC093818F81981327C0948166
:10CC60008E81981323C095818D8198131FC0968162
:10CC70008C8198131BC097818B81981317C0908566
:10CC80008A81981313C09185898198130FC0F80188
:10CC900010821092C632EE24E394F12CB701C80141
:10CCA000F2D1F2E0EF0EF11CC70103C0E12CF12C30
:10CCB000FBCF2896CDBFDEBFDF91CF911F910F91A3
:10CCC000FF90EF90DF90CF90BF90AF909F907F90BC
:10CCD0006F9008954091EC3350E060E070E00C9468
:10CCE000CD114091EC3350E060E070E00C944314BF
:10CCF0001092CB328091C7329091C832936080936A
:10CD0000C7329093C832EEE7F9E3108211821282A3
:10CD100013821482158216821782108641E050E039
:10CD200068E270E08DE799E30C94CD111092CB325C
:10CD3000EEE7F9E3108211821282138214821582C7
:10CD4000168217821086089508950895E091EC33B5
:10CD5000F0E03197E80FF91FDC01AE17BF0730F4A0
:10CD60008C9190819D9331978183F7CF0895CF93D4
:10CD7000DF93EC014091EC3350E060E270E00E9400
:10CD8000CD11CE01DF91CF91E1CF6F927F928F9243
:10CD90009F92AF92BF92CF92DF92EF920F931F9329
:10CDA000CF93DF93CDB7DEB76C013B01ADB6BEB616
:10CDB0008091EC332DB73EB7281B31092DBF3EBF04
:10CDC0008DB79EB701964C01D2DF94E069167104CD
:10CDD00008F41AC1B30162507109C60164D18823F5
:10CDE00009F412C121E08091CB32813009F020E0BA
:10CDF000E0907D3984014EE759E3B301C60169D162
:10CE0000882309F401C18091CB328111FDC0E091EA
:10CE10008039F09181398081813031F5F6011082BD
:10CE20001182F4018781F6018283F4018681F60183
:10CE30008383F4018581F6018483F4018481F60102
:10CE40008583F4018381F6018683F4018281F601F2
:10CE50008783F4018181F6018087F4018081F601E6
:10CE600081870AE010E0CAC0823041F49091853990
:10CE7000992309F4BDC08093CB32C6C0803209F03B
:10CE800047C080918439813009F0BEC0E091823979
:10CE9000F09183396081F6016B3018F0808380E176
:10CEA000AAC0808186FF25C081E090E0062E02C0E6
:10CEB000880F991F0A94E2F72091C7323091C83247
:10CEC00028233923232B11F082E00AC02091C93294
:10CED0003091CA3282239323892B21F081E0F6011D
:10CEE000818302C0F6011182C601029606E010E0BD
:10CEF00004C0C601019605E010E0F6011082F4E0DE
:10CF00006F9FB001112444E050E00E94CD1176C023
:10CF10008132C9F580918439853009F075C08091DE
:10CF2000823990918339FC0160816C3028F081E076
:10CF3000F601808383E05FC021E030E0062E02C06E
:10CF4000220F331F0A94E2F74091C7325091C83242
:10CF500042235323452B59F74091C9325091CA328D
:10CF600024233523232B29F081E0F601808382E1FD
:10CF700042C0F4E06F9FB001112444E050E00196FC
:10CF80000E94431430C0823299F5809184398130F7
:10CF9000D9F5E0918239F091833920812C3038F62F
:10CFA00081E090E002C0880F991F2A95E2F7209156
:10CFB000C7323091C83228233923232B49F42091DA
:10CFC000C9323091CA32AC0142235323452B29F098
:10CFD00081E0F601808381E10EC0822B932B809348
:10CFE000C9329093CA32F601108201E010E006C007
:10CFF00081E0F6018083818302E010E0B801C60180
:10D0000042D0C801029602C080E090E0ADBEBEBE34
:10D01000DF91CF911F910F91EF90DF90CF90BF9054
:10D02000AF909F908F907F906F900895CF93DF93F4
:10D03000EC018CDE4091EC3350E060E270E0CE0118
:10D04000DF91CF910C944314A82FFC018FEF9FEF39
:10D050002E2F2A1B30E02617370790F421918227C4
:10D0600028E0AC015695479580FF06C0CA0138E01C
:10D07000832734E8932701C0CA01215091F7E8CFF4
:10D080008095909508950F931F93CF93DF938C0114
:10D09000EB01DADFC00FD11F88839983DF91CF9135
:10D0A0001F910F9108950F931F93CF93DF938C01DE
:10D0B000EB01CADFC00FD11F2881281303C081E014
:10D0C0002981291380E08170DF91CF911F910F9109
:10D0D0000895EF920F931F93CF93DF93DC01FA0132
:10D0E000E801808391830196828393838C9182FDF2
:10D0F00009C085FB882780F987838C918295817090
:10D10000808702C0178210863781CD01332311F04A
:10D110000A9601C002968483958311968C9111978B
:10D12000803A40F012969C9112978981981761F08D
:10D1300080E04AC0813069F48C9184FF0AC0129665
:10D140008C9112978E11F4CF8481958101968483FE
:10D1500095834481558162507109A60FB71FA41BA6
:10D16000B50BA683332349F1DA0118979C918F817F
:10D170009813DECF11969C918E819813D9CF11967A
:10D180009C918D819813D4CF11969C918C8198138A
:10D19000CFCF11969C918B819813CACF11969C91F9
:10D1A0008A819813C5CF11969C9189819813C0CF1D
:10D1B00011969C9188819813BBCF8085882319F0A4
:10D1C000211102C0B5CF81E0DF91CF911F910F9166
:10D1D000EF900895EF92FF921F93CF93DF93CDB717
:10D1E000DEB72897CDBFDEBFF901878189838681AD
:10D1F0008A8385818B8384818C8383818D838281E3
:10D200008E8381818F8380818887DA011496ED91E6
:10D21000FC9115972191822F869586958695AE0172
:10D220004F5F5F4F7A01AF0190E0B701981751F05F
:10D23000D7011D917D01DA013D91AD01131318C095
:10D240009F5FF4CF892F90E0E80FF91FDB01A80F53
:10D25000B91F30818C913827277081E090E001C0A0
:10D26000880F2A95EAF78150932F982381E009F0DF
:10D2700080E02896CDBFDEBFDF91CF911F91FF9058
:10D28000EF9008951092CC32EEE7F9E3108211820C
:10D2900012821382148215821682178210861092CF
:10D2A000873941E050E068ED70E08DE799E30C9438
:10D2B000CD111092CC32EEE7F9E310821182128286
:10D2C0001382148215821682178210861092873973
:10D2D000089508950895FF920F931F93CF93DF93BE
:10D2E0001F92CDB7DEB7E0918239F0918339F0809B
:10D2F00019820F2D10E000521F4F41E050E0B8019D
:10D30000CE0101960E94CD1180918439813071F453
:10D3100094E39F1558F09981911108C0898341E0E9
:10D3200050E0B801CE0101960E94431480E090E0E5
:10D330000F90DF91CF911F910F91FF900895CF92A1
:10D34000DF92EF92FF920F931F93CF93DF931F9281
:10D35000CDB7DEB7C0908239D0908339F601008115
:10D36000198220918439253019F080E090E01FC0A7
:10D370000533D8F77C0110E0B80160527F4F41E0DF
:10D3800050E0CE0101960E94CD118981837069F72A
:10D39000B801660F771F660F771F44E050E0C601A3
:10D3A00001960E944314F701108281E090E00F90F3
:10D3B000DF91CF911F910F91FF90EF90DF90CF9071
:10D3C0000895CF92DF92EF92FF920F931F93CF9326
:10D3D000DF931F92CDB7DEB7E0918239F0918339A8
:10D3E00060811982F090843921E0F21244C06433E4
:10D3F00058F0209185392223F1F1FC01F0822FE0D1
:10D40000218382E090E039C08C01FC018081C62E2E
:10D41000D12C86FF1BC041E050E0B60160527F4F27
:10D42000CE0101960E94CD11898181FF04C082E066
:10D43000F801818305C0F80180FF06C0F18282E017
:10D44000EE24E394F12C05C01182F9CF81E0E12CA8
:10D45000F12CB601660F771F660F771F44E050E08E
:10D460009801280F311DC9010E94CD11F8011082C9
:10D47000C701059602C080E090E00F90DF91CF9148
:10D480001F910F91FF90EF90DF90CF9008953F9202
:10D490004F925F926F927F928F929F92AF92BF92C4
:10D4A000CF92DF92EF92FF920F931F93CF93DF9370
:10D4B000CDB7DEB78C014DB65EB68091843982302F
:10D4C00009F0A3C0E0918239F091833990819433BF
:10D4D00070F080918539882309F497C081E0D801E4
:10D4E0008C938FE011968C9382E090E090C08180C5
:10D4F00033243394380CC92ED12C9601230D311DC1
:10D50000243331051CF084E3382E391AF801808168
:10D51000832C912C86FD0FC0880C991C880C991CBB
:10D52000B601660F771F660F771FA401C801019629
:10D530000E94CD1165C06DB67EB6A401440F551F83
:10D54000440F551F8DB79EB7841B950B8DBF9EBF93
:10D55000ADB7BEB711967D01EDB7FEB7E819F90971
:10D56000EDBFFEBF8DB79EB701965C01B601660F99
:10D57000771F660F771FCD010E94CD11B601605253
:10D580007F4FA401C5010E94CD11F70190E081E019
:10D59000391681F1D5014D915D019801280F311D9A
:10D5A000D9014C9321E0280FA801420F511D9A0187
:10D5B0004081D9014C9322E0280FA801420F511D50
:10D5C0009A014181D9014C9323E0280FA801420F11
:10D5D000511D9A014281D9014C9324E0280FA801E2
:10D5E000420F511D9A018B5F4381D9014C939F5F7C
:10D5F0003496CECFB5E03B9E400111246DBE7EBE79
:10D60000F8011082C401019602C080E090E04DBE96
:10D610005EBEDF91CF911F910F91FF90EF90DF9051
:10D62000CF90BF90AF909F908F907F906F905F90C2
:10D630004F903F900895CF93DF931F921F92CDB7E5
:10D64000DEB7E0918239F091833980818A83198233
:10D65000809184398130B1F441E050E06CED70E0AC
:10D66000CE0101960E94CD11898180FD0BC041E061
:10D6700050E068ED70E0CE0102960E9443148A816A
:10D6800080937D3980E090E00F900F90DF91CF91F3
:10D690000895CF93DF931F92CDB7DEB719828091A3
:10D6A0008439811115C041E050E06CED70E0CE018D
:10D6B00001960E94CD11898180FD0AC08160898315
:10D6C00041E050E06CED70E0CE0101960E94431401
:10D6D00080E090E00F90DF91CF910895CF93DF939A
:10D6E0001F921F92CDB7DEB7E0918239F091833956
:10D6F00080818A83198280918439813099F441E054
:10D7000050E06CED70E0CE0101960E94CD11898150
:10D7100081FD08C041E050E069ED70E0CE01029665
:10D720000E94431480E090E00F900F90DF91CF9122
:10D730000895CF93DF931F92CDB7DEB71982809102
:10D740008439811115C041E050E06CED70E0CE01EC
:10D7500001960E94CD11898181FD0AC08260898372
:10D7600041E050E06CED70E0CE0101960E94431460
:10D7700080E090E00F90DF91CF9108950F931F9379
:10D78000CF93DF9320918439223001F5E0918239E3
:10D79000F091833920812533C8F4C181CF5F622F96
:10D7A00070E0AB014C0F511D4433510514F0C4E33C
:10D7B000C21B8C01D0E060527F4FAE0101960E94E7
:10D7C000CD11F8011082CE01019602C080E090E0F8
:10D7D000DF91CF911F910F910895FC01DA019281A1
:10D7E00017968C911797981328C0938116968C9151
:10D7F0001697981322C0948115968C9115979813BB
:10D800001CC0958114968C911497981316C096811C
:10D8100013968C911397981310C0978112968C9140
:10D82000129798130AC0908511968C9111979813AE
:10D8300004C081E021859C91291380E0908195FFAF
:10D8400012C094FD10C0811103C01092CC320BC0E5
:10D850008091CC328130C9F381E08093CC32108248
:10D8600081E090E0089580E090E00895EEE7F9E32C
:10D8700010821182128213821482158216821782FC
:10D8800010861092CC32FC01108281E090E0089565
:10D89000FF920F931F93CF93DF9300D01F92CDB7CA
:10D8A000DEB719821A821B821C82209184392430AF
:10D8B00049F520918539222329F1209186392223A7
:10D8C00009F1F090CC3221E0F2121CC08C0144E04E
:10D8D00050E064E171E0CE0101960E94CD11F0921A
:10D8E000873944E050E064E171E0809182399091A1
:10D8F00083390E944314F0928739F801108281E045
:10D9000090E002C080E090E02496CDBFDEBFDF91C2
:10D91000CF911F910F91FF900895FC018091843960
:10D92000813059F41082118212821382148215827E
:10D930001682178288E090E0089580E090E00895D4
:10D94000209184392B3049F4FC01119263E0CF011E
:10D950000E944E1184E090E0089580E090E00895E8
:10D960004091EC3350E060ED70E00C94CD11CF921B
:10D97000DF92EF92FF920F931F93CF93DF93CDB778
:10D98000DEB78C01CDB6DEB68091843981114AC0F4
:10D990008FE0F80181838091EC332DB73EB7281BCF
:10D9A00031092DBF3EBF8DB79EB701967C01D8DFF0
:10D9B000F7018781F8018283F7018681F80183836B
:10D9C000F7018581F8018483F7018481F80185835B
:10D9D000F7018381F8018683F7018281F80187834B
:10D9E000F7018181F8018087F7018081F801818743
:10D9F00041E050E069ED70E0C8010A960E94CD1147
:10DA000041E050E068ED70E0C8010B960E94CD1136
:10DA100083E3F801848783E0858782E0868710822C
:10DA20008FE001C080E0CDBEDEBEDF91CF911F91BF
:10DA30000F91FF90EF90DF90CF9008956F927F92BB
:10DA40008F929F92AF92BF92CF92DF92EF920F93FD
:10DA50001F93CF93DF93CDB7DEB76C015B016DB63B
:10DA60007EB68091EC332DB73EB7281B31092DBF10
:10DA70003EBF8DB79EB701964C0172DF94E0A916A8
:10DA8000B10418F480E090E0E6C0B501625071097D
:10DA9000C60109DB8823B1F3F6018181853231F4B7
:10DAA000A401B501C60199DE8C0112C021E080916C
:10DAB000CC32813009F020E0E0907D3984014EE7DE
:10DAC00059E3B501C60105DB8823E1F200E010E06F
:10DAD0008091CC32823008F0ACC0E0918039F09176
:10DAE000813980818130C9F580918439882351F250
:10DAF00094014EE759E3B501C6016CDB882309F4B4
:10DB0000A1C0F6011192CF0141E050E069ED70E053
:10DB10000E94CD11F4018781F6018283F401868190
:10DB2000F6018383F4018581F6018483F401848105
:10DB3000F6018583F4018381F6018683F4018281F5
:10DB4000F6018783F4018181F6018087F4018081E9
:10DB5000F6018187065F1F4F75C0823041F49091B6
:10DB60008539992309F45AC08093CC326BC0803236
:10DB700021F4B501C60125DC05C0813229F4B501C7
:10DB8000C601DDDB8C015EC0823221F4B501C60125
:10DB9000A2DBF8CF833221F4B501C60178DCF2CFE5
:10DBA000873221F4B501C60146DDECCF883221F47D
:10DBB000B501C6016EDDE6CF893221F4B501C6019B
:10DBC0008DDDE0CF8A3221F4B501C601B2DDDACFB6
:10DBD0008B3231F4B501C601CADE082F10E032C025
:10DBE0008C3221F4B501C601C9DDCCCF863221F4D7
:10DBF000B501C6013BDEC6CF843E21F4B501C601A6
:10DC000047DEC0CF803E21F4B501C60186DEBACF23
:10DC1000813E21F4B501C60193DEB4CF80918539F0
:10DC2000882381F081E0F6018083818302E010E0A7
:10DC30000DC0823039F4E0918039F09181398081D2
:10DC40008632B1F20115110509F41CCFB801C601E5
:10DC50001ADAC80102966DBE7EBEDF91CF911F9188
:10DC60000F91EF90DF90CF90BF90AF909F908F90EB
:10DC70007F906F9008954091EC3350E060ED70E03C
:10DC80000C9443140F931F93CF93DF93CDB7DEB75C
:10DC9000EA97CDBFDEBF0DE819E395D2F801819375
:10DCA0008F01F9E305391F07C1F70E94E01F06D372
:10DCB000882309F4FAC080918D3990918E3995307E
:10DCC00009F46FC030F4913069F168F0933051F18C
:10DCD000ECC0983009F4C2C0993009F4C8C096303D
:10DCE00009F0E3C072C0803891F0823809F0DDC0DD
:10DCF000809191398F7087D2E0919739F09198395E
:10DD0000118112FB112710F980E07DD206C010911D
:10DD1000893980918A3981111260EAD2812F63D2C8
:10DD200080E0A1C0282F2D7F09F0BFC0882319F003
:10DD3000823061F0BAC080918F39813009F0B5C06E
:10DD4000933009F080E080938A3927C080918F3921
:10DD5000811123C0E09191391E2F1F7009F4A5C0D5
:10DD6000812F51D280918E39833011F4EDD215C0BC
:10DD7000E0919739F091983981818B7F818324E8F4
:10DD8000129FF0011124E552F64C1082E091973970
:10DD9000F091983980818E7F808380E034D2A8D240
:10DDA00064C0811182C010918F391F77A1D28FD3A7
:10DDB0005FD28823E9F31093C304111102C082E0FB
:10DDC00001C083E080938C3970C08058823008F0A5
:10DDD0006CC080918F39909190398C3DE3E09E0723
:10DDE00061F583E08A838AE389834FB7F894DE0183
:10DDF000139620E038E052E05093CA01E32FF0E0A0
:10DE0000E4911092CA0120FF03C0E295EF703F5FDA
:10DE1000EF708E2F90E0EA3010F0C79601C0C096E8
:10DE20008D939D932F5F2C3139F74FBF61D26AE3F9
:10DE300070E0CE010196A5D00FC0AE014F5F5F4FDD
:10DE4000609191390E94B70F8C01892B71F150D2EA
:10DE5000B80189819A8111D1A7D127C0803829F5CD
:10DE600047D280918839BFD186D131D31EC081116C
:10DE70001CC080918F399091903999270297ACF40A
:10DE800037D280918F398093883921D38091883916
:10DE9000811106C08091C304811102C081E001C0DC
:10DEA00084E080938C390E94DC1F08D2882311F013
:10DEB0001FD24AD2EA96CDBFDEBFDF91CF911F912C
:10DEC0000F9108950895CF9380918C39882351F054
:10DED000C091993980E097D1F1D18111D3DE8C2F97
:10DEE000CF9191C1CF910895CF92DF92EF92FF929F
:10DEF0000F931F93CF93DF93EC018B017A01FDD237
:10DF0000811136C0E114F10439F0F701808191816B
:10DF1000081B190BC80FD91FC12CD12C01151105D5
:10DF200031F18091953990919639FC01EF5BFF4F6B
:10DF3000208131978081281790F01DD1C4DFE11432
:10DF4000F10449F0F70180819181C80ED91EC08289
:10DF5000D18285E00DC0D1D2882301F309C0899117
:10DF600042D101501109FFEFCF1ADF0AD7CF80E06D
:10DF7000DF91CF911F910F91FF90EF90DF90CF90A5
:10DF80000895DF92EF92FF920F931F93CF93DF9349
:10DF9000D82FC92F8B0180919939806834D1809115
:10DFA0009339909194398017910728F00115110544
:10DFB00019F4E1D001C08C01ED2EFC2ED12C0115FD
:10DFC000110509F440C080918C39811102C082E0B2
:10DFD0004CC0853011F483E048C070D1882311F023
:10DFE00081E043C051D181113CC042D1882339F333
:10DFF000209199398091953990919639FC0127FFAC
:10E0000005C0EF5BFF4FC081D0E013C0E05CFF4F65
:10E01000C08131968081D0E0C81BD1090AC0C830C8
:10E02000D10550F4F70181917F01DDD00150110934
:10E0300021960115110599F7DD24D394289709F04D
:10E04000D12C99D0BCCFD110BECF0BC080918C39D0
:10E05000882309F4BCCF853009F4BDCF2FD18111BD
:10E06000BFCF12D1882391F380E0DF91CF911F9130
:10E070000F91FF90EF90DF900895DF92EF92FF9263
:10E080000F931F93CF93DF93D82FC92F8B018091CC
:10E0900099398068B8D080919339909194398017DC
:10E0A000910728F00115110519F465D001C08C0104
:10E0B000ED2EFC2ED12C0115110509F442C08091E2
:10E0C0008C39811102C082E04EC0853011F483E0AA
:10E0D0004AC0F4D0882311F081E045C0D5D0811129
:10E0E0003EC0C6D0882339F3209199398091953963
:10E0F00090919639FC0127FF05C0EF5BFF4FC0816F
:10E10000D0E015C0E05CFF4FC08131968081D0E047
:10E11000C81BD1090CC0C830D10560F4F701849147
:10E1200062D0FFEFEF1AFF0A015011092196011585
:10E13000110589F7DD24D394289709F0D12C1BD041
:10E14000BACFD110BCCF0BC080918C39882309F491
:10E15000BACF853009F4BBCFB1D08111BDCF94D0F7
:10E16000882391F380E0DF91CF911F910F91FF9071
:10E17000EF90DF900895E0919739F0919839A09150
:10E180009539B0919639AF5BBF4F8C9190E0828307
:10E19000938380818D798083E0919539F0919639D0
:10E1A000EF5BFF4F10820895E0919739F091983915
:10E1B00080818D798083E0919539F0919639EF5B7C
:10E1C000FF4F108208958091953990919639FC0106
:10E1D000EF5BFF4F208131E0320F3083FC01E20F13
:10E1E000F11D808108952091953930919639F9017A
:10E1F000EF5BFF4F908141E0490F4083F901E90F48
:10E20000F11D8083089580939939482F4F7050E015
:10E210006091C6047091C7049A0194E0220F331FE5
:10E220009A95E1F7E4E887FF11C0E49FC001E59FFC
:10E23000900D11248452964C809395399093963981
:10E24000C90108969B01280F391F0DC0E49FC0012A
:10E25000E59F900D11248656964C809395399093A6
:10E260009639260F371F20939739309398390895A0
:10E27000809199398068C7DFE0919739F09198399A
:10E280008081869581700895809199398F77BBDF61
:10E29000A0919739B09198398C9185FF0DC0E0918C
:10E2A0009539F091963912968D919C911397E05C77
:10E2B000FF4F808381E0089580E00895809199392F
:10E2C0008F77A1DFA0919739B09198398C9184FF15
:10E2D0000DC0E0919539F091963912968D919C91EF
:10E2E0001397E05CFF4F808381E0089580E00895FC
:10E2F000809199398F7787DFE0919739F09198393C
:10E3000080818D788083E0919739F0919839808170
:10E3100081608083E0919539F0919639EF5BFF4FF2
:10E3200010828091993980686EDFE0919739F09181
:10E330009839808181608083E0919539F091963998
:10E34000EF5BFF4F10820895E0919739F091983973
:10E35000818184608183E0919739F091983981813E
:10E36000807C803459F48091993980584CDFE09159
:10E370009739F091983981818460818308951F9342
:10E38000CF93DF93C82F162FD42F3DDFE09197391D
:10E39000F09198391182E0919739F09198398C2F4A
:10E3A000881F8827881F880F8083E0919739F09114
:10E3B00098391183E0919739F0919839128213823C
:10E3C000209195393091963924833583CC0FCC0B2D
:10E3D000CD23F901E05CFF4FC0833196108281E0CC
:10E3E000DF91CF911F910895CF92DF92EF92FF922C
:10E3F0000F931F93CF93DF93C62E8C01D12CDC1487
:10E4000009F43FC0F801D081D11104C0D3940B5F4F
:10E410001F4FF5CFF801E180F28093818481823033
:10E4200010F488E001C088E128E030E0C0E02E155B
:10E430003F0520F4CF5F220F331FF9CFC82B8D2F5C
:10E440008F70863010F080E01DC0CF7EF1E4EF16B3
:10E45000F104C8F7992321F0913021F4C06C0AC06F
:10E46000C06403C0C068911105C04E2D6C2F80E8B8
:10E470008D0F85DF4E2D6C2F8D2F81DF8111C6CF43
:10E48000E2CF81E0DF91CF911F910F91FF90EF904C
:10E49000DF90CF90089580E090E0E091C604F09185
:10E4A000C7049C0144E0220F331F4A95E1F7E20FB5
:10E4B000F31F11864091C6045091C704FA01E20F80
:10E4C000F31F118201968630910539F708958091E6
:10E4D0008D3987FF0DC0D8DE811105C080918C3940
:10E4E0008111F9CF09C060CE80918C39882321F049
:10E4F000BFDE8823C9F33FCE08950F931F93CF93B8
:10E50000E091C604F091C704E05AFF4F00811181E9
:10E51000C4E68091993987FF0AC0AADE811105C03F
:10E5200080918C39811105C022C080E025C0ACDE0D
:10E53000F5CF8530F1F0E0919739F09198398181EC
:10E5400082FD19C0E091C604F091C704E05AFF4F64
:10E55000808191810817190711F48C01DACF2FEF10
:10E560002C0FCC2311F0C22FF8CF84E005C082E03D
:10E5700003C083E001C081E0CF911F910F91089506
:10E5800063D069D0E0ECF4E081818E7F818380816B
:10E590008F77808310928B390895CF93DF93E0E4D7
:10E5A000F0E014828481836084834ED054D0C0EC28
:10E5B000D4E088818F7788838881806888831092EF
:10E5C0008C391092883910928A3910928939888151
:10E5D0008064888348E068E480E8D1DE48E068E44D
:10E5E00080E0CDDE88858064888789818160898329
:10E5F000DF91CF910895CF93DF933FB7F894C0ECAC
:10E60000D1E022E02A87EAE1F0E0E491A0ECB4E076
:10E61000DA96EC93DA97EBE1F0E0E491DB96EC9399
:10E62000DB971A8683EB9CE38E7F16968D939C93E3
:10E63000179785E18C9318962C933FBF81E08093C8
:10E640008B39DF91CF91A9CFE0ECF4E08085837026
:10E65000808711860895E0ECF4E08FEF828784874D
:10E6600008951F920F920FB60F92112408B60F92C1
:10E6700018BE09B60F9219BE0BB60F921BBE2F9390
:10E680003F934F935F936F937F938F939F93AF933A
:10E69000BF93EF93FF938091CA0487FF08C08091D6
:10E6A000C80487FF04C080E88093CA040BDC809113
:10E6B000CA0486FF07C080E48093CA0410928C3994
:10E6C0000E94D91F8091CA0485FF14C080E2809304
:10E6D000CA0480918839882311F084E007C08091B2
:10E6E000C304811102C081E001C083E080938C39B2
:10E6F0000E94D61F8091CA0484FF14C080E18093D9
:10E70000CA0482E080938C39109288391092C30435
:10E71000C2DE48E068E480E832DE48E068E480E099
:10E720002EDED0DBFF91EF91BF91AF919F918F9142
:10E730007F916F915F914F913F912F910F900BBE01
:10E740000F9009BE0F9008BE0F900FBE0F901F9044
:10E750001895CF93DF93EC01FC0170968BE0DF01FD
:10E760001D928A95E9F782E08C83898783E08E8702
:10E7700061E0CE01019638DE882361F061E0CE01D0
:10E78000069632DE882331F061E0CE010B96DF91F0
:10E79000CF912ACE80E0DF91CF9108950F931F9300
:10E7A000CF93DF9320918C392430B1F4FC0104899C
:10E7B000158926893789012B022B032B69F08A01E1
:10E7C000EB01818120DD40E050E0B801CE01DF9116
:10E7D000CF911F910F9188CB82E0DF91CF911F9154
:10E7E0000F9108950F931F93CF9320918C3924306C
:10E7F00009F5FC010489158926893789012B022B2B
:10E80000032BC1F0C62F8181FEDC80919539909158
:10E810009639FC01EF5BFF4F2081319780812817EB
:10E8200020F48C2FE0DC80E006C0A5DC66DE8823C7
:10E83000C1F301C082E0CF911F910F910895CF9352
:10E84000DF9320918C39243091F5FC01448955895E
:10E8500066897789452B462B472B49F18181D3DC8B
:10E86000809199392091953930919639F90187FF36
:10E8700005C0EF5BFF4F808190E008C0E05CFF4F78
:10E8800080813196408190E0841B9109892B69F049
:10E89000F901EF5BFF4FD0813197C0816CDCDC1751
:10E8A00020F02BDE811104C066DC80E001C082E034
:10E8B000DF91CF910895CF93DF9320918C3924304D
:10E8C00099F4FC014489558966897789452B462B43
:10E8D000472B51F0EC01818196DCCADC882321F0C2
:10E8E000CE01DF91CF91ABCFDF91CF910895CF9340
:10E8F000DF9320918C39243019F08FEF9FEF46C0C1
:10E90000FC014489558966897789452B462B472B1D
:10E91000A1F3868178DCB8DC882379F3809199397A
:10E920002091953930919639F90187FF05C0EF5B49
:10E93000FF4F808190E008C0E05CFF4F80813196FE
:10E94000208190E0821B9109892B21F03CDCC82FAB
:10E95000D0E002C0CFEFDFEF209199398091953957
:10E9600090919639FC0127FF05C0EF5BFF4F208196
:10E9700030E008C0E05CFF4F20813196808130E0BC
:10E98000281B3109232B09F40FDCCE01DF91CF9135
:10E9900008950895FF920F931F93CF93DF93EC0197
:10E9A0008DDC882309F48EC0888190E02091913914
:10E9B000309192392817390709F084C080918E3937
:10E9C000813259F018F4803249F17CC0823209F466
:10E9D00057C0833209F467C075C080918D39813A80
:10E9E00009F070C085DC44DC8823E9F38C89FD885C
:10E9F0000E891F89F8DB8F2DF6DB802FF4DB812F4A
:10EA0000F2DB888DF0DB898DEEDB8A8DECDBB3DB0E
:10EA1000DF91CF911F910F91FF9059CD80918D394A
:10EA2000813209F04FC064DC2FDC811105C0809178
:10EA30008C398111F9CF46C0C6DBF82EC4DB182F04
:10EA4000C2DB082FC0DB402F50E060E070E0BA016D
:10EA500055274427782B4F29512B4C8B5D8B6E8B80
:10EA60007F8BB1DB888FAFDB898FADDB8A8F9CDB3F
:10EA70002EDDCE01DF91CF911F910F91FF9089CFB5
:10EA800080918D398132F1F433DC21DD80918F3931
:10EA900090919039888B998BCE01DF91CF911F9106
:10EAA0000F91FF9076CF80918D39813259F420DC1F
:10EAB0000EDD60918F39CE01DF91CF911F910F91C3
:10EAC000FF9067CFDF91CF911F910F91FF90089535
:10EAD000AA1BBB1B51E107C0AA1FBB1FA617B70784
:10EAE00010F0A61BB70B881F991F5A95A9F78095A0
:10EAF0009095BC01CD010895B7FF04C003D0821BDF
:10EB0000930B089509D0A59F900DB49F900DA49FDD
:10EB1000800D911D11240895A29FB001B39FC001E3
:10EB2000A39F700D811D1124911DB29F700D811D39
:10EB30001124911D08958F929F92AF92BF92CF9210
:10EB4000DF92EF92FF92CF93DF93EC01688179819E
:10EB50008A819B81611571058105910521F464E22B
:10EB600079ED8BE597E02DE133EF41E050E037D7C9
:10EB700049015A019B01AC01A7EAB1E4C3DF6B0173
:10EB80007C01ACEEB4EFA5019401B8DFDC01CB0150
:10EB90008C0D9D1DAE1DBF1DB7FF03C00197A109C0
:10EBA000B04888839983AA83BB839F77DF91CF91F5
:10EBB000FF90EF90DF90CF90BF90AF909F908F909D
:10EBC0000895B9CF82E790E2B6CFA0E0B0E080939D
:10EBD000722090937320A0937420B09375200895B1
:10EBE000FB01DC0102C005900D9241505040D8F766
:10EBF0000895FB01DC018D91059080190110D9F376
:10EC0000990B0895FB01DC014150504048F00590FC
:10EC10000D920020C9F701C01D9241505040E0F70D
:10EC20000895FB01DC0104C08D910190801921F44D
:10EC300041505040C8F7881B990B0895FB01DC0137
:10EC400002C001900D9241505040D8F708956817C6
:10EC5000790768F4FB01DC01E40FF51FA40FB51F71
:10EC600002C002900E9241505040D8F70895E6CF6E
:10EC7000DC0101C06D9341505040E0F70895FC0164
:10EC80008191861721F08823D9F799270895319724
:10EC9000CF010895FB01DC0101900D920020E1F706
:10ECA00008950F931F93CF93DF93CDB7DEB72E97C1
:10ECB000CDBFDEBF0E891F89888D998D26E02C83FC
:10ECC00009831A8397FF02C080E090E801978D8343
:10ECD0009E83AE01445E5F4F6A8D7B8DCE010196AF
:10ECE00067D04D815E8157FD0AC02F81388542175C
:10ECF00053070CF49A01F801E20FF31F10822E96CD
:10ED0000CDBFDEBFDF91CF911F910F9108950F937B
:10ED10001F93CF93DF93CDB7DEB72E97CDBFDEBF66
:10ED20000E891F89888D998D2EE02C8309831A8383
:10ED300097FF02C080E090E801978D839E83AE012B
:10ED4000445E5F4F6A8D7B8DCE01019631D04D813F
:10ED50005E8157FD0AC02F813885421753070CF496
:10ED60009A01F801E20FF31F10822E96CDBFDEBF8D
:10ED7000DF91CF911F910F910895CF93DF93CDB77E
:10ED8000DEB72E97CDBFDEBF8DE08C838C899D8949
:10ED900089839A83AE01485E5F4F6E897F89CE0179
:10EDA0000196A9D32E96CDBFDEBFDF91CF910895F6
:10EDB0002F923F924F925F926F927F928F929F928B
:10EDC000AF92BF92CF92DF92EF92FF920F931F9379
:10EDD000CF93DF93CDB7DEB72B97CDBFDEBF6C01EE
:10EDE0007B018A01FC0116821782838181FFBFC1EA
:10EDF000CE0101963C01F6019381F70193FD8591C7
:10EE000093FF81917F01882309F4ADC1853239F4E4
:10EE100093FD859193FF81917F01853221F4B601A5
:10EE200090E0E7D4E8CF912C212C312CFFE1F315B1
:10EE3000D8F08B3279F038F4803279F08332A1F453
:10EE4000232D20611DC08D3261F0803369F4232DA4
:10EE5000216016C0832D8260382EE32DE4603E2EA3
:10EE60002AC0F32DF8601DC037FC2DC020ED280FFF
:10EE70002A3040F08E32B9F436FC75C1232D20645F
:10EE8000322E19C036FE06C08AE0989E200D11244D
:10EE9000922E11C0EAE02E9E200D1124222EF32D79
:10EEA000F0623F2E08C08C3621F4832D8068382E06
:10EEB00002C0883641F4F70193FD859193FF81915B
:10EEC0007F018111B3CF982F9F7D9554933028F403
:10EED0000C5F1F4F9FE399830DC0833631F083375A
:10EEE00071F0833509F055C020C0F8018081898315
:10EEF0000E5F1F4F88248394912C530112C0280168
:10EF0000F2E04F0E511CF801A080B18036FE03C024
:10EF1000692D70E002C06FEF7FEFC50121D44C0175
:10EF20008201F32DFF773F2E15C0280122E0420E0B
:10EF3000511CF801A080B18036FE03C0692D70E03D
:10EF400002C06FEF7FEFC50100D44C01F32DF068D4
:10EF50003F2E820133FC19C0822D90E0881699065D
:10EF6000A0F4B60180E290E044D42A94F5CFF501F4
:10EF700037FC859137FE81915F01B60190E039D46D
:10EF800021102A9421E0821A91088114910479F7C2
:10EF9000E1C0843611F0893639F5F80137FE07C033
:10EFA00060817181828193810C5F1F4F08C06081F5
:10EFB0007181072E000C880B990B0E5F1F4FF32DEC
:10EFC000FF763F2E97FF09C09095809570956195CB
:10EFD0007F4F8F4F9F4FF0683F2E2AE030E0A30114
:10EFE0005DD4882E861844C0853731F4232D2F7EBA
:10EFF000B22E2AE030E025C0932D997FB92E8F36AE
:10F00000C1F018F4883579F0AEC0803719F0883730
:10F0100021F0A9C0E92FE061BE2EB4FE0DC0FB2D8A
:10F02000F460BF2E09C034FE0AC0292F2660B22E1C
:10F0300006C028E030E005C020E130E002C020E159
:10F0400032E0F801B7FE07C060817181828193814F
:10F050000C5F1F4F06C06081718180E090E00E5F01
:10F060001F4FA3011BD4882E8618FB2DFF773F2E40
:10F0700036FE0DC0232D2E7FA22E891458F434FEA7
:10F080000BC032FC09C0832D8E7EA82E05C0B82C83
:10F09000A32C03C0B82C01C0B92CA4FE0FC0FE01E4
:10F0A000E80DF11D8081803321F49A2D997EA92EDF
:10F0B00009C0A2FE06C0B394B39404C08A2D86781A
:10F0C00009F0B394A3FC10C0A0FE06C0B21480F4F3
:10F0D000280C922C9B180DC0B21458F4B60180E293
:10F0E00090E087D3B394F8CFB21418F42B1802C071
:10F0F000982C212CA4FE0FC0B60180E390E079D3B8
:10F10000A2FE16C0A1FC03C088E790E002C088E51B
:10F1100090E0B6010CC08A2D867851F0A1FE02C0A5
:10F120008BE201C080E2A7FC8DE2B60190E061D3E2
:10F13000891430F4B60180E390E05BD39A94F8CF61
:10F140008A94F301E80DF11D8081B60190E051D35E
:10F150008110F6CF222009F44ECEB60180E290E075
:10F1600048D32A94F7CFF6018681978102C08FEFAA
:10F170009FEF2B96CDBFDEBFDF91CF911F910F91F7
:10F18000FF90EF90DF90CF90BF90AF909F908F90C7
:10F190007F906F905F904F903F902F90089520FD4B
:10F1A00009C0FC0123FD05C022FF02C073836283F6
:10F1B00051834083089544FD17C046FD17C0AB013D
:10F1C000BC01DA01FB01AA0FBB1FEE1FFF1F109449
:10F1D000D1F74A0F5B1F6E1F7F1FCB01BA01660F6D
:10F1E000771F881F991F09C033E001C034E0660F04
:10F1F000771F881F991F3150D1F7620F711D811D34
:10F20000911D08950F931F93CF93DF938C01C80135
:10F21000B2D2EC0197FD06C085D2892BC1F7B801A7
:10F22000CE0123D3CE01DF91CF911F910F9108958D
:10F230008F929F92AF92BF92EF92FF920F931F9384
:10F24000CF93DF938C01D62F7A01B22E94D29C01FA
:10F2500033272B32310531F02D32310559F48B2D06
:10F260008068B82ED15011F480E061C0C80183D20B
:10F2700097FDFACFCB2DCD7F2B2D2073F9F4803362
:10F28000E9F4AA24AA94AD0E09F43EC0C80173D2D1
:10F2900097FD3AC09C012F7D33272835310541F475
:10F2A000C264D25089F1C80166D297FF07C02CC052
:10F2B000B6FE02C0C26001C0C261DA2D812C912C61
:10F2C000540120ED280F283078F0C4FF03C0B801A6
:10F2D000CCD217C02A3040F0C6FFF9CF2F7D3FEEC9
:10F2E000320F3630A0F727504C2FC501B40163DF31
:10F2F0004B015C01C260D15051F0C8013CD297FF74
:10F30000E0CFC1FD04C0B0CF812C912C5401C7FFC8
:10F3100008C0B094A09490948094811C911CA11C6E
:10F32000B11C2C2FB501A401C70139DF81E0DF91A9
:10F33000CF911F910F91FF90EF90BF90AF909F9052
:10F340008F9008955F926F927F928F929F92AF926B
:10F35000BF92CF92DF92EF92FF920F931F93CF93C2
:10F36000DF93CDB7DEB7A097CDBFDEBF5C01962E91
:10F370007A01F9018E010F5F1F4F680180E2D80109
:10F380001D928A95E9F7D50113968C9080E090E064
:10F39000612C712C30E061E070E083FC259183FEEC
:10F3A00021918F01522E211103C080E090E090C086
:10F3B0002E3511F4009751F1432F50E048175907AB
:10F3C0003CF42D3559F12D3219F4772009F103C0A1
:10F3D000772009F468C0452D469546954695D60197
:10F3E000A40FB11D452D47708B0102C0000F111FE6
:10F3F0004A95E2F7A8015C91452B4C93651459F0AE
:10F40000561410F45394E7CF5A94E5CF31E004C07A
:10F410007724739401C0712C0196BFCF772019F027
:10F420008E8180628E83311103C08824839417C03B
:10F43000F6019E012F5D3F4F8081809581932E17AD
:10F440003F07D1F7F2CFE114F10429F0D7018C93F3
:10F45000F70131967F019A94812C9920E9F0C5013A
:10F460008AD197FD17C0FC01FF2723E0F595E795AA
:10F470002A95E1F7EC0DFD1D208130E0AC014770CD
:10F48000552702C0359527954A95E2F720FDDBCF39
:10F49000B501EBD1811089CFE114F10411F0D7014E
:10F4A0001C92C80115C0422F469546954695D60137
:10F4B000A40FB11D422F47708B0102C0000F111F16
:10F4C0004A95E2F7A8015C91452B4C93622EA4CF9C
:10F4D000A096CDBFDEBFDF91CF911F910F91FF901E
:10F4E000EF90DF90CF90BF90AF909F908F907F90E4
:10F4F0006F905F9008955F926F927F928F929F922C
:10F50000AF92BF92CF92DF92EF92FF920F931F9331
:10F51000CF93DF936C01EB015A01FC011682178235
:10F52000512CF601E380FE01E3FC8591E3FE81911D
:10F53000182FEF01882309F4E0C090E0F3D0892B65
:10F5400019F0C6015FDEEDCF153241F4FE01E3FC98
:10F550001591E3FE1191EF01153271F4C6010BD143
:10F5600097FDC9C0412F50E09C0133272417350770
:10F57000C1F2B6017AD1C1C01A3239F4E3FC159157
:10F58000E3FE1191EF0101E001C000E0F12C20ED5C
:10F59000210F2A3078F402606F2D70E080E090E057
:10F5A00040E209DEF62EFE01E3FC1591E3FE119127
:10F5B000EF01EDCF01FF03C0F11003C09EC0FF2497
:10F5C000FA94183619F01C3651F010C0FE01E3FC15
:10F5D0001591E3FE1191EF01183641F408600460C3
:10F5E000FE01E3FC1591E3FE1191EF01112309F4F3
:10F5F00084C0612F70E08CEF91E09CD0892B09F4DE
:10F600007CC000FD07C0F50180809180C501029695
:10F610005C0102C0812C912C1E3649F4F601468112
:10F62000578160E070E0202FC401B9DD7ACF133636
:10F63000A1F401FD02C0FF24F394C6019CD097FD04
:10F640005AC08114910429F0F4018083C401019609
:10F650004C01FA94F110F1CF4AC01B3551F49E01D0
:10F66000A4016F2DC6016EDEEC01892B09F03FC0AD
:10F6700039C0C601C7DD97FD3EC01F3649F128F4E9
:10F68000143621F1193639F125C0133771F01537C9
:10F69000E9F020C08114910429F0F4016082C401D2
:10F6A00001964C01FA94FF2059F0C60164D03C0148
:10F6B00097FD06C037D0892B69F3B601C301D5D0B9
:10F6C00081149104A1F0F401108211C0006203C002
:10F6D000006101C00064202FA4016F2DC601A8DDC8
:10F6E000811105C0F6018381807329F406C000FDF5
:10F6F00018CF539416CF552019F0852D90E002C0F5
:10F700008FEF9FEFDF91CF911F910F91FF90EF90BF
:10F71000DF90CF90BF90AF909F908F907F906F9031
:10F720005F900895911118C1803219F08950855069
:10F73000D0F70895FC010590061621F00020D9F7B6
:10F74000C00108953197CF010895FC0105906150E3
:10F7500070400110D8F7809590958E0F9F1F0895E7
:10F76000FC016150704001900110D8F78095909590
:10F770008E0F9F1F0895CF93DF93EC012B8120FF05
:10F7800033C026FF0AC02F7B2B838E819F81019679
:10F790008E839F838A8190E029C022FF0FC0E88179
:10F7A000F9818081082E000C990B009719F42062D2
:10F7B0002B831AC03196E883F9830EC0EA85FB8556
:10F7C000199597FF09C02B81019611F080E201C0C5
:10F7D00080E1822B8B8308C02E813F812F5F3F4FBA
:10F7E0002E833F83992702C08FEF9FEFDF91CF9148
:10F7F00008950F931F93CF93DF93FB01238121FD86
:10F8000003C08FEF9FEF2CC022FF16C046815781A7
:10F81000248135814217530744F4A081B1819D01B1
:10F820002F5F3F4F208331838C93268137812F5F59
:10F830003F4F2683378314C08B01EC01FB0100840A
:10F84000F185E02D1995892BE1F6D80116968D9159
:10F850009C911797019616968D939C931797CE01BE
:10F86000DF91CF911F910F910895FB01238120FF1C
:10F8700012C026FD10C08F3F3FEF930761F08283D7
:10F880002F7D2064238326813781215031092683EF
:10F890003783992708958FEF9FEF0895FA01AA27DC
:10F8A000283051F1203181F1E8946F936E7F6E5FC3
:10F8B0007F4F8F4F9F4FAF4FB1E03ED0B4E03CD071
:10F8C000670F781F891F9A1FA11D680F791F8A1F54
:10F8D000911DA11D6A0F711D811D911DA11D20D0BB
:10F8E00009F468943F912AE0269F11243019305D75
:10F8F0003193DEF6CF010895462F4770405D419366
:10F90000B3E00FD0C9F7F6CF462F4F70405D4A33B2
:10F9100018F0495D31FD4052419302D0A9F7EACF7A
:10F92000B4E0A6959795879577956795BA95C9F7A9
:10F9300000976105710508959B01AC010A2E06949C
:10F940005795479537952795BA95C9F7620F731F55
:10F95000841F951FA01D089599278827089503D017
:10F96000808199270895E0ECF1E0378537FDFDCFE0
:10F97000348538603487FC01E050F04F0895262F1D
:10F98000F2DF0080021611F008D001970197089568
:10F990000196272FF5DFF3CF262FE0ECF1E0378536
:10F9A00037FDFDCF3485377F3487378531FF09C078
:10F9B00036E3328738ED34BF31E03387378537FDA2
:10F9C000FDCF33E33287808391831282248325E342
:10F9D000228728ED31E024BF338701960895052E54
:10F9E00097FB16F400940FD057FD05D014D007FCF8
:10F9F00002D046F408C050954095309521953F4F70
:10FA00004F4F5F4F089590958095709561957F4F0A
:10FA10008F4F9F4F0895A1E21A2EAA1BBB1BFD0119
:10FA20000DC0AA1FBB1FEE1FFF1FA217B307E407DD
:10FA3000F50720F0A21BB30BE40BF50B661F771F35
:10FA4000881F991F1A9469F7609570958095909515
:0EFA50009B01AC01BD01CF010895F894FFCFDA
:10FA5E000240FF0100020202000102020200000148
:10FA6E000202000000020200000201020000020079
:10FA7E00020000020201000002020000000001026A
:10FA8E000100C20100C876312E3020323032302DC6
:10FA9E0030362D32322031313A30383A343300019B
:10FAAE00090083100000010410000001820800000C
:10FABE0001000000000000000000000004000270C1
:10FACE00800001000000000000004F2C562C562C28
:10FADE00622C6E2C782C952CA32CCC2CCF2CD32CCA
:10FAEE003E000426140004043E00042E040C0404FC
:10FAFE0000080008000000000000000800080808C8
:10FB0E000808080008000800000008080008080897
:10FB1E0000800080000000000000008000808080D7
:10FB2E0080808000800080000000808000808080C7
:10FB3E0000010001000000000000000100010101B1
:10FB4E00010101000100010000000101000101019D
:10FB5E000000000000000000000000000000000097
:10FB6E000101010101010101010101010101010177
:10FB7E000101010101010101010101010101010167
:10FB8E000101010101010101010101010101010157
:10FB9E000000000000000000000000000000000057
:10FBAE000000000000000000000000000000000047
:10FBBE000000000000000000000000000000000037
:10FBCE000101010101010101010101010101010117
:10FBDE000000000000000000000000000000000017
:10FBEE000000000000000000000000000000000007
:10FBFE0001010101010101010101010101010101E7
:10FC0E0000000000000000000000000000000000E6
:10FC1E0001010101010101010101010101010101C6
:10FC2E0001010101010101010101010101010101B6
:10FC3E0000000000000000000000000000000000B6
:10FC4E000101010101010101010101010101010196
:10FC5E000000000202000002000202020200000286
:10FC6E000000000202000002000202020200000276
:10FC7E000000000202000002000202020200000266
:10FC8E000404040606040406040606060604040616
:10FC9E000404040606040406040606060604040606
:10FCAE000000000202000002000202020200000236
:10FCBE000000000202000002000202020200000226
:10FCCE0004040406060404060406060606040406D6
:10FCDE000000000202000002000202020200000206
:10FCEE0004040406060404060406060606040406B6
:10FCFE0004040406060404060406060606040406A6
:10FD0E000404040606040406040606060604040695
:10FD1E000404040606040406040606060604040685
:10FD2E0000000002020000020002020202000002B5
:10FD3E0000000002020000020002020202000002A5
:10FD4E000404040606040406040606060604040655
:10FD5E000008080800000008000008000808000855
:10FD6E000008080800000008000008000808000845
:10FD7E000008080800000008000008000808000835
:10FD8E001018181810101018101018101818101825
:10FD9E001018181810101018101018101818101815
:10FDAE000008080800000008000008000808000805
:10FDBE0000080808000000080000080008080008F5
:10FDCE0010181818101010181010181018181018E5
:10FDDE0000080808000000080000080008080008D5
:10FDEE0010181818101010181010181018181018C5
:10FDFE0010181818101010181010181018181018B5
:10FE0E0010181818101010181010181018181018A4
:10FE1E001018181810101018101018101818101894
:10FE2E000008080800000008000008000808000884
:10FE3E000008080800000008000008000808000874
:10FE4E001018181810101018101018101818101864
:10FE5E000000AA60AF60CD60D660FB6015611E61C8
:10FE6E0051617161B761EA61434C4F4E4500256C9B
:10FE7E007500546F6F206D616E7920646174612E10
:10FE8E00000D0A000D0A5041524954592045525254
:10FE9E004F52000D0A504152495459204F4B0025E4
:10FEAE0034753A200025337500556E6B6E6F776E84
:10FEBE00206361726420747970652E002573206F43
:10FECE007220004D756C7469706C6520706F737361
:10FEDE006962696C69746965732C206E6F74206336
:10FEEE006C6F6E61626C652100436C6F6E65642091
:10FEFE004F4B2100436C6F6E6520756E737570707D
:10FF0E006F7274656421004E4F20444154410000CD
:020000021000EC
:10000000BC59FC0F160804000138E31F63B2971DAA
:1000100000000000000000000000000000000000E0
:1000200000000000000000000000000000000000D0
:10003000FFFFFFFFFFFFFF078069FFFFFFFFFFFFDD
:1000400000000000000000000000000000000000B0
:1000500000000000000000000000000000000000A0
:100060000000000000000000000000000000000090
:10007000FFFFFFFFFFFFFF078069FFFFFFFFFFFF9D
:100080000000000000000000000000000000000070
:100090000000000000000000000000000000000060
:1000A0000000000000000000000000000000000050
:1000B000FFFFFFFFFFFFFF078069FFFFFFFFFFFF5D
:1000C0000000000000000000000000000000000030
:1000D0000000000000000000000000000000000020
:1000E0000000000000000000000000000000000010
:1000F000FFFFFFFFFFFFFF078069FFFFFFFFFFFF1D
:1001000000000000000000000000000000000000EF
:1001100000000000000000000000000000000000DF
:1001200000000000000000000000000000000000CF
:10013000FFFFFFFFFFFFFF078069FFFFFFFFFFFFDC
:1001400000000000000000000000000000000000AF
:10015000000000000000000000000000000000009F
:10016000000000000000000000000000000000008F
:10017000FFFFFFFFFFFFFF078069FFFFFFFFFFFF9C
:10018000000000000000000000000000000000006F
:10019000000000000000000000000000000000005F
:1001A000000000000000000000000000000000004F
:1001B000FFFFFFFFFFFFFF078069FFFFFFFFFFFF5C
:1001C000000000000000000000000000000000002F
:1001D000000000000000000000000000000000001F
:1001E000000000000000000000000000000000000F
:1001F000FFFFFFFFFFFFFF078069FFFFFFFFFFFF1C
:1002000000000000000000000000000000000000EE
:1002100000000000000000000000000000000000DE
:1002200000000000000000000000000000000000CE
:10023000FFFFFFFFFFFFFF078069FFFFFFFFFFFFDB
:1002400000000000000000000000000000000000AE
:10025000000000000000000000000000000000009E
:10026000000000000000000000000000000000008E
:10027000FFFFFFFFFFFFFF078069FFFFFFFFFFFF9B
:10028000000000000000000000000000000000006E
:10029000000000000000000000000000000000005E
:1002A000000000000000000000000000000000004E
:1002B000FFFFFFFFFFFFFF078069FFFFFFFFFFFF5B
:1002C000000000000000000000000000000000002E
:1002D000000000000000000000000000000000001E
:1002E000000000000000000000000000000000000E
:1002F000FFFFFFFFFFFFFF078069FFFFFFFFFFFF1B
:1003000000000000000000000000000000000000ED
:1003100000000000000000000000000000000000DD
:1003200000000000000000000000000000000000CD
:10033000FFFFFFFFFFFFFF078069FFFFFFFFFFFFDA
:1003400000000000000000000000000000000000AD
:10035000000000000000000000000000000000009D
:10036000000000000000000000000000000000008D
:10037000FFFFFFFFFFFFFF078069FFFFFFFFFFFF9A
:10038000000000000000000000000000000000006D
:10039000000000000000000000000000000000005D
:1003A000000000000000000000000000000000004D
:1003B000FFFFFFFFFFFFFF078069FFFFFFFFFFFF5A
:1003C000000000000000000000000000000000002D
:1003D000000000000000000000000000000000001D
:1003E000000000000000000000000000000000000D
:1003F000FFFFFFFFFFFFFF078069FFFFFFFFFFFF1A
:10040000FFFFFFFFFFFFFFFFFFFFFFFFFFFFFFFFFC
:10041000FFFFFFFFFFFFFFFFFFFFFFFFFFFFFFFFEC
:10042000FFFFFFFFFFFFFFFFFFFFFFFFFFFFFFFFDC
:10043000FFFFFFFFFFFFFFFFFFFFFFFFFFFFFFFFCC
:10200000123456780819040062636465666768696B
:1020100000000000000000000000000000000000C0
:1020200000000000000000000000000000000000B0
:10203000FFFFFFFFFFFFFF078069FFFFFFFFFFFFBD
:102040000000000000000000000000000000000090
:102050000000000000000000000000000000000080
:102060000000000000000000000000000000000070
:10207000FFFFFFFFFFFFFF078069FFFFFFFFFFFF7D
:102080000000000000000000000000000000000050
:102090000000000000000000000000000000000040
:1020A0000000000000000000000000000000000030
:1020B000FFFFFFFFFFFFFF078069FFFFFFFFFFFF3D
:1020C0000000000000000000000000000000000010
:1020D0000000000000000000000000000000000000
:1020E00000000000000000000000000000000000F0
:1020F000FFFFFFFFFFFFFF078069FFFFFFFFFFFFFD
:1021000000000000000000000000000000000000CF
:1021100000000000000000000000000000000000BF
:1021200000000000000000000000000000000000AF
:10213000FFFFFFFFFFFFFF078069FFFFFFFFFFFFBC
:10214000000000000000000000000000000000008F
:10215000000000000000000000000000000000007F
:10216000000000000000000000000000000000006F
:10217000FFFFFFFFFFFFFF078069FFFFFFFFFFFF7C
:10218000000000000000000000000000000000004F
:10219000000000000000000000000000000000003F
:1021A000000000000000000000000000000000002F
:1021B000FFFFFFFFFFFFFF078069FFFFFFFFFFFF3C
:1021C000000000000000000000000000000000000F
:1021D00000000000000000000000000000000000FF
:1021E00000000000000000000000000000000000EF
:1021F000FFFFFFFFFFFFFF078069FFFFFFFFFFFFFC
:1022000000000000000000000000000000000000CE
:1022100000000000000000000000000000000000BE
:1022200000000000000000000000000000000000AE
:10223000FFFFFFFFFFFFFF078069FFFFFFFFFFFFBB
:10224000000000000000000000000000000000008E
:10225000000000000000000000000000000000007E
:10226000000000000000000000000000000000006E
:10227000FFFFFFFFFFFFFF078069FFFFFFFFFFFF7B
:10228000000000000000000000000000000000004E
:10229000000000000000000000000000000000003E
:1022A000000000000000000000000000000000002E
:1022B000FFFFFFFFFFFFFF078069FFFFFFFFFFFF3B
:1022C000000000000000000000000000000000000E
:1022D00000000000000000000000000000000000FE
:1022E00000000000000000000000000000000000EE
:1022F000FFFFFFFFFFFFFF078069FFFFFFFFFFFFFB
:1023000000000000000000000000000000000000CD
:1023100000000000000000000000000000000000BD
:1023200000000000000000000000000000000000AD
:10233000FFFFFFFFFFFFFF078069FFFFFFFFFFFFBA
:10234000000000000000000000000000000000008D
:10235000000000000000000000000000000000007D
:10236000000000000000000000000000000000006D
:10237000FFFFFFFFFFFFFF078069FFFFFFFFFFFF7A
:10238000000000000000000000000000000000004D
:10239000000000000000000000000000000000003D
:1023A000000000000000000000000000000000002D
:1023B000FFFFFFFFFFFFFF078069FFFFFFFFFFFF3A
:1023C000000000000000000000000000000000000D
:1023D00000000000000000000000000000000000FD
:1023E00000000000000000000000000000000000ED
:1023F000FFFFFFFFFFFFFF078069FFFFFFFFFFFFFA
:10240000FFFFFFFFFFFFFFFFFFFFFFFFFFFFFFFFDC
:10241000FFFFFFFFFFFFFFFFFFFFFFFFFFFFFFFFCC
:10242000FFFFFFFFFFFFFFFFFFFFFFFFFFFFFFFFBC
:10243000FFFFFFFFFFFFFFFFFFFFFFFFFFFFFFFFAC
:10400000123456780819440062636465666768690B
:1040100000000000000000000000000000000000A0
:104020000000000000000000000000000000000090
:10403000FFFFFFFFFFFFFF078069FFFFFFFFFFFF9D
:104040000000000000000000000000000000000070
:104050000000000000000000000000000000000060
:104060000000000000000000000000000000000050
:10407000FFFFFFFFFFFFFF078069FFFFFFFFFFFF5D
:104080000000000000000000000000000000000030
:104090000000000000000000000000000000000020
:1040A0000000000000000000000000000000000010
:1040B000FFFFFFFFFFFFFF078069FFFFFFFFFFFF1D
:1040C00000000000000000000000000000000000F0
:1040D00000000000000000000000000000000000E0
:1040E00000000000000000000000000000000000D0
:1040F000FFFFFFFFFFFFFF078069FFFFFFFFFFFFDD
:1041000000000000000000000000000000000000AF
:10411000000000000000000000000000000000009F
:10412000000000000000000000000000000000008F
:10413000FFFFFFFFFFFFFF078069FFFFFFFFFFFF9C
:10414000000000000000000000000000000000006F
:10415000000000000000000000000000000000005F
:10416000000000000000000000000000000000004F
:10417000FFFFFFFFFFFFFF078069FFFFFFFFFFFF5C
:10418000000000000000000000000000000000002F
:10419000000000000000000000000000000000001F
:1041A000000000000000000000000000000000000F
:1041B000FFFFFFFFFFFFFF078069FFFFFFFFFFFF1C
:1041C00000000000000000000000000000000000EF
:1041D00000000000000000000000000000000000DF
:1041E00000000000000000000000000000000000CF
:1041F000FFFFFFFFFFFFFF078069FFFFFFFFFFFFDC
:1042000000000000000000000000000000000000AE
:10421000000000000000000000000000000000009E
:10422000000000000000000000000000000000008E
:10423000FFFFFFFFFFFFFF078069FFFFFFFFFFFF9B
:10424000000000000000000000000000000000006E
:10425000000000000000000000000000000000005E
:10426000000000000000000000000000000000004E
:10427000FFFFFFFFFFFFFF078069FFFFFFFFFFFF5B
:10428000000000000000000000000000000000002E
:10429000000000000000000000000000000000001E
:1042A000000000000000000000000000000000000E
:1042B000FFFFFFFFFFFFFF078069FFFFFFFFFFFF1B
:1042C00000000000000000000000000000000000EE
:1042D00000000000000000000000000000000000DE
:1042E00000000000000000000000000000000000CE
:1042F000FFFFFFFFFFFFFF078069FFFFFFFFFFFFDB
:1043000000000000000000000000000000000000AD
:10431000000000000000000000000000000000009D
:10432000000000000000000000000000000000008D
:10433000FFFFFFFFFFFFFF078069FFFFFFFFFFFF9A
:10434000000000000000000000000000000000006D
:10435000000000000000000000000000000000005D
:10436000000000000000000000000000000000004D
:10437000FFFFFFFFFFFFFF078069FFFFFFFFFFFF5A
:10438000000000000000000000000000000000002D
:10439000000000000000000000000000000000001D
:1043A000000000000000000000000000000000000D
:1043B000FFFFFFFFFFFFFF078069FFFFFFFFFFFF1A
:1043C00000000000000000000000000000000000ED
:1043D00000000000000000000000000000000000DD
:1043E00000000000000000000000000000000000CD
:1043F000FFFFFFFFFFFFFF078069FFFFFFFFFFFFDA
:10440000FFFFFFFFFFFFFFFFFFFFFFFFFFFFFFFFBC
:10441000FFFFFFFFFFFFFFFFFFFFFFFFFFFFFFFFAC
:10442000FFFFFFFFFFFFFFFFFFFFFFFFFFFFFFFF9C
:10443000FFFFFFFFFFFFFFFFFFFFFFFFFFFFFFFF8C
:10600000123456780808040062636465666768693C
:106010000000000000000000000000000000000080
:106020000000000000000000000000000000000070
:10603000FFFFFFFFFFFFFF078069FFFFFFFFFFFF7D
:106040000000000000000000000000000000000050
:106050000000000000000000000000000000000040
:106060000000000000000000000000000000000030
:10607000FFFFFFFFFFFFFF078069FFFFFFFFFFFF3D
:106080000000000000000000000000000000000010
:106090000000000000000000000000000000000000
:1060A00000000000000000000000000000000000F0
:1060B000FFFFFFFFFFFFFF078069FFFFFFFFFFFFFD
:1060C00000000000000000000000000000000000D0
:1060D00000000000000000000000000000000000C0
:1060E00000000000000000000000000000000000B0
:1060F000FFFFFFFFFFFFFF078069FFFFFFFFFFFFBD
:10610000000000000000000000000000000000008F
:10611000000000000000000000000000000000007F
:10612000000000000000000000000000000000006F
:10613000FFFFFFFFFFFFFF078069FFFFFFFFFFFF7C
:10614000000000000000000000000000000000004F
:10615000000000000000000000000000000000003F
:10616000000000000000000000000000000000002F
:10617000FFFFFFFFFFFFFF078069FFFFFFFFFFFF3C
:10618000000000000000000000000000000000000F
:1061900000000000000000000000000000000000FF
:1061A00000000000000000000000000000000000EF
:1061B000FFFFFFFFFFFFFF078069FFFFFFFFFFFFFC
:1061C00000000000000000000000000000000000CF
:1061D00000000000000000000000000000000000BF
:1061E00000000000000000000000000000000000AF
:1061F000FFFFFFFFFFFFFF078069FFFFFFFFFFFFBC
:10620000000000000000000000000000000000008E
:10621000000000000000000000000000000000007E
:10622000000000000000000000000000000000006E
:10623000FFFFFFFFFFFFFF078069FFFFFFFFFFFF7B
:10624000000000000000000000000000000000004E
:10625000000000000000000000000000000000003E
:10626000000000000000000000000000000000002E
:10627000FFFFFFFFFFFFFF078069FFFFFFFFFFFF3B
:10628000000000000000000000000000000000000E
:1062900000000000000000000000000000000000FE
:1062A00000000000000000000000000000000000EE
:1062B000FFFFFFFFFFFFFF078069FFFFFFFFFFFFFB
:1062C00000000000000000000000000000000000CE
:1062D00000000000000000000000000000000000BE
:1062E00000000000000000000000000000000000AE
:1062F000FFFFFFFFFFFFFF078069FFFFFFFFFFFFBB
:10630000000000000000000000000000000000008D
:10631000000000000000000000000000000000007D
:10632000000000000000000000000000000000006D
:10633000FFFFFFFFFFFFFF078069FFFFFFFFFFFF7A
:10634000000000000000000000000000000000004D
:10635000000000000000000000000000000000003D
:10636000000000000000000000000000000000002D
:10637000FFFFFFFFFFFFFF078069FFFFFFFFFFFF3A
:10638000000000000000000000000000000000000D
:1063900000000000000000000000000000000000FD
:1063A00000000000000000000000000000000000ED
:1063B000FFFFFFFFFFFFFF078069FFFFFFFFFFFFFA
:1063C00000000000000000000000000000000000CD
:1063D00000000000000000000000000000000000BD
:1063E00000000000000000000000000000000000AD
:1063F000FFFFFFFFFFFFFF078069FFFFFFFFFFFFBA
:10640000FFFFFFFFFFFFFFFFFFFFFFFFFFFFFFFF9C
:10641000FFFFFFFFFFFFFFFFFFFFFFFFFFFFFFFF8C
:10642000FFFFFFFFFFFFFFFFFFFFFFFFFFFFFFFF7C
:10643000FFFFFFFFFFFFFFFFFFFFFFFFFFFFFFFF6C
:10800000123456780808040062636465666768691C
:108010000000000000000000000000000000000060
:108020000000000000000000000000000000000050
:10803000FFFFFFFFFFFFFF078069FFFFFFFFFFFF5D
:108040000000000000000000000000000000000030
:108050000000000000000000000000000000000020
:108060000000000000000000000000000000000010
:10807000FFFFFFFFFFFFFF078069FFFFFFFFFFFF1D
:1080800000000000000000000000000000000000F0
:1080900000000000000000000000000000000000E0
:1080A00000000000000000000000000000000000D0
:1080B000FFFFFFFFFFFFFF078069FFFFFFFFFFFFDD
:1080C00000000000000000000000000000000000B0
:1080D00000000000000000000000000000000000A0
:1080E0000000000000000000000000000000000090
:1080F000FFFFFFFFFFFFFF078069FFFFFFFFFFFF9D
:10810000000000000000000000000000000000006F
:10811000000000000000000000000000000000005F
:10812000000000000000000000000000000000004F
:10813000FFFFFFFFFFFFFF078069FFFFFFFFFFFF5C
:10814000000000000000000000000000000000002F
:10815000000000000000000000000000000000001F
:10816000000000000000000000000000000000000F
:10817000FFFFFFFFFFFFFF078069FFFFFFFFFFFF1C
:1081800000000000000000000000000000000000EF
:1081900000000000000000000000000000000000DF
:1081A00000000000000000000000000000000000CF
:1081B000FFFFFFFFFFFFFF078069FFFFFFFFFFFFDC
:1081C00000000000000000000000000000000000AF
:1081D000000000000000000000000000000000009F
:1081E000000000000000000000000000000000008F
:1081F000FFFFFFFFFFFFFF078069FFFFFFFFFFFF9C
:10820000000000000000000000000000000000006E
:10821000000000000000000000000000000000005E
:10822000000000000000000000000000000000004E
:10823000FFFFFFFFFFFFFF078069FFFFFFFFFFFF5B
:10824000000000000000000000000000000000002E
:10825000000000000000000000000000000000001E
:10826000000000000000000000000000000000000E
:10827000FFFFFFFFFFFFFF078069FFFFFFFFFFFF1B
:1082800000000000000000000000000000000000EE
:1082900000000000000000000000000000000000DE
:1082A00000000000000000000000000000000000CE
:1082B000FFFFFFFFFFFFFF078069FFFFFFFFFFFFDB
:1082C00000000000000000000000000000000000AE
:1082D000000000000000000000000000000000009E
:1082E000000000000000000000000000000000008E
:1082F000FFFFFFFFFFFFFF078069FFFFFFFFFFFF9B
:10830000000000000000000000000000000000006D
:10831000000000000000000000000000000000005D
:10832000000000000000000000000000000000004D
:10833000FFFFFFFFFFFFFF078069FFFFFFFFFFFF5A
:10834000000000000000000000000000000000002D
:10835000000000000000000000000000000000001D
:10836000000000000000000000000000000000000D
:10837000FFFFFFFFFFFFFF078069FFFFFFFFFFFF1A
:1083800000000000000000000000000000000000ED
:1083900000000000000000000000000000000000DD
:1083A00000000000000000000000000000000000CD
:1083B000FFFFFFFFFFFFFF078069FFFFFFFFFFFFDA
:1083C00000000000000000000000000000000000AD
:1083D000000000000000000000000000000000009D
:1083E000000000000000000000000000000000008D
:1083F000FFFFFFFFFFFFFF078069FFFFFFFFFFFF9A
:10840000FFFFFFFFFFFFFFFFFFFFFFFFFFFFFFFF7C
:10841000FFFFFFFFFFFFFFFFFFFFFFFFFFFFFFFF6C
:10842000FFFFFFFFFFFFFFFFFFFFFFFFFFFFFFFF5C
:10843000FFFFFFFFFFFFFFFFFFFFFFFFFFFFFFFF4C
:10A0000012345678080804006263646566676869FC
:10A010000000000000000000000000000000000040
:10A020000000000000000000000000000000000030
:10A03000FFFFFFFFFFFFFF078069FFFFFFFFFFFF3D
:10A040000000000000000000000000000000000010
:10A050000000000000000000000000000000000000
:10A0600000000000000000000000000000000000F0
:10A07000FFFFFFFFFFFFFF078069FFFFFFFFFFFFFD
:10A0800000000000000000000000000000000000D0
:10A0900000000000000000000000000000000000C0
:10A0A00000000000000000000000000000000000B0
:10A0B000FFFFFFFFFFFFFF078069FFFFFFFFFFFFBD
:10A0C0000000000000000000000000000000000090
:10A0D0000000000000000000000000000000000080
:10A0E0000000000000000000000000000000000070
:10A0F000FFFFFFFFFFFFFF078069FFFFFFFFFFFF7D
:10A10000000000000000000000000000000000004F
:10A11000000000000000000000000000000000003F
:10A12000000000000000000000000000000000002F
:10A13000FFFFFFFFFFFFFF078069FFFFFFFFFFFF3C
:10A14000000000000000000000000000000000000F
:10A1500000000000000000000000000000000000FF
:10A1600000000000000000000000000000000000EF
:10A17000FFFFFFFFFFFFFF078069FFFFFFFFFFFFFC
:10A1800000000000000000000000000000000000CF
:10A1900000000000000000000000000000000000BF
:10A1A00000000000000000000000000000000000AF
:10A1B000FFFFFFFFFFFFFF078069FFFFFFFFFFFFBC
:10A1C000000000000000000000000000000000008F
:10A1D000000000000000000000000000000000007F
:10A1E000000000000000000000000000000000006F
:10A1F000FFFFFFFFFFFFFF078069FFFFFFFFFFFF7C
:10A20000000000000000000000000000000000004E
:10A21000000000000000000000000000000000003E
:10A22000000000000000000000000000000000002E
:10A23000FFFFFFFFFFFFFF078069FFFFFFFFFFFF3B
:10A24000000000000000000000000000000000000E
:10A2500000000000000000000000000000000000FE
:10A2600000000000000000000000000000000000EE
:10A27000FFFFFFFFFFFFFF078069FFFFFFFFFFFFFB
:10A2800000000000000000000000000000000000CE
:10A2900000000000000000000000000000000000BE
:10A2A00000000000000000000000000000000000AE
:10A2B000FFFFFFFFFFFFFF078069FFFFFFFFFFFFBB
:10A2C000000000000000000000000000000000008E
:10A2D000000000000000000000000000000000007E
:10A2E000000000000000000000000000000000006E
:10A2F000FFFFFFFFFFFFFF078069FFFFFFFFFFFF7B
:10A30000000000000000000000000000000000004D
:10A31000000000000000000000000000000000003D
:10A32000000000000000000000000000000000002D
:10A33000FFFFFFFFFFFFFF078069FFFFFFFFFFFF3A
:10A34000000000000000000000000000000000000D
:10A3500000000000000000000000000000000000FD
:10A3600000000000000000000000000000000000ED
:10A37000FFFFFFFFFFFFFF078069FFFFFFFFFFFFFA
:10A3800000000000000000000000000000000000CD
:10A3900000000000000000000000000000000000BD
:10A3A00000000000000000000000000000000000AD
:10A3B000FFFFFFFFFFFFFF078069FFFFFFFFFFFFBA
:10A3C000000000000000000000000000000000008D
:10A3D000000000000000000000000000000000007D
:10A3E000000000000000000000000000000000006D
:10A3F000FFFFFFFFFFFFFF078069FFFFFFFFFFFF7A
:10A40000FFFFFFFFFFFFFFFFFFFFFFFFFFFFFFFF5C
:10A41000FFFFFFFFFFFFFFFFFFFFFFFFFFFFFFFF4C
:10A42000FFFFFFFFFFFFFFFFFFFFFFFFFFFFFFFF3C
:10A43000FFFFFFFFFFFFFFFFFFFFFFFFFFFFFFFF2C
:10C0000012345678080804006263646566676869DC
:10C010000000000000000000000000000000000020
:10C020000000000000000000000000000000000010
:10C03000FFFFFFFFFFFFFF078069FFFFFFFFFFFF1D
:10C0400000000000000000000000000000000000F0
:10C0500000000000000000000000000000000000E0
:10C0600000000000000000000000000000000000D0
:10C07000FFFFFFFFFFFFFF078069FFFFFFFFFFFFDD
:10C0800000000000000000000000000000000000B0
:10C0900000000000000000000000000000000000A0
:10C0A0000000000000000000000000000000000090
:10C0B000FFFFFFFFFFFFFF078069FFFFFFFFFFFF9D
:10C0C0000000000000000000000000000000000070
:10C0D0000000000000000000000000000000000060
:10C0E0000000000000000000000000000000000050
:10C0F000FFFFFFFFFFFFFF078069FFFFFFFFFFFF5D
:10C10000000000000000000000000000000000002F
:10C11000000000000000000000000000000000001F
:10C12000000000000000000000000000000000000F
:10C13000FFFFFFFFFFFFFF078069FFFFFFFFFFFF1C
:10C1400000000000000000000000000000000000EF
:10C1500000000000000000000000000000000000DF
:10C1600000000000000000000000000000000000CF
:10C17000FFFFFFFFFFFFFF078069FFFFFFFFFFFFDC
:10C1800000000000000000000000000000000000AF
:10C19000000000000000000000000000000000009F
:10C1A000000000000000000000000000000000008F
:10C1B000FFFFFFFFFFFFFF078069FFFFFFFFFFFF9C
:10C1C000000000000000000000000000000000006F
:10C1D000000000000000000000000000000000005F
:10C1E000000000000000000000000000000000004F
:10C1F000FFFFFFFFFFFFFF078069FFFFFFFFFFFF5C
:10C20000000000000000000000000000000000002E
:10C21000000000000000000000000000000000001E
:10C22000000000000000000000000000000000000E
:10C23000FFFFFFFFFFFFFF078069FFFFFFFFFFFF1B
:10C2400000000000000000000000000000000000EE
:10C2500000000000000000000000000000000000DE
:10C2600000000000000000000000000000000000CE
:10C27000FFFFFFFFFFFFFF078069FFFFFFFFFFFFDB
:10C2800000000000000000000000000000000000AE
:10C29000000000000000000000000000000000009E
:10C2A000000000000000000000000000000000008E
:10C2B000FFFFFFFFFFFFFF078069FFFFFFFFFFFF9B
:10C2C000000000000000000000000000000000006E
:10C2D000000000000000000000000000000000005E
:10C2E000000000000000000000000000000000004E
:10C2F000FFFFFFFFFFFFFF078069FFFFFFFFFFFF5B
:10C30000000000000000000000000000000000002D
:10C31000000000000000000000000000000000001D
:10C32000000000000000000000000000000000000D
:10C33000FFFFFFFFFFFFFF078069FFFFFFFFFFFF1A
:10C3400000000000000000000000000000000000ED
:10C3500000000000000000000000000000000000DD
:10C3600000000000000000000000000000000000CD
